:020000040800F2
:1000000000500020316801080000000000000000DE
:10001000656801086568010865680108000000005E
:1000200000000000000000000000000065680108FA
:100030006568010800000000656801085147010873
:100040006568010865680108656801086568010858
:100050006568010865680108656801086568010848
:100060006568010865680108656801086568010838
:100070006568010865680108656801086568010828
:100080006568010865680108656801086568010818
:100090006568010865680108656801086568010808
:1000A00065680108656801086568010865680108F8
:1000B0001D5E0108C55801086568010865680108EA
:1000C00065680108656801086568010865680108D8
:1000D000656801088156010865680108195701081B
:1000E000656801086568010865680108000000008E
:1000F0000000000000000000000000000000000000
:1001000000000000000000005FF808F170B542F246
:10011000FB16C3F6E97621F00044B44286B00246ED
:100120000B461ADD4FF6FF75C7F6EF75AC4203DDDF
:1001300001F028FF06B070BD02AA00F07DF800F0C3
:100140000303012B17D0022B0CD0F3B9DDE9020118
:10015000DDE9042300F098FAECE70022002300F028
:1001600093FAE7E7DDE90201DDE9042300F08CFA08
:1001700001F10041DEE70093DDE90201DDE904233E
:1001800000F07EFF01F10041D4E70123DDE9020127
:100190000093DDE9042300F073FFCBE770B542F272
:1001A000FB16C3F6E97621F00044B44286B002465D
:1001B0000B461CDD4FF6FF75C7F6EF75AC4203DD4D
:1001C00001F0E0FE06B070BD02AA00F035F800F0C4
:1001D000030001281DD0022810D008BB0123DDE94F
:1001E00002010093DDE9042300F04AFFEAE7002260
:1001F00000230024009400F043FFE3E70123DDE93E
:1002000002010093DDE9042300F03AFF01F100410F
:10021000D8E7DDE90201DDE9042300F035FAD1E792
:10022000DDE90201DDE9042300F02EFA01F10041CD
:10023000C8E700BF0000000042F2FB132DE9F04FB9
:10024000C3F6E97321F000448DB09C428046894694
:100250000E46154640F3A7804DF67B13C4F2020309
:100260009C4226DC002940F3AD8191A3D3E9002311
:1002700001F088FE42F2FB13C3F6F9739C428046FC
:10028000894600F0A5808CA3D3E90023012701F063
:1002900079FE02460B46C5E900014046494601F099
:1002A00071FE85A3D3E9002301F06CFEC5E90201CC
:1002B00080E042F2FB13C4F239139C4240F3A58064
:1002C0004FF6FF73C7F6EF739C4277DC4FEA245B6F
:1002D0000246ABF5826BABF1060B4FEA0B51631A8A
:1002E000CDE90223194602F09BFA01F099FF8046FE
:1002F000894602460B46DDE90201CDE9068901F097
:1003000041FE00230022C4F2701301F0EFFFCDE99B
:10031000020102F085FA01F083FF02460B46804697
:100320008946DDE90201CDE9088901F02BFE0023B1
:100330000022C4F2701301F0D9FF00220023CDE99E
:100340000A0102F03BFA002800F060810DF1180A62
:10035000032440464946002200230AF10807013CD5
:1003600002F02CFA40B177E9020100220023013C9F
:1003700002F024FA0028F6D12346574C504629466D
:100380005A4601940224009400F0A6FA002E074673
:1003900010DA6A68474202F100426A60EA6802F1D4
:1003A0000042EA6006E00027C2E90089002300223B
:1003B000C5E9022338460DB0BDE8F08F02460B4672
:1003C00001F0E0FD0027C5E90201C5E90001F1E700
:1003D0003BA3D3E90023012701F0D4FD3AA3D3E9DD
:1003E00000238046894601F0CDFD02460B46C5E953
:1003F00000014046494601F0C5FD33A3D3E900237F
:1004000001F0C0FDC5E90201D4E700F0EDFE30A324
:10041000D3E900238046894601F068FF00230022CB
:10042000C3F6E07301F0B0FD02F0FAF9074601F0FF
:10043000F7FE1FA3D3E90023CDE9020101F056FF27
:1004400002460B464046494601F09CFD1AA3D3E9FB
:10045000002380468946DDE9020101F047FF1F2F96
:1004600082468B463ADC49F698537A1EC0F6010361
:1004700053F82230A34231D052465B4640464946AB
:1004800001F080FD02460B46C5E90023404649467F
:1004900001F078FD52465B4601F074FD002EC5E97F
:1004A000020187DA6A687F4275E700BFAFF3008018
:1004B00000004054FB21F93F3163621A61B4D03D22
:1004C0000000601A61B4D03D7370032E8A19A33BFB
:1004D00083C8C96D305FE43F189E010852465B46F1
:1004E0004046494601F04EFD24150B46C1F30A5122
:1004F000611A02461029C5E90023C7DD56A3D3E9D6
:100500000023DDE9020101F0F1FE82468B465246EE
:100510005B464046494601F035FDCDE904014046C1
:10052000DDE90423494601F02DFD52465B4601F00A
:1005300029FD4BA3D3E9002380468946DDE902016A
:1005400001F0D4FE42464B4601F01CFD82468B462C
:100550005246DDE904015B4601F014FD0B46C1F390
:100560000A51641A0246312CC5E9002370DD3EA30E
:10057000D3E90023DDE9020101F0B8FE82468B4693
:1005800052465B46DDE9040101F0FCFC80468946E9
:1005900042464B46DDE9040101F0F4FC52465B465D
:1005A00001F0F0FC32A3D3E9002382468B46DDE95B
:1005B000020101F09BFE52465B4601F0E3FC8246DD
:1005C0008B4659E72CA3D3E9002301F0DDFC42F26E
:1005D000FB13C3F6F9739C42804689461AD028A3C0
:1005E000D3E900234FF0FF3701F0CEFC02460B4663
:1005F000C5E900014046494601F0C4FC20A3D3E907
:10060000002301F0C1FCC5E90201D3E603240DF18A
:10061000180AB1E610A3D3E900234FF0FF3701F029
:10062000B3FC0FA3D3E900238046894601F0ACFC5C
:1006300002460B46C5E900014046494601F0A2FCCE
:1006400007A3D3E9002301F09FFCC5E90201B1E64D
:10065000DDE904891AE700BF0000601A61B4D03DEB
:100660007370032E8A19A33B0000002E8A19A33B46
:10067000C14920259A837B3900004054FB21F93F72
:100680003163621A61B4D03D2DE9F04F21F000468C
:1006900085B0B6F1795F80468946CDE900236DDAF1
:1006A00002F0BEF8002800F0F78042464B46404674
:1006B000494601F01BFE7CA3D3E9002304460D4606
:1006C00001F014FE7AA3D3E9002301F05DFC224679
:1006D0002B4601F00BFE78A3D3E9002301F052FC76
:1006E00022462B4601F002FE75A3D3E9002301F058
:1006F0004BFC22462B4601F0F9FD73A3D3E90023FE
:1007000001F040FC22462B4601F0F0FD70A3D3E936
:10071000002301F039FC22462B4601F0E7FD82461A
:100720008B460023002220462946C3F6E07301F0E1
:10073000DDFD52465B4606460F462046294601F03F
:10074000D5FDDDE9002304460D464046494601F04B
:10075000CDFD02460B462046294601F013FC024619
:100760000B463046394601F00DFC0B46002102468F
:10077000C3F6F071002001F005FC7FE002460B4655
:1007800001F0B4FD48A3D3E9002304460D4601F06F
:10079000ADFD47A3D3E9002301F0F6FB22462B462B
:1007A00001F0A4FD44A3D3E9002301F0EBFB2246B2
:1007B0002B4601F09BFD42A3D3E9002301F0E4FBAB
:1007C00022462B4601F092FD3FA3D3E9002301F01E
:1007D000D9FB22462B4601F089FD3DA3D3E9002336
:1007E00001F0D2FB2B46224601F080FD43F232336A
:1007F000C3F6D3739E4282468B4692DD0023C3F636
:10080000E9739E423DDC0021A6F500130022002082
:10081000C3F6F07116461F4601F0B4FBCDE90201A4
:100820000023204629460022C3F6E07301F05EFD56
:1008300032463B4601F0A6FB52465B4606460F4653
:100840002046294601F052FDDDE9002304460D460D
:100850004046494601F04AFD02460B4620462946DD
:1008600001F090FB02460B463046394601F08AFB08
:1008700002460B46DDE9020101F084FB05B0BDE84C
:10088000F08F002300270022C3F6E7730026CDE98E
:100890000223C3F6D277C3E700210020C3F6F0712C
:1008A000ECE700BFAFF30080D43888BEE9FAA8BDFA
:1008B000C4B1B4BD9EEE213EAD529C804F7E923EAF
:1008C0009015CB19A001FA3E7751C1166CC1563F65
:1008D0004C5555555555A53F2DE9F04FADF51B7DB0
:1008E000144649F620750590D01EA49AC0F601055D
:1008F000089118211F4655F82250099501F0E4F996
:100900007B1E18220393099D20EAE0700A90C343DE
:1009100002FB0342039C15EB040806921BD4041B44
:10092000A5985CAEA04400EB840509E02868043576
:1009300001F076FC444504F10104E6E902010AD025
:10094000002CF3DA0020002104354445E6E90201D9
:1009500004F10104F4D109990029C0F26883099CCB
:10096000BA460DF1300B0EAB079303EBC4040194B0
:10097000DDF80CE0BEF1000FBCBF4FF000084FF0F7
:10098000000919DB5EA8059E00EBCA054FF00008C0
:100990004FF00009002475E902230134F6E8020152
:1009A00001F0A4FC02460B464046494601F0ECFA31
:1009B000BC4280468946EED1019E0AF1010AEBE96C
:1009C0000289B345D4D1099986AA9AAC4B1E0E462A
:1009D00002EB81020C929B000B93E4180D94079894
:1009E0004FEAC60E002ECDF804E000EB0E04D4E969
:1009F00000892EDD86A9BB460D1F82460296002384
:100A00000022C3F670634046494601F06FFC01F0D6
:100A100007FF01F005FC00230022C4F27013064614
:100A20000F4601F063FC02460B464046494601F082
:100A3000A9FA01F0F5FE32463B4645F8040F74E989
:100A4000020101F0A1FA544580468946D7D1029EA1
:100A50005F46069A4046494600F05EFC00224FF091
:100A60007F5304460D4601F041FC00F0C1FB00231A
:100A70000022C4F2200301F039FC02460B46204656
:100A8000294601F07FFA0D46044601F0C9FE824670
:100A900001F0C6FB02460B462046294601F072FAD9
:100AA000069A002A8046894640F3E480731E0DF5BD
:100AB0001A7EC2F11801C2F117040EEB830353F83A
:100AC000502C52FA01F0824410FA01F1521A43F804
:100AD000502C52FA04F5002D37DD002E0AF1010AE0
:100AE00040F3A18286AB002403EB860007E021B12E
:100AF0000124C1F1807143F8041C83420ED053F8E5
:100B0000041B002CF3D04FF6FF7201248342C0F285
:100B1000FF02C1EB020243F8042CF0D10699002930
:100B200011DD012900F0AE8002290CD1721E0DF5F5
:100B30001A7E0EEB820252F8503C23F07F4323F4DE
:100B4000400342F8503C022D77D0404649460022EF
:100B5000002301F033FE002800F0AC8009988642A3
:100B60000DDD86A90C9801EB8603002253F8041DC5
:100B7000834242EA0102F9D1002A40F0E4800D9A52
:100B800052F8503C002B40F050820B9B86ACE21890
:100B9000012352F8041D01330029FAD09B1906F1F4
:100BA000010A9A45049346DCDDF828E0F319A5987C
:100BB000013B7644019A07995EAC00EB860B04EB8F
:100BC000C3048918019402915BF8040F01F028FB1B
:100BD000DDF80CE0019EBEF1000FBCBF4FF0000835
:100BE0004FF00009E6E9020101961BDB0AEB07055D
:100BF0005EA8059E4FF000084FF00009002400EBAE
:100C0000C50575E902230134F6E8020101F06EFB27
:100C100002460B464046494601F0B6F9BC428046C2
:100C20008946EED1049A0AF1010A02999245E1E956
:100C300002890291C8DD049ED1E6002142464B465E
:100C40000020C3F6F07101F09DF980468946002C22
:100C50003FF47BAF0021069A0020C3F6F07100F04C
:100C60005BFB02460B464046494601F08BF9804645
:100C700089466AE713D19AA800EB860353F8545CBF
:100C8000ED1528E7721E9AAB03EB820252F8503C36
:100C900023F07F4323F4000342F8503C53E7002342
:100CA0000022C3F6E07301F0A7FD08B900254CE768
:100CB000022512E7CDF80CA00195002846D1DDF8F9
:100CC00018E040464946CEF1000200F025FB002323
:100CD0000022C4F2701304460D4601F08DFD002879
:100CE00000F0A88100230022C3F670632046294645
:100CF00006F1010B01F0FAFA9AAA02EB860701F05D
:100D00008FFD01F08DFA00230DF51A7E0022C4F24A
:100D100070130EEB8B068046894601F0E7FA0B460E
:100D200002462946204601F02DF9069A183206920D
:100D300001F076FD494647F8500C404601F070FD41
:100D400046F8500C19E0CDF80CA00195069B06F171
:100D5000FF3B9AAC183B06934FEA8B03E21852F81C
:100D6000502C52B986AE069AF31853F8041D0BF1B5
:100D7000FF3B183A0029F8D0069200210020C3F664
:100D8000F071069A00F0C8FABBF1000F06460F4654
:100D90005CDB0BF10105DDF81CE00DF5067808EBD6
:100DA00085040EEBC50554F8040D01F039FA3246FE
:100DB0003B4601F09BFA00230022C3F6706365E90D
:100DC00002013046394601F091FA444506460F4685
:100DD000E9D10DF1D80A0BF1FF33CDF808A00027B7
:100DE000DDF824A0CDF810B09B46BAF1000FC0F298
:100DF0001381002FC0F2108107994FF00008944E24
:100E00004FF0000901EBCB05002401E0BC4210DCEF
:100E1000F5E902230134F6E9020101F067FA02461E
:100E20000B464046494601F0AFF8A2458046894648
:100E3000ECDA02980BF1FF3B00EBC70301371BF123
:100E4000020FC3E90089D0D1DDF810B0A49A032ABB
:100E500022D8DFE812F0C3008200820028000027B9
:100E60000DF1D80A3E46019B002B00F0F880DAF81D
:100E7000000006F10046DAF80820089CDAF80410B1
:100E8000DAF80C3001F10041206003F100436160A9
:100E9000A260E36027616661039E06F007000DF51E
:100EA0001B7DBDE8F08FBBF1000FD8DD0DF1D80A36
:100EB0000AEBCB0454E9026774E8028930463946EC
:100EC00042464B4601F060F8C4E900013046D4E9DF
:100ED0000023394601F056F802460B464046494683
:100EE00001F052F85445C4E90201E3D1BBF1010F0E
:100EF00040F3C3800BF1FF340AEBC40474E80267CB
:100F000030463946D4E9042301F03EF8804689464C
:100F100042464B463046394601F034F802460B460D
:100F2000D4E9040101F030F85445C4E90289C4E968
:100F30000401E3D10BF1010400270AF110053E463C
:100F40000AEBC404384674E90223314601F01CF868
:100F5000AC4207460E46F5D185E7BBF1000F79DBC1
:100F60000BF101040DF1D80A00260AEBC404354642
:100F7000304674E90223294601F006F85445064636
:100F80000D46F5D1019800284BD005F100442146CB
:100F900032463446089E2B460D46DAE90001C6E982
:100FA000004500F0EFFFBBF1000F03460C460BDDE0
:100FB0000AEBCB0B18462146FAE9022300F0E4FFC6
:100FC000DA4503460C46F5D1019808B104F1004416
:100FD000089A18462146C2E902015DE7BBF1000FFD
:100FE00033DB0BF1010436AD002705EBC4043E46AC
:100FF000384674E90223314600F0C6FFAC4207468A
:101000000E46F5D1019C0CB106F100463346089E10
:101010003A46C6E900233FE74FF000084FF00009C9
:1010200007E72C46B3E7002478E50123B6E50EAACE
:101030000792C8E420469AAB294603EB860401F0E8
:10104000EFFBB34644F8500C97E600273E46D9E73D
:10105000289F010800260DF1D80A354692E7DAE903
:1010600000013346DAE902453A46089EC6E9042300
:10107000C6E90001C6E902450EE700273E46F2E652
:101080002DE9F04F9B4621F0004385B0B3F1795F25
:1010900004460D46924603DA01F0C2FB00286ED0EA
:1010A00022462B462046294601F020F922462B46AF
:1010B00006460F4601F01AF93FA3D3E90023804604
:1010C00089463046394601F011F93DA3D3E90023A2
:1010D00000F058FF32463B4601F008F93AA3D3E945
:1010E000002300F051FF32463B4601F0FFF838A3E1
:1010F000D3E9002300F046FF32463B4601F0F6F804
:1011000035A3D3E9002300F03FFF0E9BCDE900019A
:10111000002B39D000230022C3F6E0735046594615
:1011200001F0E4F8DDE90023CDE90201404649463B
:1011300001F0DCF802460B46DDE9020100F022FF77
:1011400032463B4601F0D2F852465B4600F01AFFA9
:1011500023A3D3E9002306460F464046494601F043
:10116000C5F802460B463046394600F00DFF0246F0
:101170000B462046294600F005FF04460D46204652
:10118000294605B0BDE8F08F02460B463046394689
:1011900001F0ACF812A3D3E9002300F0F3FE4246BD
:1011A0004B4601F0A3F802460B462046294600F0C4
:1011B000EBFE04460D46E2E77CD5CF5A3AD9E53D31
:1011C000EB9C2B8AE6E55A3E7DFEB157E31DC73EF8
:1011D000D561C119A0012A3FA6F810111111813F54
:1011E000495555555555C53F21F00041704700BF41
:1011F000C1F30A5C0246ACF57E7C0B462DE9F04754
:10120000ACF10704132C06460F468946804621DCC4
:10121000002C40DB4FF6FF7CC0F20F0C4CFA04FAB6
:101220000AEA0105054311D039A3D3E9002300F0F0
:10123000ABFE0022002301F0E9FA00283AD0002F8B
:101240005DDB29EA0A0900264B463246104619465C
:10125000BDE8F087332C07DDB4F5806FF6D100F0E0
:1012600093FE02460B46F1E74FF0FF35ACF11B0C45
:1012700025FA0CF50542E9D025A3D3E9002300F0B7
:1012800083FE0022002301F0C1FA98B1002F18DB81
:1012900026EA05060FE01EA3D3E9002300F074FE42
:1012A0000022002301F0B2FA28B1002F17DB00263C
:1012B000B14600E0B9464B46324610461946BDE8F5
:1012C000F087142C06D00126C4F13404A64016EB96
:1012D0000806DDD307F1010926EA0506EBE727F04A
:1012E00000454FF0000945EA0608CBF6F079B8F161
:1012F000000F08BFB9460CBF46460026DBE74FF497
:10130000801353FA04F407EB04099AE7AFF3008063
:101310009C7500883CE4377EF8B5C1F30A53044657
:101320000D4616460F46002B2BD121F000470743F0
:1013300024D000230022C4F2503343F6B04700F01B
:10134000D5FFCFF6FF77BE4204460D4639DBC1F329
:101350000A5340F2FE72363B0F469B19934219DD49
:1013600022462B462AA1D1E9000100F059F828A312
:10137000D3E9002300F0BAFF04460D462046294673
:10138000F8BD40F2FF72934225D09B1940F2FE72E5
:101390009342E5DC002BC2BF27F0FE4727F470071D
:1013A00047EA0355EADC13F1350F1DDA4CF25033EE
:1013B0009E42D5DC22462B4617A1D1E9000100F060
:1013C0002FF815A3D3E9002300F090FF04460D4643
:1013D00020462946F8BD02460B4600F0D5FD0446DE
:1013E0000D4620462946F8BD363327F0FE4727F440
:1013F0007007204647EA0355002329460022C3F61A
:10140000904300F073FF04460D46B7E7AFF300804A
:101410009C7500883CE4377E59F3F8C21F6EA50125
:1014200010B421F0004203F0004444EA020110BC71
:10143000704700BF00210A2200F0FCBA00220A23F4
:1014400000F046BA032A2DE9F00109D82AB1002399
:10145000CC5CC45401339342FAD1BDE8F00170472B
:101460000B468218014603E02478013301F8014B52
:1014700011F0030F1C46F7D113F003055DD06E4247
:10148000C5F1040CED009B594FEACC0C08E0043484
:10149000A7593B4607FA0CF748EA070741F8047BCF
:1014A000571A23FA05F8032FF1DC03E014F8013B87
:1014B00001F8013B8A42F9D8CFE753F8404C41F894
:1014C000404C53F83C4C41F83C4C53F8384C41F8F4
:1014D000384C53F8344C41F8344C53F8304C41F804
:1014E000304C53F82C4C41F82C4C53F8284C41F814
:1014F000284C53F8244C41F8244C53F8204C41F824
:10150000204C53F81C4C41F81C4C53F8184C41F833
:10151000184C53F8144C41F8144C53F8104C41F843
:10152000104C53F80C4C41F80C4C53F8084C41F853
:10153000084C53F8044C41F8044C561A1D460C460E
:10154000403340313F2EB8DC2B460FE053F8101CDF
:1015500044F8101C53F80C1C44F80C1C53F8081CDD
:1015600044F8081C53F8041C44F8041C161B2146BC
:101570001D46103410330F2EE8DC2B4602E02468A1
:1015800041F8044B551A1C46032D03F10403F6DC05
:1015900090E700BF032AC9B270B408D82AB1034645
:1015A000121803F8011B9342FBD170BC70478218DC
:1015B000044601E004F8011B14F0030FFAD14FF0C8
:1015C000013303FB01F31FE044F8403C44F83C3C8A
:1015D00044F8383C44F8343C44F8303C44F82C3C63
:1015E00044F8283C44F8243C44F8203C44F81C3C93
:1015F00044F8183C44F8143C44F8103C44F80C3CC3
:1016000044F8083C44F8043C161B254640343F2E61
:10161000DADC2C4607E044F8103C44F80C3C44F873
:10162000083C44F8043C161B254610340F2EF2DC0F
:1016300001E045F8043B541B032CFADC01E005F8FB
:10164000011B9542FBD3B0E710F0030F38B50446F9
:1016500012D10368A3F1013222EA030313F0803FA1
:101660000AD1031D184653F8042BA2F1013525EACF
:10167000020212F0803FF5D003782BB1431C1846CC
:1016800013F8012B002AFAD100F002F8204638BDE9
:1016900080EA0102844612F0030F4FD111F0030FCC
:1016A00032D14DF8044D11F0040F51F8043B0BD02A
:1016B000A3F101329A4312F0803F04BF4CF8043B7F
:1016C00051F8043B16D100BF51F8044BA3F101328D
:1016D0009A4312F0803FA4F101320BD14CF8043B45
:1016E000A24312F0803F04BF51F8043B4CF8044B76
:1016F000EAD023460CF8013B13F0FF0F4FEA3323E7
:10170000F8D15DF8044B704711F0010F06D011F8C5
:10171000012B0CF8012B002A08BF704711F0020FB3
:10172000BFD031F8022B12F0FF0F16BF2CF8022B9E
:101730008CF8002012F47F4FB3D1704711F8012BC1
:101740000CF8012B002AF9D1704700BF20F00301EB
:1017500010F00300C0F1000051F8043B00F1040C4C
:101760004FEACC0C6FF000021CBF22FA0CF21343BC
:101770004FF0010C4CEA0C2C4CEA0C4CA3EB0C0285
:1017800022EA030212EACC1204BF51F8043B0430EF
:10179000F4D013F0FF0F1FBF013013F47F4F01305F
:1017A00013F47F0F18BF0130704700BFF0B4002A58
:1017B00046D041EA000313F003032CD1032A074665
:1017C0000E4643D904680D68AC423FD1043A37D085
:1017D000A4F1013525EA040414F0803F18BF18462F
:1017E0002CD1041D0D1D0EE054F8043B55F8041BCC
:1017F000A3F101308B4220EA030027D1043A1FD025
:1018000010F0803F1ED1032A27462E46ECD82046F2
:101810002946002A1DD00478013A0D78AC420CD13B
:1018200072B18CB1002302E093420BD064B101335A
:1018300010F8014FCD5CAC42F6D0601BF0BC704795
:101840001046FBE70020F9E72046F7E73846314627
:10185000E1E724782D78F0E741EA000313F0030F65
:101860000B4670B414BF00240124032A94BF002443
:1018700004F001040546D4B9BAB10E782B46013AFA
:1018800003F8016B56B1AC1C7AB111F8015F234625
:10189000013A04F8015C0134002DF5D12AB19A18FF
:1018A000002103F8011B9342FBD170BC704719461D
:1018B00053F8044BA4F1013626EA040616F0803FE3
:1018C000DAD1043A45F8044B032A1946EFD8D3E796
:1018D0002DE9F04F40F20C24C2F2000485B01F46FF
:1018E0008C4626680B460390029213F8014B32197E
:1018F0001D4692F801B01BF0080BF6D12D2C73D0C9
:101900002B2C08BF15F8014BD7F1010338BF00237A
:10191000102F14BF1A4643F0010232B1302C73D09D
:101920001BB1302C00F083800A27B946BBF1000FB1
:1019300049460CBF6FF0004A4FF0004ACDF804C092
:10194000504600F0B3F950468846494600F080F80A
:1019500033190022DDF804C05B78114613F0040F40
:101960001ED0303CA74225DD814294BF00230123D5
:1019700053EAD2722ED10A1A534243EB0203444572
:10198000D4BF002303F00103002B23D109FB014145
:1019900015F8014B012233195B7813F0040FE0D1E5
:1019A00013F0030306D0012B14BF57233723E41A87
:1019B000A742D9DCB2F1FF3F1BD00846BBF1000FB4
:1019C00010D1029B1BB152B90299C1F800C005B0F9
:1019D000BDE8F08F4FF0FF3215F8014BDBE705F162
:1019E000FF3CF1E74842ECE715F8014B4FF0010BE3
:1019F0008AE70399BBF1000F0CBF6FF000404FF076
:101A0000004022230B60DCE72A78A2F178004142F3
:101A100041EB0001582A14BF0A4641F00102002A96
:101A20003FF47EAF10276C78B94602357EE7082771
:101A3000B9467BE730B440F21024C2F200040D46F0
:101A4000134601462A46206830BC41E700000000EA
:101A50004A1E08BF7047C0F02481884240F21681B8
:101A6000114200F01781B0FA80F3B1FA81F2A2EBD3
:101A70000303C3F11F0304A202EB03134FF00002A0
:101A80009F4600BFAFF30080B0EBC17F00BF42EBC9
:101A9000020228BFA0EBC170B0EB817F00BF42EB18
:101AA000020228BFA0EB8170B0EB417F00BF42EB88
:101AB000020228BFA0EB4170B0EB017F00BF42EBF8
:101AC000020228BFA0EB0170B0EBC16F00BF42EB78
:101AD000020228BFA0EBC160B0EB816F00BF42EBF8
:101AE000020228BFA0EB8160B0EB416F00BF42EB68
:101AF000020228BFA0EB4160B0EB016F00BF42EBD8
:101B0000020228BFA0EB0160B0EBC15F00BF42EB57
:101B1000020228BFA0EBC150B0EB815F00BF42EBD7
:101B2000020228BFA0EB8150B0EB415F00BF42EB47
:101B3000020228BFA0EB4150B0EB015F00BF42EBB7
:101B4000020228BFA0EB0150B0EBC14F00BF42EB37
:101B5000020228BFA0EBC140B0EB814F00BF42EBB7
:101B6000020228BFA0EB8140B0EB414F00BF42EB27
:101B7000020228BFA0EB4140B0EB014F00BF42EB97
:101B8000020228BFA0EB0140B0EBC13F00BF42EB17
:101B9000020228BFA0EBC130B0EB813F00BF42EB97
:101BA000020228BFA0EB8130B0EB413F00BF42EB07
:101BB000020228BFA0EB4130B0EB013F00BF42EB77
:101BC000020228BFA0EB0130B0EBC12F00BF42EBF7
:101BD000020228BFA0EBC120B0EB812F00BF42EB77
:101BE000020228BFA0EB8120B0EB412F00BF42EBE7
:101BF000020228BFA0EB4120B0EB012F00BF42EB57
:101C0000020228BFA0EB0120B0EBC11F00BF42EBD6
:101C1000020228BFA0EBC110B0EB811F00BF42EB56
:101C2000020228BFA0EB8110B0EB411F00BF42EBC6
:101C3000020228BFA0EB4110B0EB011F00BF42EB36
:101C4000020228BFA0EB0110B0EBC10F00BF42EBB6
:101C5000020228BFA0EBC100B0EB810F00BF42EB36
:101C6000020228BFA0EB8100B0EB410F00BF42EBA6
:101C7000020228BFA0EB4100B0EB010F00BF42EB16
:101C8000020228BFA0EB0100104670470CBF0120E4
:101C900000207047B1FA81F2C2F11F0220FA02F06F
:101CA000704708B14FF0FF3000F066B90029F8D056
:101CB0002DE90340FFF7CCFEBDE8064002FB00F330
:101CC000A1EB0301704700BF002900F03E8180EACC
:101CD000010C48BF49424A1E00F01F81030048BF63
:101CE00043428B4240F21E81114200F02381B3FA3D
:101CF00083F2B1FA81F0A0EB0202C2F11F0204A04C
:101D000000EB02124FF00000974600BFAFF30080D7
:101D1000B3EBC17F00BF40EB000028BFA3EBC17352
:101D2000B3EB817F00BF40EB000028BFA3EB8173C2
:101D3000B3EB417F00BF40EB000028BFA3EB417332
:101D4000B3EB017F00BF40EB000028BFA3EB0173A2
:101D5000B3EBC16F00BF40EB000028BFA3EBC16332
:101D6000B3EB816F00BF40EB000028BFA3EB8163A2
:101D7000B3EB416F00BF40EB000028BFA3EB416312
:101D8000B3EB016F00BF40EB000028BFA3EB016382
:101D9000B3EBC15F00BF40EB000028BFA3EBC15312
:101DA000B3EB815F00BF40EB000028BFA3EB815382
:101DB000B3EB415F00BF40EB000028BFA3EB4153F2
:101DC000B3EB015F00BF40EB000028BFA3EB015362
:101DD000B3EBC14F00BF40EB000028BFA3EBC143F2
:101DE000B3EB814F00BF40EB000028BFA3EB814362
:101DF000B3EB414F00BF40EB000028BFA3EB4143D2
:101E0000B3EB014F00BF40EB000028BFA3EB014341
:101E1000B3EBC13F00BF40EB000028BFA3EBC133D1
:101E2000B3EB813F00BF40EB000028BFA3EB813341
:101E3000B3EB413F00BF40EB000028BFA3EB4133B1
:101E4000B3EB013F00BF40EB000028BFA3EB013321
:101E5000B3EBC12F00BF40EB000028BFA3EBC123B1
:101E6000B3EB812F00BF40EB000028BFA3EB812321
:101E7000B3EB412F00BF40EB000028BFA3EB412391
:101E8000B3EB012F00BF40EB000028BFA3EB012301
:101E9000B3EBC11F00BF40EB000028BFA3EBC11391
:101EA000B3EB811F00BF40EB000028BFA3EB811301
:101EB000B3EB411F00BF40EB000028BFA3EB411371
:101EC000B3EB011F00BF40EB000028BFA3EB0113E1
:101ED000B3EBC10F00BF40EB000028BFA3EBC10371
:101EE000B3EB810F00BF40EB000028BFA3EB8103E1
:101EF000B3EB410F00BF40EB000028BFA3EB410351
:101F0000B3EB010F00BF40EB000028BFA3EB0103C0
:101F1000BCF1000F48BF404270479CEA000F48BF29
:101F20004042704738BF002004BF4FEAEC7040F0D9
:101F300001007047B1FA81F2C2F11F02BCF1000F3B
:101F400023FA02F048BF404270470028C8BF6FF034
:101F50000040B8BF4FF0004000F00EB80029F4D0A8
:101F60002DE90340FFF7B3FEBDE8064002FB00F396
:101F7000A1EB0301704700BF704700BF81F0004133
:101F800002E000BF83F0004330B54FEA41044FEA5E
:101F9000430594EA050F08BF90EA020F1FBF54EAF9
:101FA000000C55EA020C7FEA645C7FEA655C00F095
:101FB000E2804FEA5454D4EB5555B8BF6D420CDD66
:101FC0002C4480EA020281EA030382EA000083EAE9
:101FD000010180EA020281EA0303362D88BF30BD89
:101FE00011F0004F4FEA01314FF4801C4CEA1131DF
:101FF00002D0404261EB410113F0004F4FEA03333E
:102000004CEA133302D0524263EB430394EA050FC8
:1020100000F0A780A4F10104D5F1200E0DDB02FA37
:102020000EFC22FA05F2801841F1000103FA0EF2CB
:10203000801843FA05F359410EE0A5F120050EF191
:10204000200E012A03FA0EFC28BF4CF0020C43FAC2
:1020500005F3C01851EBE37101F0004507D54FF0CF
:10206000000EDCF1000C7EEB00006EEB0101B1F51F
:10207000801F1BD3B1F5001F0CD349085FEA300065
:102080004FEA3C0C04F101044FEA445212F5800F70
:1020900080F09A80BCF1004F08BF5FEA500C50F10D
:1020A000000041EB045141EA050130BD5FEA4C0CF0
:1020B000404141EB010111F4801FA4F10104E9D179
:1020C00091F0000F04BF01460020B1FA81F308BF70
:1020D0002033A3F10B03B3F120020CDA0C3208DD3C
:1020E00002F1140CC2F10C0201FA0CF021FA02F117
:1020F0000CE002F11402D8BFC2F1200C01FA02F187
:1021000020FA0CFCDCBF41EA0C019040E41AA2BFAB
:1021100001EB0451294330BD6FEA04041F3C1CDA73
:102120000C340EDC04F11404C4F1200220FA04F093
:1021300001FA02F340EA030021FA04F345EA03013D
:1021400030BDC4F10C04C4F1200220FA02F001FAFF
:1021500004F340EA0300294630BD21FA04F0294681
:1021600030BD94F0000F83F4801306BF81F480111A
:102170000134013D4EE77FEA645C18BF7FEA655C8D
:1021800029D094EA050F08BF90EA020F05D054EA5F
:10219000000C04BF1946104630BD91EA030F1EBF64
:1021A0000021002030BD5FEA545C05D14000494168
:1021B00028BF41F0004130BD14F580043CBF01F55B
:1021C000801130BD01F0004545F0FE4141F4700141
:1021D0004FF0000030BD7FEA645C1ABF194610461C
:1021E0007FEA655C1CBF0B46024650EA013406BF1D
:1021F00052EA033591EA030F41F4002130BD00BFDC
:1022000090F0000F04BF0021704730B54FF4806498
:1022100004F132044FF000054FF0000150E700BF19
:1022200090F0000F04BF0021704730B54FF4806478
:1022300004F1320410F0004548BF40424FF0000165
:102240003EE700BF42004FEAE2014FEA31014FEAA8
:1022500002701FBF12F07F4393F07F4F81F06051F7
:10226000704792F0000F14BF93F07F4F704730B566
:102270004FF4607401F0004521F0004120E700BFF9
:1022800050EA010208BF704730B54FF000050AE080
:1022900050EA010208BF704730B511F0004502D581
:1022A000404261EB41014FF4806404F132045FEA83
:1022B000915C3FF4DCAE4FF003025FEADC0C18BF28
:1022C00003325FEADC0C18BF033202EBDC02C2F11E
:1022D000200300FA03FC20FA02F001FA03FE40EAB0
:1022E0000E0021FA02F11444C1E600BF70B54FF0B0
:1022F000FF0C4CF4E06C1CEA11541DBF1CEA135592
:1023000094EA0C0F95EA0C0F00F0DEF82C4481EAF9
:10231000030621EA4C5123EA4C5350EA013518BF19
:1023200052EA033541F4801143F4801338D0A0FB06
:1023300002CE4FF00005E1FB02E506F00042E0FBB3
:1023400003E54FF00006E1FB03569CF0000F18BFB9
:102350004EF0010EA4F1FF04B6F5007F64F5407461
:1023600004D25FEA4E0E6D4146EB060642EAC621F4
:1023700041EA55514FEAC52040EA5E504FEACE2E61
:10238000B4F1FD0C88BFBCF5E06F1ED8BEF1004F64
:1023900008BF5FEA500E50F1000041EB045170BDE0
:1023A00006F0004646EA010140EA020081EA030124
:1023B000B4EB5C04C2BFD4EB0C0541EA045170BD20
:1023C00041F480114FF0000E013C00F3AB8014F19A
:1023D000360FDEBF002001F0004170BDC4F10004E3
:1023E000203C35DA0C341BDC04F11404C4F1200564
:1023F00000FA05F320FA04F001FA05F240EA0200BF
:1024000001F0004221F0004110EBD37021FA04F6F4
:1024100042EB06015EEA430E08BF20EAD37070BDAE
:10242000C4F10C04C4F1200500FA04F320FA05F00D
:1024300001FA04F240EA020001F0004110EBD3700F
:1024400041F100015EEA430E08BF20EAD37070BD7F
:10245000C4F1200500FA05F24EEA020E20FA04F358
:1024600001FA05F243EA020321FA04F001F0004107
:1024700021FA04F220EA020000EBD3705EEA430E78
:1024800008BF20EAD37070BD94F0000F0FD101F0A7
:102490000046400041EB010111F4801F08BF013CE0
:1024A000F7D041EA060195F0000F18BF704703F01E
:1024B0000046520043EB030313F4801F08BF013DA5
:1024C000F7D043EA0603704794EA0C0F0CEA135561
:1024D00018BF95EA0C0F0CD050EA410618BF52EA1B
:1024E0004306D1D181EA030101F000414FF0000021
:1024F00070BD50EA410606BF1046194652EA43062F
:1025000019D094EA0C0F02D150EA013613D195EAA2
:102510000C0F05D152EA03361CBF104619460AD1EA
:1025200081EA030101F0004141F0FE4141F47001F4
:102530004FF0000070BD41F0FE4141F4780170BDE4
:1025400070B54FF0FF0C4CF4E06C1CEA11541DBF49
:102550001CEA135594EA0C0F95EA0C0F00F0A7F84B
:10256000A4EB050481EA030E52EA03354FEA013178
:1025700000F088804FEA03334FF0805545EA13138B
:1025800043EA12634FEA022245EA111545EA106553
:102590004FEA00260EF000419D4208BF964244F1EA
:1025A000FD0404F5407402D25B084FEA3202B61A09
:1025B00065EB03055B084FEA32024FF480104FF4DD
:1025C000002CB6EB020E75EB030E22BFB61A754651
:1025D00040EA0C005B084FEA3202B6EB020E75EBE4
:1025E000030E22BFB61A754640EA5C005B084FEA4C
:1025F0003202B6EB020E75EB030E22BFB61A754619
:1026000040EA9C005B084FEA3202B6EB020E75EB23
:10261000030E22BFB61A754640EADC0055EA060EE4
:1026200018D04FEA051545EA16754FEA06164FEA27
:10263000C30343EA52734FEAC2025FEA1C1CC0D1D3
:1026400011F4801F0BD141EA00014FF000004FF060
:10265000004CB6E711F4801F04BF01430020B4F121
:10266000FD0C88BFBCF5E06F3FF6AFAEB5EB030CD9
:1026700004BFB6EB020C5FEA500C50F1000041EBD6
:10268000045170BD0EF0004E4EEA113114EB5C04A3
:10269000C2BFD4EB0C0541EA045170BD41F4801176
:1026A0004FF0000E013C90E645EA060E8DE60CEA7E
:1026B000135594EA0C0F08BF95EA0C0F3FF43BAF9B
:1026C00094EA0C0F0AD150EA01347FF434AF95EA52
:1026D0000C0F7FF425AF104619462CE795EA0C0F36
:1026E00006D152EA03353FF4FDAE1046194622E703
:1026F00050EA410618BF52EA43067FF4C5AE50EADD
:1027000041047FF40DAF52EA43057FF4EBAE12E7CC
:102710004FF0FF3C06E000BF4FF0010C02E000BFAD
:102720004FF0010C4DF804CD4FEA410C7FEA6C5C90
:102730004FEA430C18BF7FEA6C5C1BD001B050EA33
:10274000410C0CBF52EA430C91EA030F02BF90EA1E
:10275000020F0020704710F1000F91EA030F58BFDD
:10276000994208BF90422CBFD8176FEAE37040F03F
:10277000010070474FEA410C7FEA6C5C02D150EADD
:10278000013C07D14FEA430C7FEA6C5CD6D152EA98
:10279000033CD3D05DF8040B704700BF844610465D
:1027A00062468C461946634600E000BF01B5FFF75C
:1027B000B7FF002848BF10F1000F01BD4DF808ED2C
:1027C000FFF7F4FF0CBF012000205DF808FB00BFFD
:1027D0004DF808EDFFF7EAFF34BF012000205DF857
:1027E00008FB00BF4DF808EDFFF7E0FF94BF0120A4
:1027F00000205DF808FB00BF4DF808EDFFF7CEFFA5
:1028000094BF012000205DF808FB00BF4DF808EDE3
:10281000FFF7C4FF34BF012000205DF808FB00BFB4
:102820004FEA410212F5001215D211D56FF47873F8
:10283000B3EB625212D94FEAC12343F0004343EA9B
:10284000505311F0004F23FA02F018BF4042704776
:102850004FF00000704750EA013005D111F0004000
:1028600008BF6FF0004070474FF00000704700BF96
:102870004A0011D212F5001211D20DD56FF47873FF
:10288000B3EB62520ED44FEAC12343F0004343EA54
:10289000505323FA02F070474FF00000704750EA9F
:1028A000013002D14FF0FF3070474FF00000704709
:1028B0004FEA4102B2F1E04324BFB3F5001CDCF162
:1028C000FE5C0DD901F0004C4FEAC0024CEA50709A
:1028D000B2F1004F40EB830008BF20F001007047C9
:1028E00011F0804F21D113F13872BCBF01F00040CC
:1028F000704741F480114FEA5252C2F11802C2F1FE
:10290000200C10FA0CF320FA02F018BF40F001007E
:102910004FEAC1234FEAD32303FA0CFC40EA0C0030
:1029200023FA02F34FEA4303CCE77FEA625307D16D
:1029300050EA01331EBF4FF0FE4040F440007047A4
:1029400001F0004040F0FE4040F40000704700BF3E
:1029500080F0004002E000BF81F0004142001FBF54
:102960005FEA410392EA030F7FEA226C7FEA236C5D
:102970006AD04FEA1262D2EB1363C1BFD218414052
:1029800048404140B8BF5B42192B88BF704710F0E8
:10299000004F40F4000020F07F4018BF404211F08B
:1029A000004F41F4000121F07F4118BF494292EAF3
:1029B000030F3FD0A2F1010241FA03FC10EB0C001F
:1029C000C3F1200301FA03F100F0004302D54942AC
:1029D00060EB4000B0F5000F13D3B0F1807F06D359
:1029E00040084FEA310102F10102FE2A51D2B1F151
:1029F000004F40EBC25008BF20F0010040EA030046
:102A00007047490040EB000010F4000FA2F10102F2
:102A1000EDD1B0FA80FCACF1080CB2EB0C0200FA7C
:102A20000CF0AABF00EBC25052421843BCBFD040CA
:102A30001843704792F0000F81F4000106BF80F444
:102A400000000132013BB5E74FEA41037FEA226C07
:102A500018BF7FEA236C21D092EA030F04D092F0D2
:102A6000000F08BF0846704790EA010F1CBF002006
:102A7000704712F07F4F04D1400028BF40F0004063
:102A8000704712F100723CBF00F50000704700F083
:102A9000004343F0FE4040F4000070477FEA2262AA
:102AA00016BF08467FEA23630146420206BF5FEA7B
:102AB000412390EA010F40F4800070474FF000037B
:102AC00004E000BF10F0004348BF40425FEA000C42
:102AD00008BF704743F0964301464FF000001CE0EA
:102AE00050EA010208BF70474FF000030AE000BF40
:102AF00050EA010208BF704711F0004302D540427E
:102B000061EB41015FEA010C02BF844601460020EF
:102B100043F0B64308BFA3F18053A3F50003BCFA0A
:102B20008CF2083AA3EBC25310DB01FA02FC6344B7
:102B300000FA02FCC2F12002BCF1004F20FA02F2BE
:102B400043EB020008BF20F00100704702F12002B1
:102B500001FA02FCC2F1200250EA4C0021FA02F212
:102B600043EB020008BF20EADC7070474FF0FF0C17
:102B70001CEAD0521EBF1CEAD15392EA0C0F93EA12
:102B80000C0F6FD01A4480EA010C400218BF5FEAB4
:102B900041211ED04FF0006343EA501043EA511127
:102BA000A0FB01310CF00040B1F5000F3EBF490021
:102BB00041EAD3715B0040EA010062F17F02FD2A25
:102BC0001DD8B3F1004F40EBC25008BF20F0010008
:102BD000704790F0000F0CF0004C08BF49024CEA1F
:102BE000502040EA51207F3AC2BFD2F1FF0340EAB1
:102BF000C250704740F400004FF00003013A5DDC22
:102C000012F1190FDCBF00F000407047C2F1000262
:102C1000410021FA02F1C2F1200200FA02FC5FEA4F
:102C2000310040F1000053EA4C0308BF20EADC7099
:102C3000704792F0000F00F0004C02BF400010F40B
:102C4000000F013AF9D040EA0C0093F0000F01F0B8
:102C5000004C02BF490011F4000F013BF9D041EADA
:102C60000C018FE70CEAD15392EA0C0F18BF93EADC
:102C70000C0F0AD030F0004C18BF31F0004CD8D106
:102C800080EA010000F00040704790F0000F17BF8D
:102C900090F0004F084691F0000F91F0004F14D0D3
:102CA00092EA0C0F01D142020FD193EA0C0F03D12B
:102CB0004B0218BF084608D180EA010000F000402E
:102CC00040F0FE4040F40000704740F0FE4040F409
:102CD000400070474FF0FF0C1CEAD0521EBF1CEAA8
:102CE000D15392EA0C0F93EA0C0F69D0A2EB0302C6
:102CF00080EA010C49024FEA402037D04FF0805360
:102D000043EA111143EA10130CF000408B4238BF24
:102D10005B0042F17D024FF4000C8B4224BF5B1A32
:102D200040EA0C00B3EB510F24BFA3EB510340EA80
:102D30005C00B3EB910F24BFA3EB910340EA9C002E
:102D4000B3EBD10F24BFA3EBD10340EADC001B019E
:102D500018BF5FEA1C1CE0D1FD2A3FF650AF8B4242
:102D600040EBC25008BF20F0010070470CF0004C4F
:102D70004CEA50207F32C2BFD2F1FF0340EAC2507A
:102D8000704740F400004FF00003013A37E792F03B
:102D9000000F00F0004C02BF400010F4000F013A99
:102DA000F9D040EA0C0093F0000F01F0004C02BF94
:102DB000490011F4000F013BF9D041EA0C0195E7FD
:102DC0000CEAD15392EA0C0F08D142027FF47DAF96
:102DD00093EA0C0F7FF470AF084676E793EA0C0F86
:102DE00004D14B023FF44CAF08466EE730F0004C84
:102DF00018BF31F0004CCAD130F000427FF45CAF14
:102E000031F000437FF43CAF5FE700BF4FF0FF3C81
:102E100006E000BF4FF0010C02E000BF4FF0010CD4
:102E20004DF804CD4FEA40024FEA41037FEA226C9D
:102E300018BF7FEA236C11D001B052EA530C18BFBF
:102E400090EA010F58BFB2EB030088BFC81738BF24
:102E50006FEAE17018BF40F0010070477FEA226C12
:102E600002D15FEA402C05D17FEA236CE4D15FEA0E
:102E7000412CE1D05DF8040B704700BF8446084642
:102E80006146FFE70FB5FFF7C9FF002848BF10F103
:102E9000000F0FBD4DF808EDFFF7F4FF0CBF012048
:102EA00000205DF808FB00BF4DF808EDFFF7EAFFD2
:102EB00034BF012000205DF808FB00BF4DF808ED8D
:102EC000FFF7E0FF94BF012000205DF808FB00BF82
:102ED0004DF808EDFFF7D2FF94BF012000205DF808
:102EE00008FB00BF4DF808EDFFF7C8FF34BF012015
:102EF00000205DF808FB00BF4FEA4002B2F1FE4F30
:102F00000FD34FF09E03B3EB12620DD94FEA0023AB
:102F100043F0004310F0004F23FA02F018BF404284
:102F200070474FF00000704712F1610F01D142026B
:102F300005D110F0004008BF6FF0004070474FF01F
:102F400000007047012808B507D002D302280CD131
:102F500007E0DC204121054B9847DC208121034B11
:102F60009847DC208521014B984708BDD15B0108BB
:102F7000012810B50DD002D3022812D10DE0DC20BB
:102F80008021084CA047DC208421A047DC20402180
:102F9000A047DC208021034B9847DC208421014B93
:102FA000984710BDD15B0108022808B501D8D8B9EF
:102FB00002E0642823D117E0DC200121154B98475B
:102FC00010F0800F02D0144B984718E010F0200F3B
:102FD00017D100F00503052B15D010F0040F14D104
:102FE00010F0010F04D012E0DC200121094B9847BA
:102FF00000F0400000280CBF0120022008BD012085
:1030000008BD002008BD0D2008BD0C2008BD0B2008
:1030100008BD00BFA55C0108C55A010864282DE958
:10302000F04740F0CD8043F6982467484FF40031D4
:10303000664B984708B94CB906E0013CA4B24FF67C
:10304000FF739C42F1D101E0614B98475E4801213A
:10305000604FB84743F698245B485F495F4DA847E7
:1030600018B914B1013CA4B2F6E74FF42F705C4CD0
:10307000A0475C4E5448DC210022B04743F6982814
:1030800051485949A84738B9B8F1000F04D008F1A0
:10309000FF381FFA88F8F3E74FF42F70A0474A482B
:1030A0000221524B984743F6982847485049A84771
:1030B00038B9B8F1000F04D008F1FF381FFA88F8CA
:1030C000F3E74FF42F70A0473F480121B84743F67C
:1030D00098273D484049A84718B917B1013FBFB2EA
:1030E000F7E74FF42F70A0473748DD210122B047A2
:1030F00043F6982634483F49A84718B916B1013E0F
:10310000B6B2F7E74FF42F70A04743F698262E4843
:103110003949A84718B916B1013EB6B2F7E72A48AF
:10312000364EB0475FFA80F94FF42F70A04743F650
:10313000982725483049A84718B917B1013FBFB2B1
:10314000F7E72148B04749EA00294FF42F70A0471C
:103150001FFA89F943F699271B482749A84718B948
:10316000013FBFB2002FF7D11748B0475FFA80FA8E
:103170004FF42F70A047DFF88C8013480021C04720
:1031800043F6992710481C49A84718B9013FBFB218
:10319000002FF7D10C48B0474AEA00254FF42F70B2
:1031A000A047ADB208480121154B9847AD0206482B
:1031B0000121C04795FBF9F91FFA89F0BDE8F087B6
:1031C00040F6E440BDE8F087005400406173010818
:1031D000C55A0108DF7201080100030047730108A6
:1031E0006345010837730108820007002D73010849
:1031F000840007000200030040000300317301084F
:10320000F9720108137301082DE9F04FDC20012148
:1032100091B09A4B984710F0800F23D00021984826
:10322000984B9847984B9847984E3221984D4FF4B9
:103230004870B047974CA8476420A04732214FF40C
:103240004870B047A8476420A04732214FF4487027
:10325000B047A8476420A0474FF47A70A0478E4B30
:1032600098470BE202208D4CA0470120A047642024
:103270008B4CA047022840F0F681DA308721894A3A
:1032800090474FF00008012364254446079300202F
:10329000834FB8470D2812D1002D3CD00021824821
:1032A000784BDFF8E4A19847D0474FF42F700A21FC
:1032B000764B9847764B98470020B847D3E10B28C8
:1032C0000ED155B1631EDBB2022B06D9D130872156
:1032D000DFF8D0C1E047012207924FF448700EE0BA
:1032E0000C2819D14DB1631EDBB2022B05D9D030A9
:1032F00086216C4FB847002207924FF461700A2173
:10330000624B9847624B98470020654B002C14BFD6
:103310000A24002498476425644B64209847DFF80A
:10332000C4B10690D847DFF8B8A10646D0474FF0A1
:103330000109721E431EFF2600200146D2B2DBB2F5
:10334000CDF800905A4F019602960396B847D84799
:103350000746D047FA1EC31E00270220DFF850C1DF
:103360000146CDF80090019702970397D2B2DBB2E5
:10337000E047069ACDF8009011B203233A4608A818
:103380004C4FB8474C494D4B08A89847DFF848C107
:103390004B48CDF810C0E0470746D0470523B0FBA7
:1033A000F3F1474A38460096464F0196C9B2334674
:1033B000B847DDF810C0079AD9465746DFF804B180
:1033C000E24682B14048E0470590B8474FF0050C0F
:1033D000B0FBFCF1059B490000960196184601F0F0
:1033E000FE013A4A0EE03A48E0470590B847052208
:1033F000B0FBF2F1059B4900364A0096019618464B
:1034000001F0FE013346D84708A8D0470590B847D9
:103410004FF0050CB0FBFCF1059BFF2601EB4101D1
:10342000184608AA00960196C9B23346D847069AAC
:10343000B2F5616F19D2B8F1000F00F0FA80264B97
:1034400026489847264B044698470523B0FBF3F1DE
:103450008900204600961B4C019601F0FC011F4A92
:1034600033460025A0472C46E7E0DDF818C0BCF540
:103470007F6F39D2002C40F0DF8072E0A55C01083C
:10348000C8750108AD640008893B01088144010842
:103490009944010851450108C55A0108712F0008D7
:1034A000A92F0008D15B0108D37501081D30000861
:1034B0000534010849450008DE7501084916000871
:1034C000E3750108BD380108EC750108ED750108C8
:1034D000F3750108F475010879500008F9750108C1
:1034E0006B3B0108673B0108069A41F203039A42CD
:1034F00001D8002C35D0B8F1000F0FD06148D0476B
:103500000646B8470521B0FBF1F1FF23890000937F
:103510000193304601F0FC015A4AD847022C00F2D0
:103520008C80594E5CB94FF416701421B0470027B7
:10353000DC208621554B9847322501340797B8F196
:10354000000F02D04FF4487001E04FF47A7014215C
:10355000B0470DB14E4B98470020DFF848A1D04747
:103560006BE0C8470446B8478246C8470646B84796
:10357000640872084FF0010C0026193CAAF10E01F4
:10358000A0F108031932CDF800C0CDF810C0C9B2BF
:10359000D2B2DBB2E0B201963E4C02960396A0474F
:1035A000C8478346B8478246C8470446B8474FEAEB
:1035B0005B0E6208AEF1190EFF24AAF10E01A0F114
:1035C000080319325FFA8EF0C9B201940294039491
:1035D000D2B2DBB2DFF8BCA00096D047069A4FF01B
:1035E0000C0AA2F55C631E3B93FBFAFAC8470590F0
:1035F000B8478346C8478146B847059BDDF810C0E9
:103600005B08AAF1190AA3F11702ABF10C01A0F1B2
:103610000A030AEB5909019402940394D0B21D4C99
:10362000CDF800C0C9B25FFA89F2DBB2A0473446D8
:1036300003E04546444600E00024174FB8476420A5
:10364000164B984735B1013D0120DFF858A0ADB2C7
:10365000D04703E02846DFF84CC0E047C8F1010836
:103660005FFA88F813E68721084ADC2090470C4C63
:103670000020A0470220A0470120A04711B0BDE8CC
:10368000F08F00BF0276010881440108D15B010878
:103690009944010805340108893B01085145010896
:1036A000452F0008D13E0108FF230370FF3B8370C4
:1036B000643343707047FF230370F53B83705A33C4
:1036C0004370643BC370704738B5002504464570AD
:1036D0000E4B043098470E4B04F108009847FF2327
:1036E0006422237023736273A373E273237462747E
:1036F000A374E274072395FBF3F3643BC835237589
:1037000063750434B5F5C86FF4D138BDB736000819
:10371000A936000837B50D4B04460D4998470D4BA7
:10372000204698470C4B201819780C4D4A1C1A70EB
:103730000123002200931346A847002323826382BB
:10374000A382A375E3750023A3613EBD9116000813
:103750000A7601084D1700080903002049450008B2
:1037600037B5114B0446114998472046104B9847EE
:10377000104B20181978104D4A1C1A700022012392
:1037800000931346A84700222282A274E274227595
:103790006275A275E27522766276A276E27604F10F
:1037A0001C00064B98473EBD91160008167601088E
:1037B0004D1700080C03002049450008A9360008F1
:1037C0000023037043708370C370704770B5FF238C
:1037D0000025044643700570074B8570C5700430A2
:1037E0009847064E04F10800B04704F10C00B047BA
:1037F0002582658270BD00BFB7360008A936000873
:10380000FF2310B50370FF3B044643708370C37001
:103810000430034B984704F10800024B984710BD51
:10382000B7360008A9360008FF2310B50370FF3B28
:10383000044643708370C3700430034B984704F10F
:103840000800024B984710BDB7360008A93600089B
:1038500038B5FF230370FF3B044643708370C37089
:103860000430054B9847054D04F10800A84704F1C2
:103870000C00A84738BD00BFB7360008A9360008BD
:1038800038B5FF230370FF3B044643708370C37059
:103890000430054B9847054D04F10800A84704F192
:1038A0000C00A84738BD00BFB7360008A93600088D
:1038B00037B50D4B04460D49984720460C4B9847A9
:1038C0000C4B201819780C4D4A1C1A700123002249
:1038D00000931346A84700232382A374E37404F1E2
:1038E0001400064B98473EBD911600081D7601084E
:1038F0004D1700080A03002049450008A9360008B2
:103900000023037043708370C3708380C38003817E
:10391000438100F120030022828102309842FAD1D3
:103920007047002343708370C370C21802330021B4
:10393000202B9180F9D1704700230370437083706E
:10394000C370704738B50446124DA847201DA847DC
:1039500004F10800A84704F10C00A84700252574CD
:103960006574A574E57425756575A575E57504F12F
:103970001800094B984725776577A577E577258463
:10398000658484F8245084F8255084F8265084F8FF
:10399000275038BD39390008A93600082DE9F74FFE
:1039A0000024064646F8044B05463A4F3A4930464D
:1039B000B847DFF8EC803046C047384E28183178D9
:1039C0004FF001094B1CDFF8DCA02246337005F1F3
:1039D000140B23460430CDF80090D0472E495846AA
:1039E000B8475846C0473178281801EB09032246EA
:1039F000337005F1240B23461430CDF80090D047E6
:103A000025495846B8475846C0473178281801EB31
:103A100009032246337005F1340B23462430CDF8D8
:103A20000090D0471C495846B8475846C04731789F
:103A3000281801EB09032246337005F1440B234695
:103A40003430CDF80090D04713495846B84758460F
:103A5000C0473178281801EB09032246337005F579
:103A6000A27B23464430CDF80090D0470A495846FF
:103A7000B8475846C0473178281801EB090333701E
:103A80002246234600F5A270CDF80090D047BDE84D
:103A9000FE8F00BF91160008257601080B03002059
:103AA0004D170008494500080023038043808380A8
:103AB000C380704738B50546002405EBC400034BAE
:103AC00001349847042CF8D138BD00BFA93A00084A
:103AD00000234370C3704371C371704770B50025F4
:103AE00004460560057145718571C571A81C04EB1C
:103AF00080002E4B01359847102DF7D1103D0C203A
:103B000000FB05402A4B483001359847102DF6D16F
:103B1000103D0C2000FB0540264B00F5847001355C
:103B20009847102DF5D1103D142000FB0540224B85
:103B300000F5E47001359847102DF5D1103D342083
:103B400000FB05401D4B00F5427001359847402DA4
:103B5000F5D1403D280100F5805008302018184B61
:103B600001359847102DF5D1103D280100F58850FA
:103B700008302018134B01359847102DF5D104F566
:103B8000905606F10800104DA84706F13400A847EA
:103B900004F593500D4D04F59454A847201DA847F3
:103BA00004F128000A4B984770BD00BFC1370008D8
:103BB0000138000829380008CD370008C936000848
:103BC00051380008813800080139000823390008FD
:103BD000D13A00080023037043708370C3707047AC
:103BE00010B5054B044698470022A280E28022725D
:103BF0006272A272E27210BDB7360008002208B5E8
:103C000002608280C280027242728272C272024B71
:103C10000C30984708BD00BFB73600082DE9F347C0
:103C200004463149314FB847314E2046B047314DF7
:103C3000002229784FF001084B1C2B70DFF8D09040
:103C4000134604F1180A2018CDF80080C847264909
:103C50005046B8475046B0472978002201EB080388
:103C600018302B70201800251346CDF80080C84767
:103C700084F8285084F8295084F82A5084F82B506E
:103C8000680120182C301C4B01359847402DF7D186
:103C9000403D182000FB054000F502600C30174B3A
:103CA00001359847402DF4D1403D1C2000FB0540D4
:103CB00000F562600C30124B01359847202DF4D18D
:103CC00004F58C500F4B04F510542C3098470E4DD2
:103CD00004F15C00A84704F16C00A84704F17C00E3
:103CE0000A4B9847BDE8FC872E760108911600081C
:103CF0004D1700080803002061370008B13800089C
:103D000015370008DD3A0008FD3B0008E13B0008DC
:103D10004945000810B5064B0446984704F12000B9
:103D2000044B984704F14800034B984710BD00BF6F
:103D3000B53A0008453900089D3900080C4A0023AF
:103D400010B513700B4A044613700B4A04F5125455
:103D500013700A4A13700A4A13700A4B984704F109
:103D60000800094B984704F10C00084B984710BD18
:103D7000090300200C0300200A0300200B0300208D
:103D8000080300201D3C0008D53B0008153D000835
:103D90002DE9F04193F900406425E602361B96FBBD
:103DA000F5F6541EB04213F8244001DC30B207E0AF
:103DB00064B2E602341B94FBF5F4A042A8BF20B223
:103DC00000262AE093F90040E5022D1B642495FBB0
:103DD000F4F5A8421FDB93F9047003F1040C4FEAD9
:103DE000C728C7EB080797FBF4F7B84213DC93F931
:103DF0000130401BDA02D31A9CF9012093FBF4F343
:103E0000D602B21A92FBF4F4E41A60437F1B90FBD3
:103E1000F7F5ED1805E001360433541EA642D1DB58
:103E200000256943642391FBF3F000B2BDE8F08103
:103E30000378FF2B1AD0FE2B1AD0FD2B01D140782E
:103E400017E03F2B05D80C4A5B019B189A7952B2B8
:103E500000E0002290F9023090F901006432C01AAB
:103E60005043C82190FBF1F0C01802E0002000E0B0
:103E7000642040B2704700BFCC0E00200278034699
:103E8000FF2A17D0FE2A13D03F2A13D80E49520119
:103E90005218917990F9020049B288420ADC90796F
:103EA00093F9012040B28242B4BF0020012002E019
:103EB000012000E0002093F90330012B04BFC0F182
:103EC0000100C0B2704700BFCC0E002010B5A0B0FA
:103ED0000346ADF1020400221148182101FB020142
:103EE00001F50261183189880132402A24F8021F45
:103EF000F2D1303A182101FB0201B1F83C4802F539
:103F00008E513431013200EB4101202A0C81F1D174
:103F1000044A4021D06A6A46984720B010BD00BFCD
:103F2000940E00201420002010B51948194B984712
:103F30001748194B00F59A51083198471448174B08
:103F400000F58E51083198471148154B00F59451F2
:103F5000083198470E48134B00F5A452083200F57B
:103F6000006198471048114B00F5CC510831984733
:103F70000D480F4B00F5D451083198470D4B0A48B6
:103F800098470D4C0D48A0470D48A04710BD00BFF5
:103F9000C00E0020F9450008394A00088948000889
:103FA000F1490008594B0008C0160020DD4C0008FC
:103FB000494D0008C14D0008CD3E00088558010854
:103FC000BD3C010810B500230D4A342101FB03223A
:103FD000FE2402F5A452FD2182F8343082F83840E4
:103FE00082F83C10FD3982F83E10643182F83D10B1
:103FF00082F840300133402B82F84110E4D110BDEB
:10400000940E0020F8B59C499C4D9D48A8479D49B9
:104010009D48A8479D499E48A8479E499E48A84755
:104020009E4E9F499F48A84742F2B963F3624FF4FE
:10403000967006F5945601214FF4167386F86510B4
:104040003C22A6F86000A6F86230FF2386F86420C0
:1040500086F8683086F87510A6F870004FF4167070
:10406000A6F8720086F8742086F878303C3A844CC2
:10407000142303FB0243FE2003F59A53013283F815
:10408000380000216427FD20102A83F83E1083F8B1
:104090003D7083F83C0083F8421083F8417083F848
:1040A0004000E4D10B460C2101FB0341FE2001F549
:1040B0008E5181F838000022D138013381F83E203A
:1040C00081F83D00D030102B81F83C00EBD10C2161
:1040D00001FB0241FE2001F5945181F838000023D4
:1040E000B338013281F83E3081F83D00B230102AF9
:1040F00081F83C00EBD1342202FB0342FE2002F5A2
:10410000A45282F8380000219A38013382F83E1018
:1041100082F83D009930402B82F83C00EBD101F54C
:1041200006730333FE2204EB03131A7201F5807346
:10413000013304EB0313013103F58C53FE3A64277A
:10414000FD20102983F82E2083F82D7083F82C0091
:1041500083F8322083F8317083F83000DFD102F524
:104160000A730333FE2104EB0313197202F58873FB
:10417000013304EB0313013203F58C53FE3964273A
:10418000FD20102A83F82E1083F82D7083F82C0060
:1041900083F8321083F8317083F83000DFD10B469A
:1041A0002C2101FB0341082001F50E5181F8340058
:1041B000073881F8350081F836004FF4967008878B
:1041C00040F2DC5088874FF47A7001F13002C887E2
:1041D00042F6E06151810022162101FB032101F525
:1041E0008E511C310132002004EB4101102A08815C
:1041F000F2D10133022BD3D1023B242202FB034232
:10420000082102F51052D173F7315173FF399173C0
:104210000A46122101FB032101F5905104310132BC
:10422000002004EB4101102A0881F2D10133022B56
:10423000E3D10021182202FB014201310023FD20BD
:10424000402982F8423882F8413882F84008F1D19A
:104250005A01A218383201211172991C490100201B
:104260006118507288724872FD30087259B209297B
:104270001ADC262119E000BFBE760108911600085D
:10428000940E0020CF7601086C330020D47601080C
:104290007C3300204C9D0108AC330020142000200A
:1042A000DA760108AC0E002027210133402BD171B2
:1042B000CED12B3B84F83F30013384F85F3001339B
:1042C00084F87F306F4901336F4884F89F30A847E6
:1042D0006E496F48A8476F496F48A8476F497048B3
:1042E000A8470A27CE2232230B200C2184F84A202B
:1042F00084F8493084F8487084F86A2084F869307A
:1043000084F8680084F88A2084F8893084F888105A
:1043100084F8AA2084F8A930C13ADB1884F8A820D0
:1043200086F8553086F8573086F85930383386F895
:104330005B3086F8547086F856000A3F86F85810AD
:1043400086F85A20BB1C5B010026E3189E717B0196
:104350000137E318402F83F83E609E87F2D1514920
:104360005148A84751495248A84752495248A8477E
:1043700052495348A84753495348A84753495448BA
:10438000A84754495448A84754495548A84755494F
:104390005548A84755495648A84756493A48A84756
:1043A00055493B48A84755493B48A84754493C48CC
:1043B000A84754495448A84754495548A84755491F
:1043C0005548A84755495648A84756495648A8470A
:1043D00056495748A84757495748584CA847584B3B
:1043E00098470123237284F8533084F85130033303
:1043F00084F85230FB3384F82C6084F8346084F8FD
:104400002D6084F8356084F82E6084F8366084F876
:10441000383084F8393084F83A3084F8303084F811
:10442000313084F83230F93B84F83C30103384F872
:104430004B300D3B84F8493004F1880084F84A6021
:10444000404984F84830133384F85030A84760233B
:10445000A4F84C3032222623A4F84E7084F8402071
:1044600084F842303E3384F8416084F8466084F832
:104470004530993384F844307D3B84F83D3084F8EE
:104480003E60F8BDE276010800100020E9760108E0
:1044900020100020F076010840100020F776010877
:1044A00060100020FE760108C00E0020077701088A
:1044B000E00E002010770108000F00201977010896
:1044C000200F002022770108400F00202B770108E1
:1044D000600F002034770108800F00203D7701082D
:1044E000A00F002046770108C00F00204E7701087A
:1044F000E00F0020577701085F7701086777010810
:104500006F77010877770108801000207E77010817
:10451000A010002085770108C01000208C770108CA
:10452000E010002093770108001100209A7701081D
:1045300020110020A1770108401100201433002031
:10454000C53F0008A6770108F0B5002985B005DA57
:104550002D244942047009B22C3C00E000240025BF
:104560000BE04FF00A0C91FBFCF70CFB1711013527
:10457000303106F80C1CEDB239B204AF092907EB53
:104580000506EEDC303106F80C1C691C03E0302611
:1045900005F80C6C0131C9B204AE994206EB010575
:1045A000F5D99142F3D3002205F80C2C0A460DE010
:1045B0009A4203D12E2101550134E4B204AFB91857
:1045C00011F80D1C013A01550134E4B2002AEFD173
:1045D000025505B0F0BD000010B50024E0B2044B58
:1045E0009847044B23F814000134202CF6D110BD59
:1045F000A14A0108D6060020F0B5002585B0044682
:104600002F4694F91530EEB2042B24D1043B2375C8
:10461000A37D013BDBB2632B01D90123A375E17DAF
:10462000A37DA27C51B958B251B24118632901DC73
:104630009B183DE06423A374633B0AE050B259B277
:10464000411A11F1630F01DBD31A31E09C23A374EB
:104650009C3BE37563E094F914208AB9022B5ED188
:1046600094F91630002B5ED1A37C5AB2632A04DC85
:10467000142701335743A37455E00123A37552E077
:10468000774A012B32F815703FB213D117F5027F2C
:1046900001DA9B330CE0B7F5027F01DD642307E00C
:1046A00007F5F877033740F2E6339F4237D8002307
:1046B000A37434E0022B14D117F1640F05DAA37C44
:1046C0005AB212F1630F2ADB05E0642F27DDA37CC9
:1046D0005AB2632A23DC4FF4FA7297FBF2F7FB1805
:1046E000E6E7032B1FD1642F07DD94F916308BB951
:1046F00094F912205AB9643309E017F1640F09DA0A
:1047000094F9163033B994F9122002B99C33A3748A
:10471000012303E06337C62F01D80023A37594F962
:10472000123014275F43032E1DD84E4A05F59263BD
:10473000013302EBC303DA8812B2BF1A002F07DD80
:104740001A8912B2002A0EDDFA02D71B1B8907E074
:1047500009D09A8812B2002A05DA434A9B88574347
:104760001BB297FBF3F7237F3F2B03D9FE2B01D01E
:10477000FD2B24D13D4B04F11C00984794F91B30CC
:10478000012B15D19B3364218DF804308DF8053051
:104790009C3B8DF808308DF809008DF80C1038B26C
:1047A0008DF80D10324F032201ABB847074606E0E3
:1047B000C302181A642390FBF3F000B23F1894F977
:1047C0001A30012B284B08BF7F429F42B8BF1F46BB
:1047D00040F2FF739F42A8BF1F46264B33F81520B7
:1047E00012B2974221D0092E09D9234A1670234AC2
:1047F0001278C2B194F91520042A12D113E033F8CB
:104800001500282200B297FBF2F190FBF2F29142E0
:1048100009D0194A1670194A1278012A03D9032EB1
:1048200001D9174A167023F8157094F914302782AD
:104830007BB194F9153063B9143397FBF3F31BB2D2
:10484000642BA8BF64236FF063029342B8BF134682
:10485000A37401352034402D7FF4D3AE05B0F0BDF4
:10486000D6060020940E002001F8FFFF313E00081C
:10487000913D00080E030020F10100206533002067
:10488000F4010020000000002DE9F04F0D4685B036
:1048900000242B5D2E193F2B79D8301D424B9847B1
:1048A000012874D106F10800404B98478246002841
:1048B0006DD02E5DDFF8209173014B44988F3C4FF3
:1048C00000B2B8473B493C4B98474FF07E513B4BB9
:1048D0008046984728B9404639493A4B984718B915
:1048E00004E04FF07E5801E0DFF8D4802B195B78AC
:1048F000DFF8EC90013BDBB2012BDFF8E8B0324F80
:1049000005D84046C847CDE90001404606E040468C
:10491000C847CDE9000140464146D8474146D847FF
:104920002A4A014640469047C847214BCDE902013B
:1049300050469847C8470022DFF8ACC0244BE047F8
:1049400002460B46DDE90201B847DFF8A0C0024687
:104950000B46DDE90001E04711A3D3E90023B84786
:104960001C4A90471C4ADFF870C07301760163440B
:10497000961998873836B28840F2FF7312B29A427D
:1049800004DCB288154B12B29A4200DAB3800C34C0
:10499000C02C7FF47EAF05B0BDE8F08FAFF3008090
:1049A0000000000000FC9F407D3E0008313E0008F2
:1049B000C52A000800E0FF44D52C0008E52E0008B9
:1049C000000080BFA92E0008ED2200085929000828
:1049D0000000594021280008940E002001F8FFFF34
:1049E000452200086D2B000841250008851F00089E
:1049F000F8B504460E460025735D77193F2B12D893
:104A0000381D0B4B984701280DD10A4B07F10800C0
:104A10009847735D64215B01E318B3F910204243AA
:104A200092FBF1F21A820C35C02DE5D1F8BD00BF22
:104A30007D3E0008313E00082DE9F04704468846D7
:104A40000D46002708EB070673783F2B76D8281D04
:104A50003E4B984701286CD1DFF8F8A005F108001B
:104A6000D047814605F10C00D04718F8072073782D
:104A700092B95B01E318B3F910202B8A19B209EB44
:104A8000010C624503DD9944A5F810904BE0091A2A
:104A90008A4248DA1B1A45E05B01E318B3F910308B
:104AA000142B10DD03FB09F340F2FF7293FBF2F3CA
:104AB000B2785BB2002A28D0698A08B210189842EE
:104AC00024DA521810E013F1140F11DA4343204A8C
:104AD00093FBF2F3B2785BB242B1698A5B4208B2EF
:104AE000801A984212DD8A1A6A820FE05B420CE05B
:104AF000B37853B16A8A11B2C81A002801DDD31AFB
:104B000003E0CB424CBF9B1800236B822B8A6A8A3E
:104B1000D2180F4B2A8212B29A4203DB40F2FF7383
:104B20009A4200DD2B8273782A8A5B01E3181A828D
:104B300004E073785B01E3181B8A2B821437143569
:104B4000B7F5A07F7FF47EAFBDE8F0877D3E00081B
:104B500001F8FFFF313E00082DE9F74F0B46904664
:104B600082460E4601F5C062002119821833934235
:104B7000FAD14446002518F805303F2B00F29F80FB
:104B8000201D534B9847012840F09980514B04F168
:104B900008009847237B81463F2B21D894F90D20AC
:104BA000F2B14FF0180B0BFB036B18F80530BBF894
:104BB00010C05B015344B3F91000082204F1140340
:104BC000CDF804C04946444FB84794F90D30DDF89C
:104BD00004C04343642293FBF2F39C44ABF810C03F
:104BE000A37B3F2B21D894F90F20F2B14FF0180B83
:104BF0000BFB036B18F80530BBF810C05B01534486
:104C0000B3F91000082204F11403CDF804C049469A
:104C1000314FB84794F90F30DDF804C043436422A4
:104C200093FBF2F39C44ABF810C0237C3F2B21D8BC
:104C300094F91120F2B14FF0180B0BFB036B18F82D
:104C40000530BBF810C05B015344B3F910000822D3
:104C500004F11403CDF804C049461F4FB84794F936
:104C60001130DDF804C04343642293FBF2F39C440B
:104C7000ABF810C0A37C3F2B21D894F91320F2B1DC
:104C80004FF0180B0BFB036B18F80530BBF810C086
:104C90005B015344B3F91000082204F11403CDF86A
:104CA00004C049460C4FB84794F91330DDF804C0EE
:104CB0004343642293FBF2F39C44ABF810C03435B9
:104CC0003434B5F5506F7FF456AFBDE8FE8F00BFAA
:104CD0007D3E0008313E0008913D00082DE9F0417D
:104CE00004460E460025735D06EB05083F2B21D8D0
:104CF00008F10400124B984701281BD1725D182758
:104D000007FB0242138A19B2002902DD08F10800EC
:104D100002E073B108F10C000A4B9847735D6422FE
:104D200007FB0347B7F91030434393FBF2F33B8291
:104D300000E013821035B5F5807FD4D1BDE8F08155
:104D40007D3E0008313E00082DE9F04104460E4644
:104D50000025735D77193F2B28D8381D164B9847CF
:104D6000012823D1DFF8548007F10800C047735DA4
:104D7000182202FB0342C3026421181AB2F9103050
:104D800090FBF1F08342C8BF108207F10C00C047CE
:104D9000735D182202FB0343C2026421821A92FB54
:104DA000F1F2B3F910109142B8BF1A821035B5F57F
:104DB000807FCED1BDE8F0817D3E0008313E000805
:104DC00070B5044600F5C066237DB4F910503F2B42
:104DD00003D9FE2B01D0FD2B0AD10F4B04F1140097
:104DE0009847C3021B1A642293FBF2F31BB2ED181F
:104DF00094F91230012B094B08BF6D429D42B8BF98
:104E00001D4640F6FE139D42A8BF1D46258218345C
:104E1000B442D9D170BD00BF313E000802F6FFFF99
:104E2000704700000D282DE9F74F574B02D10022A3
:104E30001A80A7E01A88C62A07D854490024885443
:104E4000013292B21A808C5401E000221A800A28A2
:104E500040F098801B880C2B40F294804B480378DC
:104E6000422B40F08F8043784D2B40F08B8083782D
:104E70004F2B40F08780C378442B40F0838005306F
:104E8000434FB847434C06231FFA80FB23800BE0B7
:104E9000AB5D701C3A3BDBB2012B03D82818B84736
:104EA00085B20AE03B4B1880384DDFF8F480284685
:104EB000C04726888642EBD30025374E0023337047
:104EC0002388013323800CE01AF809203A3AD2B241
:104ED000012A02D8304A0133137009F10109A4F8FC
:104EE0000090DFF8A8A0B4F800905046C047814574
:104EF00002D233789D42E7DA3378013B9D4241D1BB
:104F0000062222800DE019F80A300AF101003A3B2E
:104F1000DBB2012B03D84844B84785B209E01D4BEA
:104F20001880DFF86890B4F800A04846C047824572
:104F3000E9D30023337016E01AF809203A3AD2B2C6
:104F4000012A10D809F1010001935044B847134ACF
:104F5000DFF850E01070019B1A780BEB0201013270
:104F60000EF801001A702388DFF820A00133238097
:104F70005046C047B4F80090814503D23278064BC2
:104F8000AA42D9D3BDE8FE8F8E03002092030020F1
:104F9000351400085A0400209103002090030020DB
:104FA0004D170008940E00202DE9F047274CB4B0AF
:104FB000A0420746884645D32549264B02A8984774
:104FC000254E02A8B0470022391B02AB0124234D15
:104FD0000094181809B21346A847DFF898902049A2
:104FE00002A8C84702A8B04702AB002200941818D4
:104FF0000FFA88F11346A847B246013C2E464D46AB
:105000000EE0174902A8A84702A8D0470123395D3E
:105010000022009302AB18181346B0470134E4B2E3
:105020004445EED30E4902A8A8470E4B00209847EE
:105030000D4C02A90020A04700200C4B98470020EF
:105040000B49A047002034B0BDE8F087940E002043
:10505000987A0108911600084D1700084945000884
:10506000B08C01080D550108BD55010869560108AD
:105070004A9D01084916000838B5084B9847084D65
:105080000446A847844206D2A847041B04EBD47404
:105090006010C0B238BD002038BD00BF2138010803
:1050A000673B010838B5084B9847084D0446A847A8
:1050B000844206D2A847041B04EBD4746010C0B22B
:1050C00038BD002038BD00BF45380108673B0108E6
:1050D00038B5054B05469847044B04462846984783
:1050E000201AC0B238BD00BF673B0108453801082F
:1050F00008B592F900300BB1002300E001231370D2
:1051000010460121014B9847012008BDA94F000816
:105110002DE9F04FDFF850928FB014468846C8470B
:10512000874D0646A847721E431E00260121D2B2B3
:10513000DBB2009130463146824F019602960396CB
:10514000B847C8478146A847FF21431E09F1FF32EF
:1051500001910291039130463146D2B2DBB2009602
:10516000B847DFF808A22046D047DFF8E4910130C5
:1051700099F800B0834502D8BBF10F0F01D989F827
:105180000060DFF8D4C1FF26CDF814C02046E04708
:105190006D4F22463346009601960321B8476B4A6D
:1051A000DDF814C013789346002B7FD1B8F1010FBE
:1051B0000DD1204699F800800693D0478045644E73
:1051C000069B0CD208F1010886F800803AE0B8F19D
:1051D000020F0AD199F800305D4E13B1013B3370D4
:1051E00030E02046D04730702CE0A8F103085FFA89
:1051F00088F8B8F1010F25D899F8006046B9204623
:10520000D047411C89B22046524B9847012068E1A3
:1052100006F1FF3814F808202B2A01D12D2302E0D3
:105220002D2A03D12B2304F808300BE020460693E7
:10523000D0478642069B03D9202204F80820A355B4
:105240008BF8006099F800606EB9434A4348904774
:105250000646A847FF23A0F11101009301933046B1
:10526000C9B23E4A10E02046D04786420FD93A4B99
:105270003B4898470646A847FF23A0F10901384A52
:10528000009301933046C9B2B847002622E1DFF807
:10529000C8C03448E0470646A847FF23A0F10901EB
:1052A000009301933046C9B22E4AEDE72D48E047FE
:1052B0000690A847069BA0F10901009618460196A2
:1052C000C9B2284A3346B847B8F1010F0DD19BF84F
:1052D0000030013BE25C2B2A10D02D2A12D0382A54
:1052E00001D8013215E0302213E0B8F1020F12D1DB
:1052F0009BF80030013BE25C2B2A01D1023208E02E
:105300002D2A01D1023A04E0302A01D9013A00E005
:105310003922E254B9E7A8F103085FFA88F8B8F136
:10532000010FB2D89BF800305A1EA15C202901D190
:105330002039A15489F8003000238BF80030A4E70D
:105340006B3B0108B5350108BD3801089704002002
:105350008B040020A94F000879500008A07A0108AA
:10536000A57A0108A97A0108673B01084D170008D2
:10537000A35D0022A01908908DF82C308DF82D2007
:10538000594B5A489847831CDBB2079399F8003071
:105390000990013B9E4240F08E80A35DDDF81CC069
:1053A000202B06FB0CF80CD1A84708F10508410892
:1053B000FF23009301935FFA88F0C9B24C4AB847C3
:1053C00036E00EAA08F1050C02F80C3D5FFA8CFCE1
:1053D0000692CDF814C0A847DDF814C04FF0FF08BE
:1053E0004108C9B26046069A4346CDF80080CDF820
:1053F0000480B847A8470690A847069BDDF814C06C
:105400005B08991E099BACF102029C4443080933D6
:1054100000200090CDF80480D0B2CDF808805FFA6B
:105420008CF2CDF80C80C9B2DBB2DFF8C8C0E0471F
:105430009BF80030002B4BD0089803785A1ED2B24C
:105440002B2B8DF82C2001D1023306E02D2B01D11E
:10545000023B02E02F2A02D839238DF82C30079A1C
:1054600006FB02F8A84708F105084108FF230639A2
:105470005FFA88F8009301930BAA4046C9B2B84777
:10548000089803785A1CD2B22B2B8DF82C2001D10E
:10549000023306E02D2B01D1023B02E0392A02D96A
:1054A00030238DF82C30A847FF23410806310093A4
:1054B0000193404609E0A847079B410806FB03F219
:1054C000FF23053200930193D0B2C9B20BAAB847AB
:1054D0000136F6B22046D04701308642FFF448AF8D
:1054E00000200FB0BDE8F08F213801083B7701089C
:1054F000AE7A0108B5350108F0B5012387B006463C
:105500000D461446B2F9001002A800930922013B8F
:10551000084FB847294602AAFF233046064DA84740
:10552000064D064602A8A84702A8A84720603046B4
:1055300007B0F0BD494500081151000835140008B6
:10554000F0B5012387B006460D461446B2F90010A7
:1055500003A8052200930C4F013BB8472946FF23BF
:10556000304603AA094DA847094D064603A8A84797
:10557000B0F5803F02DB0023238002E003A8A847A8
:105580002080304607B0F0BD4945000811510008A1
:1055900035140008F0B50E46B2F9001087B00029A6
:1055A000074614464FF00103174D04DA009303A891
:1055B0000622013B07E02B228DF80C2000930DF111
:1055C0000D00253A0023A8473146FF2303AA0F4DBB
:1055D0003846A8470E4D064603A8A847B0F5FA4F2F
:1055E00002DD4FF4FA4306E003A8A84710F5FA4F8E
:1055F00003DA48F20033238002E003A8A8472080A2
:10560000304607B0F0BD00BF494500081151000801
:10561000351400082DE9F04FDFF87C928DB0144668
:105620008846C8478F4E0546B0476A1E431E002570
:105630000121D2B2DBB20091284629468A4F01955A
:1056400002950395B847C8478146B047FF21431EDE
:1056500009F1FF3201910291039128462946D2B205
:10566000DBB20095B847DFF80CB22046D847DFF828
:1056700008A201309AF80090814502D8B9F10F0FC5
:1056800001D98AF80050FF25DFF810922046C8475C
:10569000764F22462B46009501950321B847744A60
:1056A000CB461378002B77D1B8F1010F0FD10493BB
:1056B0002046704A90479AF80080013080456E4D30
:1056C000049B0CD208F1010885F8008032E0B8F1A3
:1056D000020F0CD19AF80030674D13B1013B2B70CB
:1056E00028E02046634B98470130287022E0A8F15B
:1056F00003085FFA88F8B8F1010F1BD89AF8005038
:1057000055B9DFF870C12046E047411C89B22046F8
:105710005A4B9847012069E104932046554A904727
:105720008542049B04D96219202102F8011C6355AB
:105730004F4B1D709AF8005065B95148D84705463F
:10574000B047FF23A0F10901009301932846C9B295
:105750004B4A11E02046DFF81CC1E04785420ED9D4
:105760004848D8470546B047FF23A0F10901454AFC
:10577000009301932846C9B2B84700252EE142485C
:10578000D8470546B047FF23A0F1090100930193D4
:105790002846C9B23C4AEFE73B48C8478146B04774
:1057A000A0F10901009501954846C9B2364A2B4639
:1057B000B847B8F1010F09D12D480378013BE25CED
:1057C0007E2A01D801320DE020220BE0B8F1020F51
:1057D0000AD1274A1378013BE25C202A01D9013A19
:1057E00000E07F22E254C8E7A8F103085FFA88F8D6
:1057F000B8F1010FC1D81E4803785A1EA15C2029B8
:1058000001D12039A1541A4A8AF8003000231370BC
:10581000B3E763190693635D4FF0000C8DF82430F5
:105820008DF825C0194B1A4898479AF8003000F1B6
:105830000209013B9D4205905FFA89F940F0BE8064
:10584000635D05FB09F8202B2AD1B04708F1050854
:105850004108FF23009301935FFA88F0C9B20D4A13
:10586000B84755E06B3B0108B5350108BD38010864
:10587000B10400204D1700089E040020A94F000825
:10588000A07A0108A57A0108A97A0108213801083F
:105890003B770108AE7A0108673B010879500008A0
:1058A0000DF1300B08F1050C0BF80C3D5FFA8CFC88
:1058B000CDF810C0B047DDF810C04FF0FF08410828
:1058C0005A466046C9B24346CDF80080CDF8048000
:1058D000B847B0478346B047DDF810C0059BACF130
:1058E00002024FEA5B0B9C444308ABF1020100202B
:1058F00009330090CDF80480D0B2CDF808805FFA6B
:105900008CF2CDF80C80C9B2DBB2DFF8F0C0E04712
:1059100038480378002B5FD005FB09FCC9F1000370
:105920000CF1050CDBB25FFA8CFC079405934FF089
:105930000008644618E0069A0DF1300B1378013B1D
:10594000C8EB03030BF80C3DB0474108FF2304EB01
:1059500009020C39D0B200930193C9B25A46B84734
:1059600008F101085FFA88F8059BA8451C44E4B2D9
:10597000E1D1079C4FF00008A34619E006980CAC53
:1059800003780133434404F80C3DB04708EB0502AB
:1059900002FB09F24108FF2305320C31D0B200931B
:1059A0000193C9B22246B84708F101085FFA88F8A6
:1059B000C5F10E039845E1DB5C460DE0B04705FB01
:1059C00009F94108FF2309F10509009301935FFAE2
:1059D00089F0C9B209AAB8470135EDB22046064A96
:1059E000904701308542FFF414AF00200DB0BDE8B0
:1059F000F08F00BFB10400204D170008B535010835
:105A000037B50B4B0D4693F848300A2B03D9811C50
:105A1000FF23084C04E0084B084C1978FF23411879
:105A2000009301930220C9B22A46A0473EBD00BFA1
:105A300014330020BD380108FC000020753801082F
:105A40002DE9F341DFF85880064698F848300D46B6
:105A50000A2B104F104B114C08D9084698473A783A
:105A600098F84830D2438018073B08E0084698472A
:105A70003B78DFF83080DB43C01898F80030F61828
:105A8000F1B2FF232A46C0B200930193A047BDE8BC
:105A9000FC8100BF44000020D15000087538010887
:105AA00014330020FC00002070B5012386B014469A
:105AB00000220546009303A8134609B2044EB047DE
:105AC000284603A92246034B984706B070BD00BF85
:105AD00049450008415A000837B50E4B0C460546AB
:105AE00098470D4B013593F848200C4B083A19782C
:105AF0006FF012035B1A02EBD27205EB6201C01861
:105B000000230093E2B2C9B20133054CC0B2A047F2
:105B10003EBD00BF673B0108143300204400002055
:105B20009D31010870B5054686B01C46002922D17A
:105B3000012A3E4B05D13E4903A898472846242117
:105B400062E0022A02D103A83A4923E0032A02D1E3
:105B500003A8394955E0042A02D103A8374906E0D1
:105B6000052A02D103A8364914E0364903A898470C
:105B700028462B2148E0012926D1012A2B4B05D1AB
:105B8000314903A89847284625213DE0022A03D140
:105B90002E4903A8984741E0032A05D12C4903A8C0
:105BA0009847284627212FE0042A02D103A8294933
:105BB00006E0052A02D103A82749EBE7274903A8F5
:105BC000984728462A211FE0022908D1032A25D117
:105BD000234903A8154B98472846282114E0032998
:105BE00008D1032A1AD11F4903A8104B9847284609
:105BF000292109E004290AD1032A0FD11A490B4BA4
:105C000003A89847284626212246184B0AE001237C
:105C10000022009303A81346154EB047154B2846A3
:105C200003A92246984706B070BD00BF9116000830
:105C3000B47A0108BB7A0108C37A0108CA7A01085C
:105C4000CD7A0108247B010820800108D57A01085B
:105C500045830108DA7A0108DE7A01081B7B010816
:105C6000E57A0108EC7A0108F37A0108D95A0008AC
:105C700049450008415A000870B5012386B0144612
:105C800000220546009303A8134609B2064EB0470A
:105C900003A80649064B9847284603A92246054B08
:105CA000984706B070BD00BF49450008067B010853
:105CB00049160008415A000837B5064B0D461978B9
:105CC000054C4118FF230320C9B22A4600930193D3
:105CD000A0473EBDFC000020F538010837B5064B53
:105CE0000D461978054C4118FF230320C9B22A46F6
:105CF00000930193A0473EBDFC000020BD38010881
:105D00002DE9F0410E46097888B03F2905469046B6
:105D1000174C04D8174B490102A8C91805E00331F4
:105D2000C9B202291ED8144902A8144B9847144B33
:105D300030469847134E0746134902A8B047134B05
:105D400002A8984701230022009302AB39B2181829
:105D50000F4F1346B8470F4902A8B047284602A97B
:105D6000424600E00C49A04708B0BDE8F08100BF02
:105D7000415A0008C00E0020F87A01089116000868
:105D8000313E000849160008649A01084D170008C2
:105D900049450008067B0108FF7A01082DE9F0411A
:105DA0000E46097886B03F2905461746DFF864801D
:105DB000104C12D8104B4901C91868460F4B984730
:105DC0003046C0470E4B10B168460E4901E00E49FF
:105DD000684698472846694607E03046C04710B1F4
:105DE00028460A4901E00A4928463A46A04706B033
:105DF000BDE8F081415A0008C00E0020911600084D
:105E000049160008087B01080E7B0108157B010874
:105E10001E7B01087D3E0008F0B5DFF888C085B024
:105E200004461D4F1D4E21B397F848303278013B90
:105E300000250121C318C2F118020091284621460D
:105E4000D2B2DBB2019502950395E04797F848304E
:105E50003278013BFF21E318C2F11802019102914F
:105E60000391009521462846D2B2DBB20C4CA047E4
:105E700010E097F848303278013BC318C2F118029D
:105E8000012000900191029103910846D2B221466F
:105E9000DBB2E04705B0F0BD143300204400002021
:105EA000B5350108053401082DE9F043044685B0F5
:105EB0000D46234F234EDFF89480DFF8949041B3D2
:105EC000B84796F8483098F80020013BD2430025A7
:105ED00001218218E318009128462146D2B2DBB294
:105EE000019502950395C847B84796F8483098F849
:105EF0000020013BD243FF218218E3180191029157
:105F00000391009521462846D2B2DBB20E4CA04741
:105F100012E0B84796F8483098F80020013BD24389
:105F200082180121E318009128462146D2B2DBB243
:105F3000019502950395C84705B0BDE8F08300BF01
:105F4000673B010814330020B535010844000020E8
:105F50000534010838B50C46054622460449054B70
:105F6000984728463D212246034B984738BD00BF3D
:105F7000A07A0108015A0008D95A000808B50A4653
:105F8000014B0249984708BD015A0008A07A010850
:105F9000012809D11848002303701078013988427C
:105FA0000ADA0130107025E002280AD1124B0238BB
:105FB0001870137813B1013B13701BE00139117095
:105FC00018E0032807D11978FF290CBF1278FF22A7
:105FD0001A7001220CE0632805D91A78FF2AF8D13B
:105FE00064381870F5E7042804D100221A700132D1
:105FF000024B1A70002070476204002092000020BB
:106000002DE9F0471546444A88B092F800A00446AE
:10601000BAF1010F8E46DFF81C81404E404F25D16A
:10602000B8F800C040F673621FFA8CFC944517D88C
:10603000D6F854C04FF47A72BCFBF2F902FB19C2D5
:10604000B2F5FA7F0CD94FF0FF0E2A185B18CDF885
:1060500000A0CDF804E0CDF808E0CDF80CE02EE08B
:10606000012100912A197344013923E0B8F800C0D6
:1060700041F204021FFA8CFC944516D9D6F854C09C
:106080004FF47A72BCFBF2F902FB19C2B2F5FA7F47
:106090000BD9012205EB000C0092013A0192029209
:1060A00003925B185FFA8CF20AE0012100912A1931
:1060B0007344FE3101910291039120467146D2B2A0
:1060C000DBB2B84796F84930B8F80010642389B2BB
:1060D000B1FBF3F1633B0022009309B205A8114F15
:1060E000B84705A8104B9847104A96F849301178E0
:1060F0002D1A5B1A05EBD57503EBD37304EB65041E
:106100005910FF2300930193E0B2C9B205AA084CCD
:10611000A04708B0BDE8F087F30100201433002049
:1061200005340108494500082138010820010020F4
:10613000BD380108CE06002008B50146014B0248D3
:10614000984708BD91160008560700202DE9F04F2A
:106150004B1EDBB2012B144685B082466F4B704A52
:106160000BD81878884208D16E4805786EB2022E96
:1061700001DC01350570062009E0127850B20028D4
:1061800003DD6748013A027002E0664A00201070A1
:10619000012919700CD1634B22781B7859B2C1F1D7
:1061A00056018A4201DA01330BE08BB156230FE02E
:1061B000022911D15B4B22781B7859B28A4203DD48
:1061C000DB43D218227004E00BB9563300E0002301
:1061D00023702046012106E0042907D123782046B8
:1061E0005B4223700339504B984707E0032905D1E0
:1061F000204602394C4B984701208CE0DFF83C8167
:10620000C0474A4F0546B84700266A1F431F4FF054
:10621000010B0A21D2B2DBB20520DFF82891CDF8BC
:1062200000B0019602960396C847C0470546B84796
:106230006A1F431FFF250A21D2B20520019502954E
:106240000395DBB20096C847394B504698478146C4
:10625000B84781082B46009501954846354DC9B28F
:106260005246A8472378344D5B450AD9B84722786F
:10627000A0F11001023A00960A20C9B2D2B25B46E0
:10628000A84723785BB1B847227841080023023140
:10629000013A00931320C9B2D2B20133A847C047D4
:1062A0000646B84703217608B0FBF1F1F31F06312B
:1062B0000026D8B2227801230096C9B2A8472378D5
:1062C000552B12D81D4B9847184B8146984722787A
:1062D0004108A9F122090231013200965FFA89F0E2
:1062E000C9B2D2B20123144EB0472378542B0ED832
:1062F000C0470646B8472278A0F110010023193E96
:1063000002320093F0B2C9B2D2B20133A84750466C
:106310000B4B9847002005B0BDE8F08F9904002092
:10632000B004002085040020A94F00086B3B010841
:1063300079500008BD3801089D310108673B01080C
:1063400039610008B53501087FB51E4DA8471E4CC0
:106350000121A0F1170294F849301620D2B2009121
:106360001A4E0139019102910391B047A847184B89
:106370000546184898472B3D8542174D10DC174BB2
:106380001448984794F849202B78154CD31A03EBFE
:10639000D3735910FF2300930193C9B20D4A0FE044
:1063A000104B0C48984794F849202B780E4CD31A80
:1063B00003EBD3735910074AFF2300930193C9B22B
:1063C000A0477FBD673B0108143300200534010856
:1063D000213801085607002020010020A5500008A0
:1063E0007538010879500008BD38010870B5264C91
:1063F0004EF66023616D88B0B1FBF3F101250222F6
:106400000023224E05A809B20095B047204905A8EF
:10641000204B984705A8204B9847626D4FF47A733C
:10642000B2FBF3F23C23B2FBF3F103FB112305AA09
:1064300019B21018002302220095B047002094F8EA
:106440004930014616220095019002900390134DA9
:10645000A84705A8124B9847124A94F8493011787A
:10646000C0F116005B1A03EBD37300EBD070591028
:106470004010FF2300930193C9B205AA0A4CC0B291
:10648000A04708B070BD00BF143300204945000884
:106490009E7A0108491600084D17000805340108C6
:1064A0004538010820010020753801082DE9F04F1A
:1064B0002B4C89B007468B46A0472A4E0546B0476D
:1064C0004FF0010A6A1F431F00250A21D2B2DBB236
:1064D0000195029503950520DFF89480CDF800A082
:1064E000C047A0470446B047621F431FFF240A214C
:1064F000D2B2DBB200950520019402940394C04708
:10650000DFF870803846C0478146B04720FA0AF16C
:1065100006393A462346009401944846C9B2DFF84A
:106520005890C8470FFA8BF12A462B46CDF800A0A9
:1065300005A80D4DA84705A8C0470546B04720FA55
:106540000AF106312346009401942846C9B205AAEF
:10655000C8473846054B984709B0BDE8F08F00BFE3
:10656000673B01086B3B0108494500083961000899
:10657000B535010879500008BD3801080000000059
:106580000129F8B50646144610D11568224B284655
:1065900098471DA3D3E90023204FB84720B12846D0
:1065A0004FF07E511E4B11E01E4B13E0022917D114
:1065B0001568194B2846984715A3D3E900231A4FAD
:1065C000B84730B1194B28464FF07E5198472060AC
:1065D00001E0174B236020460421164B984707E043
:1065E000032905D110460131124B98470120F8BD0F
:1065F0002068114B9847114B0146304698470020C0
:10660000F8BD00BFAFF3008085EB51B8FE87C340F3
:1066100085EB51B8FE87C3C045220008D12700088A
:106620005D290008F63F1CC60D28000859290008FE
:10663000F63F1C46A94F0008F92E0008AD6400087B
:10664000F8B54B1EDBB2012B154604462A4B2B4AEC
:106650000BD81878884208D12948067877B2312FAC
:1066600001DC02360670062009E0127850B20028DC
:1066700003DD2248013A027002E0214A0020107036
:10668000012919700CD11E4B2A781B7859B2C1F11F
:10669000FF018A4201DA01330BE08BB1FF230FE0E7
:1066A000022911D1164B2A781B7859B28A4203DD90
:1066B000DB43D2182A7004E00BB9FF3300E000235B
:1066C0002B702846012106E0042907D12B782846A3
:1066D0005B422B7003390B4B984707E0032905D128
:1066E00028460239074B98470120F8BD20462978F3
:1066F000054B98470020F8BDB40400205D0400203D
:1067000089040020A94F0008AD640008F8B54B1EAD
:10671000DBB2012B154604462D4B2E4A0BD81878B8
:10672000884208D12C48067877B2312F01DC023636
:106730000670062009E0127850B2002803DD2548D3
:10674000013A027002E0244A0020107001291970F9
:106750000FD1214B2A781B7850B259B2C1F17F0179
:10676000884201DA01330FE00BB9813313E07F2354
:1067700011E0022913D1184B2A781B7851B258B274
:106780007E38884203DCDB43D2182A7004E00BB960
:106790007F3300E081232B702846012106E0042985
:1067A00007D12B7828465B422B7003390B4B984757
:1067B00007E0032905D128460239084B98470120F4
:1067C000F8BD204695F90010054B98470020F8BD0C
:1067D0009A0400209D04002091040020A94F000885
:1067E000AD6400082DE9F043234C85B094F84A309D
:1067F0008046072B02D9214B984739E0204F94F867
:106800004860B84794F84830002503EB4303821FE3
:1068100001210133D2B2DBB20091019531460295DC
:1068200003950520174EB04794F84890B84794F860
:106830004830821F03EB430300950133FF3549467F
:10684000D2B20520DBB2019502950395B0470E4BFD
:106850004046984794F8481094F84830023101EBCC
:10686000530100950195C9B242462B46074CA047FB
:1068700005B0BDE8F08300BF143300203961000883
:10688000673B0108B535010879500008BD3801089B
:106890002DE9F04F002291B00126DFF80092079019
:1068A0001346794C009608A809B2A04709F512547E
:1068B00094F84A30DFF8E881072BDFF8E8A1DFF829
:1068C000E8B138D9714DA84794F84A300746059386
:1068D000C0478046A847059B08F1FF32DB43FF18FD
:1068E000431E0020F9B2D2B2DBB2009601900290B2
:1068F0000390D04708A8D8470646A847644B94F8A9
:106900004A201B7894F84A10624CCB1A03EBD373DD
:10691000C2EB63014118FF23009301933046C9B2D3
:1069200008AAA047079D5C4B4FEA451CE14409F1CA
:106930002C009847A5E094F8485094F84810002798
:106940000691C04794F8482094F84830821A0133E1
:1069500003EB43032846D2B20699DBB200960197B7
:1069600002970397D04794F8483094F8481005935D
:106970000691C04794F8482094F848E0059B0EF132
:10698000010EFF250EEB4E0E821A06991846D2B262
:106990005FFA8EF30195029503950097D047DDF8D5
:1069A0001CA04FEA4A1C09EB0C0A0AF12C0A5046BB
:1069B000CDF818C0D84794F84810524603312B46FA
:1069C000C9B200950195DFF8CCA0D04708A8D847F8
:1069D00094F848102B464900033100950195C9B23F
:1069E00008AAD047DDF818C094F8480094F8481079
:1069F00009EB0C05383505300531EA793346009747
:106A0000C0B2C9B2DFF8A490C847AB79642B0ED1ED
:106A1000C04794F848206FF0130394F848109B1A6D
:106A2000C01805310097C0B2C9B2422227E095F8DC
:106A300006A0BAF1000F0FD1C04794F848206FF0BC
:106A4000130394F848109B1AC0180531CDF800A024
:106A5000C0B2C9B2432212E0AB795BB213F1640F4A
:106A60000FD1C04794F848206FF0130394F84810F2
:106A70009B1AC01805310097C0B2C9B244223346F0
:106A8000C84711B0BDE8F08F494500086B3B0108CD
:106A900020010020BD38010839610008940E002053
:106AA000673B0108B5350108795000089D310108A0
:106AB0002DE9F043254F85B089460546B847244E59
:106AC0000446B04700210091AB310191A4F10A02C4
:106AD0002231FF24A0F10C030A20D2B2DBB20291D2
:106AE000DFF8788001460394C047B8470746B047AF
:106AF000012100914231019122390291A7F10C024A
:106B00001239A0F10C030C200391D2B20146DBB282
:106B1000C047104F2846B847DFF8448014212A4662
:106B2000234600940194C0474846B8470746B047FB
:106B300041082346009401943846C9B24A46C047EA
:106B40002846054B984705B0BDE8F083673B010830
:106B50006B3B01087950000839610008B535010820
:106B6000BD3801082DE9F04F8FB005469DF8600053
:106B70007B4F0D9209930C9089468046B847794C1B
:106B8000794E94F849A094F84A30CAEB000AC3EB56
:106B90000A0A94F848C05FFA8AFABAFBFCFC0CF1C6
:106BA000FF3C5FFA8CFCCDF814C0704B2846984728
:106BB00094F849B0B0470546B84794F84A306A1E81
:106BC00001210025C31AD2B22846DBB200910195FB
:106BD00059460295DFF8A4B10395D84794F84910B7
:106BE0000691B84794F8493094F84A20DDF824E03B
:106BF0000699C31AD243BAFBFEFAD218043951449B
:106C0000CDF82CA0CAEB020A08FB0AFA0EF1FF3EEF
:106C10009AFBFEFACDF824E08A44B047544A94F82F
:106C2000493011780A93C1F101014118C9B20691A6
:106C3000B0470790B847079B94F84A2003F1FF3EFE
:106C40006FF0010306999B1AC31801205FFA8EF2B8
:106C5000DBB200900195084602950A990395D84742
:106C6000B047434A94F8493011780A93C1F10101C1
:106C70004118C9B20691B0470790B847079B94F8EE
:106C80004A2003F1FF3E6FF0010306999B1A5FFA59
:106C90008AFAAA4508BF4FF0010AC3180095FF35CC
:106CA0005FFA8EF20846DBB20A99019502950395C8
:106CB000D847B0472E490B7894F84910C3F1030325
:106CC000C318DBB20A930691B84794F8497094F858
:106CD0004A2007900892B047079B089ADF1BBF1A0B
:106CE0000B9A099BBF1A08FB07F7069997FBF3F766
:106CF0000231C21EC91901200AF10103C9B2009074
:106D0000DBB20195029503950A98D2B2D84799F85B
:106D10000030DDF814C0434584BF0C9989F8001099
:106D2000E04508D999F8003063449845C4BFCCEBDE
:106D3000080889F8008099F800300D9A01339C44C6
:106D40000C4B82F800C094F848201B78D31A03EB50
:106D5000D3735B10084A013313700FB0BDE8F08F96
:106D60006B3B010814330020673B010839610008C0
:106D70004400002020010020FC000020B53501085F
:106D80002DE9F04F8FB09C469DF86030CDF814C0CF
:106D9000514F0B9209931D4688460646B8474F4C03
:106DA0004FF0010B94F8491094F84A20C1EB000908
:106DB00094F84830C2EB0909304699FBF3F9484B87
:106DC000984794F849A0B84794F84A300026C31A67
:106DD0001B2230465146DBB2DFF810A10196029625
:106DE0000396CDF800B0D04794F8491009F1FF3967
:106DF0000791B84794F84A300096C31AFF36162018
:106E000007991A22DBB2019602960396D04794F8AE
:106E100049205FFA89F90692B84794F849100C9016
:106E200094F84A3094F84900079108930A90B847BB
:106E300094F84970089B0D9707996FF00307FF1AA4
:106E40000C9B7F1AFF186F43DDF814C0069A0A9B4B
:106E500097FBFCF794F84AE00232D2196FF0040174
:106E60005F1D0D9BCEEB0101C91A0918694391FB07
:106E7000FCFC07EB0C031720D1B2DBB21922CDF8D2
:106E800000B0019602960396D04798F80030AB42C6
:106E900084BF099F88F800704D4508D998F80030E4
:106EA0004B449D42C4BFC9EB050588F8005098F8D3
:106EB0000030013399440B9B83F80090094B94F800
:106EC00048201B78D31A03EBD3735B10064A0133B7
:106ED00013700FB0BDE8F08F6B3B01081433002036
:106EE0003961000820010020FC000020B5350108B0
:106EF0002DE9F04F87B09DF840509DF844A09DF8D3
:106F000048B0059004911E4617460AEB03090BEBA7
:106F100005083E4CDAB901235FFA89F95FFA88F86F
:106F200000930192029203924346304629464A4614
:106F3000A047049B012B66D1FE3301930293039378
:106F40000097304629464A464346A0475BE0002763
:106F500001235FFA89F95FFA88F8009301974346A5
:106F600002970397304629464A46A047049B012BC7
:106F700009D1FE33019302930393009730462946CB
:106F80004A464346A047BAF13C0F2FD906EB5A0AAE
:106F9000FF245FFA8AFAEB1C1D4F504629465246E1
:106FA000DBB2009401940294B847A8F10301434670
:106FB0005046C9B2524600940194029405EB5B0816
:106FC000B8475FFA88F8F21C30464146D2B24346D1
:106FD000009401940294B847A9F10300009401942D
:106FE0000294C0B241464A464346B847BBF1280F17
:106FF00009D9FF23B01CA91C00930193C0B2C9B2E8
:10700000059A044CA04707B0BDE8F08F053401088D
:1070100009370108753801082DE9F04F814693B012
:107020009DF878500D9199F9001008936943C82391
:10703000680891FBF3F19DF87CA04118C9B2059155
:107040004FEA5A01079199F90110079C01FB0AF1D7
:1070500091FBF3F39DF870809DF87460E318DBB248
:10706000114609900693924801224346914C00969E
:107070000195CDF808A0A0470998089900EB0803EE
:1070800001FB05F040F6FE7C90FBFCF01818FF2792
:10709000C0B20AEB06030246CDF810C00097019774
:1070A00002973146DBB2DFF818B2D847824C642130
:1070B00008224B460898A0470AFB00F0079ADDF823
:1070C00010C0931990FBFCF15918C9B205EB0802E6
:1070D0000097019702974046D2B20B46D847FF3F30
:1070E00003E0CDF818C0CDF814B009EB070219F988
:1070F00007B092F901C00BFB05FB0CFB0AFCC8238F
:10710000099C07989BFBF3FB9CFBF3FCA344844482
:107110003C2D5FFA8BFB5FFA8CFC19D90CEB060354
:107120000BEB0802D2B2DBB20024501E591E0094B1
:107130000132FF340133019402940394CDF810C05E
:10714000C0B2C9B2D2B2DBB25C4CA047DDF810C00D
:107150000599069AFF240CEB060301EB0800911930
:107160000BEB0802009401940294CDF810C0C0B259
:10717000C9B2D2B2DBB2524C0437A047202FDDF89F
:1071800010C0AED10D98002109EB8000059006914A
:10719000C346B1460D9A069B9A427FD1059CC823EF
:1071A00094F9002094F901C06A430CFB0AFC099889
:1071B00092FBF3F207998218D2B29CFBF3FC8C4449
:1071C00002EB0B035FFA8CFCDBB20C920CEB0908B0
:1071D000DA1E03335FFA88F8DBB20A9308F103037F
:1071E000FF24D2B2DBB20026A8F1030108921046B8
:1071F0000B930096019402940394C9B20A9A2F4FFC
:10720000CDF810C0B847642D48D9059A012392F9EA
:1072100000102C4F324600930FA83346B8472A4936
:107220002A4B0FA898472A4B0FA89847059A012385
:1072300092F901100FAA0093101833463246B8474E
:107240000C9B0998234E8342DDF810C015D3079993
:10725000214B8C4509D30FA89847089AA8F10B0138
:10726000101A00940194C0B214E00FA89847089B2C
:107270000094181A0194C0B205E00798844504D21E
:107280000A98009401940B9905E00A98A8F10B0163
:1072900000940194C9B20FAA2346B04706994B1C2B
:1072A000DBB2082B06937FF475AF13B0BDE8F08F07
:1072B000877B0108F16E0008913D00080534010844
:1072C0000937010849450008287B010849160008CC
:1072D0004D170008BD380108213801082DE9F04399
:1072E0000446994610F8043B85B03F2B0E461746DE
:1072F0009DF83080134B144D13D898470246204612
:1073000010F8143B11495B015B18B3F804E0FF214E
:1073100000960197CDF80890CDF80C800FFA8EF307
:107320000BE09847009602460197CDF80890CDF8FB
:107330000C8004F11400FF210023A84705B0BDE82C
:10734000F08300BF7D3E000819700008CC0E0020BD
:10735000F7B50C4606461F460846144B114698479B
:10736000134D14492046A8472046134B9847002246
:1073700001230093394613462018104FB84710498F
:107380002046A84720460F4B98470F4B93F84810CC
:1073900093F848200139091893F8483091FBF2F22C
:1073A0005343D8B2B04238BF3046FEBD91160008F4
:1073B000491600082A7B01084D17000849450008B6
:1073C000997B010845380108143300202DE9F04F5E
:1073D00087B099469DF840C00023824604910592EB
:1073E0001C462749342202FB031202F5A452303214
:1073F00012798B46524501D10134E4B20133402B5E
:10740000EFD1002C38D000252E462746E046342008
:1074100068430BEB000303F5A45330331B79DFF80B
:1074200060C053451FD1049B6044C9EB0301059B19
:1074300000F5A4505A1CB8FBF7F3023BB218DBB2BC
:107440000093CDF80CC04B463430C9B2D2B20D4CCB
:10745000A047DDF80CC00CF5125348331B78B3FB82
:10746000F7F3F618F6B20135402DD0D1064B93F85C
:1074700048000130C0B200E0204607B0BDE8F08F00
:10748000940E0020DD7200081433002010B5002394
:107490000C4A342101FB032101F5A45292F840402B
:1074A0003832844208D0927A824205D001F5A65241
:1074B0001179814218BF92790133402BE8D1002025
:1074C00010BD00BF940E00202DE9F04F8DB007468F
:1074D0009DF858009B460390654B894616469DF8DB
:1074E0005CA09847634B644A1978342303FB072355
:1074F00003F5A45393F8344090463F2C00F2B48037
:1075000093F84020411A01EBD171CBEB6104383381
:107510003F2AE4B219D81A7A182101FB02825B7A59
:1075200002F50262204604A90C325BB2534CA0471C
:10753000FF230446C0EB0900514D00930193C0B2F4
:10754000314604AAA847082500E00025342303FBA0
:10755000078303F5A45393F8422038333F2A1CD8FD
:107560009A7A4549182000FB0212DB7A02F5026282
:10757000204604A90C325BB2404CA047A91904462E
:10758000C0EB0900FF23DFF8F8C0C0B2C9B204AAFB
:1075900000930193E0470835EDB2342303FB0783E2
:1075A00003F5A6531A793F2A1CD81A7932491820B4
:1075B00000FB02125B7902F50262204604A90C323C
:1075C0005BB22E4CA047A9190446C0EB0900FF236B
:1075D000DFF8ACC0C0B2C9B204AA00930193E0477F
:1075E0000835EDB2342303FB078303F5A6539A79DC
:1075F0003F2A1AD89A792049182000FB0212DB7919
:1076000002F50262204604A90C325BB21B4CA04773
:10761000A9190446C0EB0900FF23DFF864C0C0B21B
:10762000C9B204AA00930193E047342303FB078700
:1076300003980634E4B2C4EB0909831EDBB2CBEB3A
:107640000901721C07F5A45000933430D2B25B4696
:10765000C9B20C4DA8470C4B93F8482093F848004A
:1076600001302418E0B200E000200DB0BDE8F08F3A
:10767000673B010844000020940E0020517300086D
:1076800075380108DD720008143300202DE9F04F31
:1076900095B09DF878C09DF87C509DF880900D9035
:1076A0000C920993CDF800C00122634CCDF818C0AC
:1076B0000195CDF808906148A047DDF818C04FEA61
:1076C0005903099C6A080B93634402EB04080027E2
:1076D000DBB20A925FFA88F8079308973C46CDF828
:1076E0004CC02E4678E0DFF884B12046D8470546E6
:1076F0003046D847DFF878A14FF07C51D047504B47
:10770000014628469847054609FB04F04D4B90FB7F
:10771000F6F09847CDE90E0129462846D04729467C
:10772000D047494B01460593284698478446474A27
:107730000B98CDF818C09047DDF818C00146604698
:10774000D047059B014628469847414DA847CDE9BB
:1077500010010D98D847A84700223E4B3E4DA84740
:107760003E4D02460B46DDE91001A8473C4D02465E
:107770000B46DDE90E01A8473A4B9847DDF81CC0DF
:10778000089D5FFA80FA07EB0C0105EB080004EB9B
:107790000802FF250AEB0C03009501950295C0B283
:1077A000C9B2D2B2DBB2DFF8C0C0E047089A079B8B
:1077B000C2EB0800D91BC4EB0802CAEB0303009517
:1077C00001950295DBB2C0B2C9B2D2B2264DA8472C
:1077D000631C08945746DCB2DDF828C0644582D3A8
:1077E0000C9A354602FB06F0C826DDF84CC090FB2B
:1077F000F6F08044FF245FFA88F009EB0C03614641
:107800000246009401940294DBB2174FB847DDF8AA
:1078100030C0079A0CFB09F1099B91FBF6F1511856
:10782000C9B2EA181846009401940294D2B20B46E9
:10783000B84715B0BDE8F08FF16E00082C7B010849
:10784000D52C00082122000859290008C52A000863
:10785000452200080000594041250008ED2200089B
:10786000891F00087128000809370108BD2A00088F
:107870006D2B00082DE9F04F8BB09DF854509DF80A
:1078800058809DF85C709DF860B008910992194687
:1078900001222B46CDF800800197CDF808B0354C79
:1078A0009DF950A0A047089A4FEA5B0C02FB0CF12F
:1078B00005EB5703DBB20CEB080606936FF063038E
:1078C000F6B291FBF3F17118FF24DFF8AC90284673
:1078D000069A3346C9B2CDF814C0009401940294BC
:1078E000C847DDF814C0099A7B19DBB2079302FB85
:1078F0000CF34FF0640C93FBFCF3F318069831463D
:10790000079ADBB2CDF814C0009401940294C847E2
:107910000AFB07F0C82390FBF3F0069B41461818BA
:10792000C0B20BEB08030246DBB200940194029450
:10793000C847BAF1000FCBBF099A089B02FB0AFAAD
:1079400003FB0AFADDF814C0C8239AFBFCFC4FFACB
:107950008CFC0BFB0CFC9CFBF3FC66443733F1B254
:107960000093019302932846079A0B46C8470BB031
:10797000BDE8F08FF16E0008093701082DE9F04FDE
:107980009946454B8BB0064605930846BDF950A075
:107990009DF854509DF858809DF85C709DF860B03B
:1079A00014469847059B0890204698473B4C099001
:1079B0004946304601222B46CDF800800197CDF88C
:1079C00008B0A047089A4FEA5B0C0CFB02F105EBEC
:1079D0005703DBB20CEB080606936FF06303F6B2B5
:1079E00091FBF3F1FF247118DFF8B4902846069A52
:1079F0003346CDF814C0009401940294C9B2C8472C
:107A0000DDF814C0099A7B19DBB207930CFB02F373
:107A10004FF0640C93FBFCF3F318CDF814C00698F8
:107A20003146079A009401940294DBB2C8470AFBDE
:107A300007F040F6FE7390FBF3F0069B41461818E2
:107A4000C0B20BEB08030246DBB20094019402942F
:107A5000C847BAF1000FCBBF099A089B0AFB02FA8C
:107A60000AFB03FADDF814C040F6FE739AFBFCFC37
:107A70000FFA8CFC0BFB0CFC9CFBF3FC6644FF2315
:107A8000F1B20093019302932846079A0B46C84728
:107A90000BB0BDE8F08F00BF313E0008F16E00086A
:107AA000093701082DE9F04F8DB0BDF958C00646E1
:107AB0009DF86800CDF814C00990534F08469DF812
:107AC0005C809DF860A09DF8649014461D46B84700
:107AD0000A902046B84709990B90CDF8049002917E
:107AE0003046294601224346CDF800A0474CA04726
:107AF0000A9B4FEA590B0BFB03F20BEB08076FF0E5
:107B00006303FFB2099892FBF3F20A99BA1840088E
:107B1000D2B2079200FB01F200EB0A06F6B292FB2A
:107B2000F3F3F318FF24DBB2394D0690089307985E
:107B300019463A463346009401940294A84708999E
:107B40004046079A0B46009401940294A8470B9A6A
:107B500006980BFB02F34FF0640B93FBFBF3FB184F
:107B6000DBB2079300FB02F393FBFBF3F318DBB2EA
:107B7000069338463146079A009401940294A84728
:107B8000069909EB0803DBB2089307981A4600949C
:107B90000B4601940294A847DDF814C040F6FE732A
:107BA0000CFB09F9099999FBF3F94F44F8B201EB81
:107BB0000A030246DBB25146009401940294A8479E
:107BC000DDF814C00998BCF1000FCBBF0B9A0A9BDB
:107BD0000CFB02FC0CFB03FC9CFBFBFB0FFA8BFB7E
:107BE00000FB0BFB40F6FE739BFBF3FB5E44FF23A5
:107BF000F1B20093019302934046089A0B46A847BE
:107C00000DB0BDE8F08F00BF313E0008F16E0008F6
:107C1000093701082DE9F04F8DB0064609929DF80D
:107C200058009DF85C200A930023894608900B9227
:107C30001D46FF2E09D14B4A0C2101FB032202F500
:107C40009452303212794A450FD0B9F1FF0F0ED15C
:107C5000DAB296420BD1434A0C2101FB062202F50F
:107C60009452303212793F2A01D80135EDB20133F6
:107C7000102BDED1002D70D00024A246A846FF2E86
:107C800009D1384B0C2202FB043303F594533033F3
:107C90001B794B450FD0B9F1FF0F55D1E3B29E428E
:107CA00052D1304B0C2202FB063303F59453303390
:107CB0001B793F2B48D84FF00C0B0BFB04FB294FD3
:107CC0000BF59453FA183C32274D06931046079251
:107CD000A847079A014607911046A847069B054604
:107CE000FB1803F13800214B9847BB440BF5945225
:107CF0003032127903465201BA1838329279DDF8DF
:107D000024E0089852B20092C0EB0E020A98D2B258
:107D10000192421C5244D2B20292DDF82CE0089A41
:107D200013480392BEFBF8F2023AD2B204920799CA
:107D30002A4607F512570F4DA84797F84830B3FB6E
:107D4000F8F39A445FFA8AFA0134102C97D10A4B5F
:107D500093F848000130C0B200E028460DB0BDE8FD
:107D6000F08F00BF940E0020313E00087D3E0008D9
:107D7000317B010875780008143300202DE9F04F9D
:107D800089B006469DF84C0006939DF848B0002344
:107D90008946059207901D46FF2E09D1454A0C21C0
:107DA00001FB032202F58E52303212794A450FD080
:107DB000B9F1FF0F0ED1DAB296420BD13D4A0C2138
:107DC00001FB062202F58E52303212793F2A01D889
:107DD0000135EDB20133102BDED1002D65D000242A
:107DE000A246A846FF2E09D1324B0C2202FB0433D7
:107DF00003F58E5330331B794B450FD0B9F1FF0F8C
:107E00004AD1E3B29E4247D12A4B0C2202FB0633F1
:107E100003F58E5330331B793F2B3DD80C2565433A
:107E2000244F05F58E53F818234A04933C309047AD
:107E3000049B8446FB1803F13800CDF810C01F4B9B
:107E400098477D1905F58E5595F83430059D5B01F1
:107E5000FB1893F83E20CBEB0503069D0146681CFA
:107E60005044079DC0B20090A81EDDF810C090FBE2
:107E7000F8F0C0B20290DBB2CDF804B05FFA8CF03B
:107E800052B20F4D07F51257A84797F84830B3FB89
:107E9000F8F39A445FFA8AFA0134102CA2D1094B04
:107EA00093F848000130C0B200E0284609B0BDE8B0
:107EB000F08F00BF940E0020313E00087D3E000888
:107EC0008D760008143300202DE9F04F8DB0064662
:107ED00009929DF858009DF85C200A93002389467A
:107EE00008900B921D46FF2E09D14C4A142101FB2C
:107EF000032202F59A52303252794A450FD0B9F135
:107F0000FF0F0ED1DAB296420BD1444A142101FB85
:107F1000062202F59A52303252793F2A01D80135B1
:107F2000EDB20133102BDED1002D72D00024A24619
:107F3000A846FF2E09D1394B142202FB043303F566
:107F40009A5330335B794B450FD0B9F1FF0F57D1BE
:107F5000E3B29E4254D1314B142202FB063303F5A7
:107F60009A5330335B793F2B4AD84FF0140B0BFBFD
:107F700004FB2A4F0BF59A5303F13802D219284D0E
:107F80000693101D0792A847079A0146079102F130
:107F90000800A847069B0546FB1803F13800214B53
:107FA0009847BB440BF59A5230325279034652013E
:107FB000BA1838329279DDF824E0089852B200926B
:107FC000C0EB0E020A98D2B20192421C5244D2B2C5
:107FD0000292DDF82CE0089A13480392BEFBF8F2F7
:107FE000023AD2B2049207992A4607F512570F4D6A
:107FF000A84797F84830B3FBF8F39A445FFA8AFA37
:108000000134102C95D10A4B93F848000130C0B2CE
:1080100000E028460DB0BDE8F08F00BF940E0020B0
:10802000313E00087D3E00083A7B01087578000863
:10803000143300202DE9F04F8DB00A939DF85C3089
:108040009DF858B00B9300230646894609921D46B9
:10805000FF2E08D103F506724349033201EB0212E9
:1080600012794A450ED0B9F1FF0F0DD1DAB296421E
:108070000AD106F506723C49033201EB021212796D
:108080003F2A01D80135EDB20133102BE0D1002D8C
:1080900065D00024A2462F46FF2E08D104F50673B2
:1080A000314A033302EB03131B794B450ED0B9F170
:1080B000FF0F4BD1E3B29E4248D106F506732A4A20
:1080C000033302EB03131B793F2B3FD82201DFF868
:1080D000988002F50652383204F50675424403359D
:1080E00002F1080108EB0515043205F108001F4BE9
:1080F00008910792984703462879182505FB0080C8
:1081000000F5026040198088099D00B20090CBEB19
:1081100005000A9DC0B20190681C50440B9DC0B27E
:108120000290B5FBF7F00238C0B20490CDF80CB065
:108130000F480899079A0F4DA84708F5125348337E
:108140001B78B3FBF7F39A445FFA8AFA0134102CD8
:10815000A2D1094B93F848000130C0B200E0284694
:108160000DB0BDE8F08F00BF940E00207D3E0008EA
:10817000417B01087D790008143300202DE9F04F80
:108180008DB00A939DF85C309DF858B00B93002396
:108190000646894609921D46FF2E08D103F50A724C
:1081A0004349033201EB021212794A450ED0B9F16C
:1081B000FF0F0DD1DAB296420AD106F50A723C4998
:1081C000033201EB021212793F2A01D80135EDB2D8
:1081D0000133102BE0D1002D65D00024A2462F469C
:1081E000FF2E08D104F50A73314A033302EB03135F
:1081F0001B794B450ED0B9F1FF0F4BD1E3B29E4234
:1082000048D106F50A732A4A033302EB03131B799C
:108210003F2B3FD82201DFF8988002F50A5238320E
:1082200004F50A754244033502F1080108EB05150F
:10823000043205F108001F4B089107929847034646
:108240002879182505FB008000F502604019808818
:10825000099D00B20090CBEB05000A9DC0B20190D1
:10826000681C50440B9DC0B20290B5FBF7F0023879
:10827000C0B20490CDF80CB00F480899079A0F4D82
:10828000A84708F5125348331B78B3FBF7F39A4419
:108290005FFA8AFA0134102CA2D1094B93F84800F6
:1082A0000130C0B200E028460DB0BDE8F08F00BF3D
:1082B000940E00207D3E0008457B0108A57A000849
:1082C000143300202DE9F04F8FB081469DF86400F3
:1082D00090460022079106901346B048342101FBD6
:1082E000020101F5A45191F838404C4503D03831D2
:1082F0000979494501D101339BB20132402AECD1C1
:10830000403ADFF898C20C2101FB02C101F58E5101
:1083100091F83800484503D038310979494501D1F1
:1083200001339BB20132102AEBD1103A9B480C2149
:1083300001FB020101F5945191F83800484503D042
:1083400038310979494501D101339BB20132102AF4
:10835000ECD1103ADFF844C2142101FB02C101F54F
:108360009A5191F83800484507D091F83C003831CF
:10837000484502D0097A494501D101339BB2013207
:10838000102AE7D1103A02F506718448033100EB58
:108390000111097A49450ED002F58071013100EBD7
:1083A000011101F58C5191F82C002831484502D07B
:1083B000097A494501D101339BB20132102AE2D139
:1083C000103A02F50A71DFF8D4C103310CEB011148
:1083D000097A49450ED002F5887101310CEB011183
:1083E00001F58C5191F82C002831484502D0097ACA
:1083F000494501D101339BB20132102AE1D1002B52
:1084000000F0A285664A042B28BF0423049392F847
:1084100048200498931E93FBF0F303EBD3735B1097
:10842000023BDBB24FF0000B079DCA4605931C468A
:108430005E46C146594A342707FB0B2707F5A45768
:1084400097F83830303753453AD15649564B08A83B
:1084500098473979514B490159182C31534B08A889
:108460009847534F08A8B847A5F10A03181A04EB18
:108470000901FF23DFF8488100930193C9B208AADC
:10848000C0B2C047DFF83C81DDF810C098F800307A
:1084900008A8023B93FBFCF3E418B847B042E4B2EF
:1084A00003D908A8424B9847064698F80030013B8C
:1084B000A34205DC0F3DAD1B059C05F0FF05002622
:1084C000342000FB0BF0354A02EB000C0CF5A45CE9
:1084D0009CF83C3053454FD10DF13808002708F87F
:1084E000187D0CF13C00CDF80CC0324B98470123AD
:1084F0003A460146009340463B462F4FB8472B4F24
:1085000040462E49B847DDF80CC040469CF8341070
:10851000DFF888C0490161442C31B847244F4046F8
:10852000B847A5F10A034246181A04EB0901FF23D4
:10853000DFF8908000930193C9B2DFF884C0C0B225
:10854000E04798F800300498023B93FBF0F308A84A
:10855000E418B847B042E4B203D908A8144B9847CE
:10856000064698F80030013BA34205DC0F3DAD1BE9
:10857000059C05F0FF0500260BF1010BBBF1400F38
:108580007FF458AFABF1400B044A0C2707FB0B27D5
:1085900007F58E5797F8383016E000BF940E00208C
:1085A000143300204E7B010891160008491600087C
:1085B00045380108313E0008494500084D7B010857
:1085C000753801085C330020303753453AD1AF4944
:1085D000AF4B08A898473979AE4B490159182C314F
:1085E000AD4B08A89847AD4F08A8B847A5F10A03B6
:1085F000181A04EB0901FF23DFF8BC8200930193F2
:10860000C9B208AAC0B2C047DFF8B082DDF810C016
:1086100098F8003008A8023B93FBFCF3E418B84735
:10862000B042E4B203D908A89C4B9847064698F894
:108630000030013BA34205DC0F3DAD1B059C05F05E
:10864000FF0500260C2000FB0BF0924A02EB000C09
:108650000CF58E5C9CF83C3053454FD10DF1380839
:10866000002708F8187D0CF13C00CDF80CC08C4BAD
:10867000984701233A460146009340463B46894FBE
:10868000B847854F40468849B847DDF80CC040469A
:108690009CF83410DFF8FCC1490161442C31B84723
:1086A0007E4F4046B847A5F10A034246181A04EB2C
:1086B0000901FF23DFF8048200930193C9B2DFF8B8
:1086C000F8C1C0B2E04798F800300498023B93FB31
:1086D000F0F308A8E418B847B042E4B203D908A8F8
:1086E0006E4B9847064698F80030013BA34205DCE4
:1086F0000F3DAD1B059C05F0FF0500260BF1010B9E
:10870000BBF1100F7FF440AFABF1100B614A0C27A7
:1087100007FB0B2707F5945797F838303037534548
:108720003AD162495A4B08A898473979594B4901BF
:1087300059182C31584B08A89847584F08A8B847E3
:10874000A5F10A03181A04EB0901FF23DFF8688179
:1087500000930193C9B208AAC0B2C047DFF85C8198
:10876000DDF810C098F8003008A8023B93FBFCF33A
:10877000E418B847B042E4B203D908A8474B984779
:10878000064698F80030013BA34205DC0F3DAD1BC7
:10879000059C05F0FF0500260C2000FB0BF03D4A70
:1087A00002EB000C0CF5945C9CF83C3053454FD127
:1087B0000DF13808002708F8187D0CF13C00CDF8C1
:1087C0000CC0374B984701233A4601460093404678
:1087D0003B46344FB847304F40463549B847DDF83F
:1087E0000CC040469CF83410DFF8A8C04901614431
:1087F0002C31B847294F4046B847A5F10A034246F5
:10880000181A04EB0901FF23DFF8B08000930193ED
:10881000C9B2DFF8A4C0C0B2E04798F800300498AD
:10882000023B93FBF0F308A8E418B847B042E4B267
:1088300003D908A8194B9847064698F80030013B21
:10884000A34205DC0F3DAD1B059C05F0FF0500268E
:108850000BF1010BBBF1100F7FF458AFABF1100B14
:108860000C4B142707FB0B3707F59A5797F838205E
:108870003037524555D10F49054B08A898477979AB
:10888000044A490151182C311AE000BF557B0108F8
:1088900091160008940E002049160008453801087A
:1088A000313E000849450008547B01085C7B010803
:1088B0005B7B0108627B0108753801085C3300208E
:1088C000AE4B08A89847AE4F08A8B847A5F10A03D1
:1088D000181A04EB0901FF23DFF8C4820093019307
:1088E000C9B208AAC0B2C047DFF8B882DDF810C02C
:1088F00098F8003008A8023B93FBFCF3E418B84753
:10890000B042E4B203D908A89D4B9847064698F8B0
:108910000030013BA34204DC0F3DAD1B059C05F07C
:10892000FF05142000FB0BF0964A02EB000C0CF53F
:108930009A5C9CF83C3053454FD10DF13808002724
:1089400008F8187D0CF13C00CDF80CC08E4B984710
:1089500001233A460146009340463B468B4FB847B9
:10896000864F40468A49B847DDF80CC040469CF81F
:108970003510DFF810C2490161442C31B847804FEF
:108980004046B847A5F10A034246181A04EB09010C
:10899000FF23DFF8108200930193C9B2DFF800C211
:1089A000C0B2E04798F800300498023B93FBF0F324
:1089B00008A8E418B847B042E4B203D908A8704B3D
:1089C0009847064698F80030013BA34205DC0F3D6E
:1089D000AD1B059C05F0FF050026142000FB0BF0E5
:1089E000684A02EB000C0CF59A5C9CF84030534549
:1089F00050D10DF138080027101808F8187D624B87
:108A0000CDF80CC000F59C50984701233A4601462A
:108A1000009340463B465D4FB847584F40465C493F
:108A2000B847DDF80CC040469CF83510DFF854C15B
:108A3000490161442C31B847514F4046B847A5F130
:108A40000A034246181A04EB0901FF23DFF8548198
:108A500000930193C9B2DFF848C1C0B2E04798F86B
:108A600000300498023B93FBF0F308A8E418B847E1
:108A7000B042E4B203D908A8414B9847064698F89B
:108A80000030013BA34205DC0F3DAD1B059C05F00A
:108A9000FF0500260BF1010BBBF1100F7FF4E0AED8
:108AA000ABF1100B0BF50677364A033702EB0717CD
:108AB0003B7A534539D13749374B08A8984739791C
:108AC000304B490159182C312C4B08A898472C4F92
:108AD00008A8B847A5F10A03181A04EB0901FF23F7
:108AE000DFF8BC8000930193C9B208AAC0B2C047A6
:108AF000DFF8B080DDF810C098F8003008A8023B1D
:108B000093FBFCF3E418B847B042E4B203D908A8D9
:108B10001B4B9847064698F80030013BA34204DC03
:108B20000F3DAD1B059C05F0FF050BF58070013076
:108B3000DFF850C000010CEB000303F58C53283321
:108B40001B7953456CD160440DF13808002700F5BE
:108B50008C5008F8187D2C30CDF80CC00A4B984783
:108B600001233A460146009340463B46074FB8472B
:108B7000024F40460949B84716E000BF49160008B1
:108B800045380108940E0020313E00084945000890
:108B9000617B0108687B010891160008677B01086A
:108BA000753801085C330020DDF80CC00BF5067346
:108BB00003330CEB03131B7940465B019C440CF11F
:108BC0002C01B847B04F4046B847A5F10A034246CA
:108BD000181A04EB0901FF23DFF8D08200930193F8
:108BE000C9B2DFF8CCC2C0B2E04798F800300498B0
:108BF000023B93FBF0F308A8E418B847B042E4B294
:108C000003D908A8A04B9847064698F80030013BC6
:108C1000A34205DC0F3DAD1B059C05F0FF050026BA
:108C20000BF580700130DFF874C200010CEB00031B
:108C300003F58C5328331B7A534554D160440DF10E
:108C40003808002700F58C5008F8187D3030CDF832
:108C50000CC08E4B984701233A460146009340468C
:108C60003B468B4FB8478B4F40468B49B847DDF8A2
:108C70000CC00BF5067303330CEB03131B79404652
:108C80005B019C440CF12C01B8477F4F4046B8472C
:108C9000A5F10A034246181A04EB0901FF23DFF885
:108CA0000C8200930193C9B2DFF804C2C0B2E0475E
:108CB00098F800300498023B93FBF0F308A8E418FE
:108CC000B847B042E4B203D908A86F4B98470646AC
:108CD00098F80030013BA34205DC0F3DAD1B059C1D
:108CE00005F0FF0500260BF1010BBBF1100F7FF41F
:108CF000D9AEC846ABF1100B0BF50A77674A0337BC
:108D000002EB07173B7A534539D16549654B08A8F3
:108D100098473979614B490159182C315D4B08A8A6
:108D20009847594F08A8B847A5F10A03181A04EB49
:108D30000901FF23DFF8788100930193C9B208AAE3
:108D4000C0B2C047DFF86481DDF810C098F8003089
:108D500008A8023B93FBFCF3E418B847B042E4B226
:108D600003D908A8484B9847064698F80030013BBD
:108D7000A34204DC0F3DAD1B059C05F0FF050BF580
:108D800088700130DFF814C100010CEB000303F51B
:108D90008C5328331B79534554D160440DF1380866
:108DA000002700F58C5008F8187D2C30CDF80CC049
:108DB000364B984701233A460146009340463B46CE
:108DC000334FB847334F40463749B847DDF80CC0FA
:108DD0000BF50A7303330CEB03131B7940465B015D
:108DE0009C440CF12C01B847274F4046B847A5F1E9
:108DF0000A034246181A04EB0901FF23DFF8AC808E
:108E000000930193C9B2DFF8A8C0C0B2E04798F858
:108E100000300498023B93FBF0F308A8E418B8472D
:108E2000B042E4B203D908A8174B9847064698F811
:108E30000030013BA34205DC0F3DAD1B059C05F056
:108E4000FF0500260BF588700130DFF850C00001E7
:108E50000CEB000303F58C5328331B7A53456CD17C
:108E600060440DF13808002700F58C5008F8187D93
:108E70003030CDF80CC0054B984701233A460146E7
:108E80000093404616E000BF45380108313E000817
:108E90004945000849160008677B0108940E002028
:108EA0006E7B010891160008737B01085C3300207B
:108EB000753801083B46284FB847284F4046284997
:108EC000B847DDF80CC00BF50A7303330CEB031342
:108ED0001B7940465B019C440CF12C01B847214FA3
:108EE0004046B847A5F10A034246181A04EB0901A7
:108EF000FF23DFF8748000930193C9B2DFF86CC0E0
:108F0000C0B2E04798F800300498023B93FBF0F3BE
:108F100008A8E418B847B042E4B203D908A8114B36
:108F20009847064698F80030013BA34205DC0F3D08
:108F3000AD1B059C05F0FF0500260BF1010BBBF1F5
:108F4000100F7FF4D9AE00E0079D079A551BE8B2D9
:108F50000FB0BDE8F08F00BF494500084916000872
:108F6000737B0108453801085C330020753801081F
:108F7000012908B5104605D113785AB2632A0ADCD4
:108F8000013307E002290BD113785AB212F1630FB3
:108F900001DB013B03700121074B9847002008BD0E
:108FA0000339C9B2012904D80121034B9847012094
:108FB00008BD002008BD00BFA94F00082DE9F043FF
:108FC000484B074693F84950474B89B01E780846EE
:108FD000FF2E90461C4664D1444E03213246444C39
:108FE000A0473378434C0093384621460DF11F02C9
:108FF0000323414FB847B14624784DE0022C45D8B1
:1090000099F8001028460B1B594241EB03013B4BDA
:109010009847012C354E0AD0022C1DD031782846B5
:10902000D1F1010138BF0021354B98472EE0354979
:10903000354B03A89847354B03A89847002203AB4C
:1090400098F90010181800941346314FB847327839
:10905000284603A9012A14E02E492B4B03A8984760
:109060002A4B03A8984701230022009303AB98F9E9
:1090700001101818264F1346B8473278284603A91E
:10908000022A14BF00220122234B9847234B0134AC
:109090001B78E4B2ED18EDB29DF81F30A342ADD8B5
:1090A0001CE0012E09D002D3022E17D108E01C4A81
:1090B00001201070FF221A7011E01A4B586802E06C
:1090C000184B01329868FF23174DA847012805D196
:1090D000134B1870FF232370013800E0002009B003
:1090E000BDE8F0831433002094000020A704002082
:1090F000915F0008AE040020816D0008195E000831
:109100007D5F000801810108911600084D170008D5
:10911000494500087A7B0108DD5C00085C330020CB
:109120009200002000010020718F00082DE9F04F0F
:10913000844B8DB093F84970834B834693F800803D
:109140000E46B8F1FF0F14461D4668D1DFF82C8299
:109150000846424611217D4EB047DFF8249298F828
:1091600000307B4E00938246494658460DF12F024F
:109170001123B04799F8006033E098F800103846A2
:109180008B1B594241EB0301724B984798F8002022
:109190003EB9D2F10101384638BF00216E4B9847E5
:1091A00019E0082E09D8C6EB020CDCF100023846A3
:1091B000314642EB0C02694B0CE0694BC6EB020EE8
:1091C000A6F1090153F82110DEF10002654B384683
:1091D00042EB0E029847644B01361B78F6B2FF183B
:1091E000FFB29DF82F30B342C7D8604B98F80060AB
:1091F00098475F4B07469847013E1C231D3F0A389E
:10920000F6B20093FFB2133BC0B201930390314614
:10921000029720460122093B564EB04764E1B8F15F
:10922000000F05D1544A01201070FF221A707EE110
:10923000B8F1090F0ED100231A46072192FBF1F174
:109240006439C832E018E1540433B2F5C86F417094
:10925000F3D14CE1B8F10A0F0ED100236422E118DA
:10926000E2540433202B4A70F8D17C3323706370AE
:109270009C3B237163713AE1B8F10B0F1BD10022C3
:109280006423A118A3540432202A4B70F8D17C32F5
:1092900022706270627133322272CF3ACE216272D2
:1092A000312062733232227421712073637423750A
:1092B0006375313A1CE1B8F10C0F0BD10023E218B1
:1092C00092F90110043301EBD1714910202B517038
:1092D000F5D10CE1B8F10D0F08D10023E218517857
:1092E00004334942202B5170F8D100E1B8F10E0F40
:1092F00012D10023E21851780139517049B211F1AD
:10930000640F01DA9C2102E0642901DD64215170BF
:109310000433202BEED1EAE0B8F10F0F32D1002355
:10932000E21851780131517049B211F1640F01DA3C
:109330009C2102E0642901DD642151700433202B5B
:10934000EED1D4E014330020C0000020915F00086B
:10935000816D0008195E00087D5F0008B95C000897
:10936000C4000020DD5C00085C330020673B01087E
:109370006B3B01081970000892000020A90400202E
:109380009F040020B8F1100F6A4FDFF8C091DFF89A
:10939000C0A16ED1DFF8A881FF23674E674842461F
:1093A000B04798F80030099046460BB90133337046
:1093B0003378402B02D9624B40221A7095F800C0D6
:1093C00096F800B00CF1FF3C5FFA8CFCDFF884816A
:1093D0003423CDF814C00BF1FF3B03FB0B8BB847D4
:1093E0000690C8470790B8470890B8470746C8474F
:1093F000069A079BD208D2B200920522B3FBF2F381
:10940000089903EB4303DBB2013901938308A1EB15
:109410009707013BDDF814C00BF5A65BDBB20BF13F
:10942000080BFFB20393043A0023029758466146A3
:10943000D047099B012B5FD10022134630780D21C4
:10944000013801FB003000F5A66008EB8000007ACF
:10945000A0543078013801FB003101F5A66108EB1A
:109460008101487A0133A1180432082B4870E5D1F4
:109470003DE0B8470746C8471D3F1C230A38009304
:10948000FFB2133BC0B208F1FF31012201930297F2
:10949000093B0390C9B22046D0472B785846013B80
:1094A00004EB83023146DBB2264FB847012E8246D9
:1094B0000DD1234604F11C011A7893F9046050B2CF
:1094C0008642B8BF1A7104338B42F5D10CE0022EEC
:1094D0000AD10023E2181279E05651B28842C8BF7F
:1094E000E25404331C2BF5D1BAF1010F04D101224F
:1094F000154B1A70FF232B700023E25612F1640FF4
:1095000001DA9C2202E0642A01DD6422E254E218BE
:1095100092F9011011F1640F01DA9C2102E0642933
:1095200001DD642151700433202BE6D100200DB001
:10953000BDE8F08F673B0108416600087D7B0108AC
:10954000A0040020BD8F0008920000206B3B0108A2
:1095500019700008940E00202DE9F04FDFF8848187
:10956000504B98F8005085B0FF2D8346144693F871
:1095700049606BD1DFF8409108464A464321434693
:10958000494FB847DFF860A199F800300DF10F029C
:109590000093464F432358465146B847444B4F46E5
:1095A0001A78FF2A05D01B780126237088F800500E
:1095B00073E09AF8004043E0397830460B1B59427B
:1095C00041EB03013B4B3C4D98473CB92A78304670
:1095D000D2F10102394938BF00220FE0012C04D139
:1095E0002A7830463649012A05E0022C08D12A782B
:1095F00034493046022A14BF00220122324B18E0BF
:10960000422C17D82A783046C4EB020CDCF1000259
:1096100042EB0C022D492C4B98472A782C4B6101C8
:10962000C4EB020EC918DEF100022A4B304642EBB1
:109630000E029847284B01341B78E4B2F618F6B2B4
:109640009DF80F30A342B7D8002626E0234A244BCA
:1096500035B9FF2101262170167088F8001019E035
:10966000012D0AD1FE2121701570FF2288F80020FB
:109670002046294698472E460FE0022D4FF001065E
:1096800002D1FD21217001E0033D25701670FF22FB
:1096900088F80020204631469847304605B0BDE89E
:1096A000F08F00BF14330020915F0008656B000845
:1096B000F1010020A95E00087E0400208D7B0108D6
:1096C0009C7B0108AC7B0108015A0008B87B0108AB
:1096D000600E0020415A00085C33002092000020F8
:1096E000A94F000891000020A8040020F0B5354BD8
:1096F000074693F84940344B10461A7885B0FF2A44
:109700004DD1324D08462A464121314EB0472B7883
:10971000304E0093384631460DF10F0241232E4F53
:10972000B847367835E0297820468B1B594241EB03
:1097300003012A4B254F984746B93A782046D2F183
:109740000102274938BF0022264B1BE0402E1AD8C1
:109750003A782046C6EB020CDCF1000242EB0C0228
:109760002149204B9847214B721E182101FB0231E1
:109770003A780431C6EB020EDEF100021C4B2046A3
:1097800042EB0E0298471B4B01361B78F6B2E418E9
:10979000E4B29DF80F30B342C5D800200FE016495F
:1097A0000124164D1AB9FF3202700C7003E0013A21
:1097B00002700C70FF221A702146A847204605B09F
:1097C000F0BD00BF1433002090000020A104002051
:1097D000915F000866040020656B0008A95E000820
:1097E000BE7B0108015A0008C37B0108BC1600209B
:1097F000415A00085C33002092000020A94F000865
:109800002DE9F04F13788BB0FD2B804615460BD019
:1098100003F1020B5FFA8BFBBBF1010F94BF4FF01A
:10982000020B4FF0040B01E04FF0030B8F4EDFF8FB
:10983000B09296F801A099F84940BAF1FF0F40F0B4
:10984000E180084632465946731C894FB847337841
:10985000884940460DF127020093874F5B46DFF8A9
:109860008482B847C047854A079099F84870904766
:109870000590C04707990346C91B01270097013F80
:109880000197029703973846C9B2059ADFF8F0C1ED
:10989000E04799F84A30002B3ED0C04799F84A304B
:1098A00076490693059088470790C047069BDDF8E8
:1098B0001CC0059ADB43D1180CF1FF32431E012076
:1098C000C9B2D2B200900197384602970397DBB233
:1098D0006B4FB8476B4F337857F823006A4B984764
:1098E0000590C047694B99F84A101B7899F84AE0EF
:1098F000059AC3EB0E0303EBD373C1EB630133781B
:109900004118CDF800A0CDF804A01046C9B257F810
:10991000232053465E4FB847564B1F786DE0317891
:109920002046CB1B594241EB03015A4B98475F45F8
:109930005DD22B785849FD2B584B0DD1022F0BD1FE
:109940004A4A204612780969A2F1020CDCF10002B1
:1099500042EB0C02984734E032782046C7EB020E07
:10996000DEF1000242EB0E0251F827109847022F59
:1099700027D03E4B032F1A7829D0012F484B2FD1E7
:1099800095F800E0BEF1FF0F02D1204645490AE0FC
:10999000BEF1FE0F02D12046434904E0BEF1FD0FA7
:1099A00003D142492046012A1DE0BEF13F0F05D8F0
:1099B0003F494FEA4E1E20467144F4E720463D4998
:1099C000F1E73278204695F90110022A03E095F973
:1099D00002102046032A14BF00220122364B05E064
:1099E00036492046BA4214BF002201229847344B20
:1099F00001371B78FFB2E418E4B29DF82730BB4270
:109A00008DD87EE0BAF1030F7BD8DFE80AF0020DB3
:109A1000246D2C4B01241C70FF23737028460421F5
:109A2000294B984720466DE01B4B284C58682A4626
:109A3000FF23A047264F04463B78FF2B5BD0254BE6
:109A400098473878244B9847002801DD642300E0CC
:109A50009C236B704FE0FD2B0F4B05F101020CBFF7
:109A6000186998681D4CFF2343E000BF680100207F
:109A7000915F000896040020656B0008673B0108B1
:109A8000053401080C010020795000082001002055
:109A9000BD380108A95E000800000020015A000836
:109AA000415A00088D7B01089C7B0108AC7B0108B2
:109AB000C00E0020CA7B0108795C0008DD7E010829
:109AC0005C33002092000020A94F0008599500083F
:109AD000F1010020DD460108A14A01080D670008D8
:109AE000143300206B3B0108084B094CD868AA1CB2
:109AF000FF23A0470446012C03D1064B1C70FF2313
:109B0000737000200BB0BDE8F08F00BF0000002094
:109B10000D670008920000202DE9F04F137893B0F4
:109B2000FD2B8046154601D10233137095F800B025
:109B3000974C0BF1020B94F805A05FFA8BFBDFF852
:109B4000D092BBF1010F94BF4FF0020B4FF0050B09
:109B5000BAF1FF0F99F8496040F0F5800846221DE0
:109B60005946631D8B4FB84723798B4940460DF109
:109B700047020093894F5B46DFF89882B847C04799
:109B8000874A079099F8487090470590C047079911
:109B90000346C91B01270097013F019702970397CE
:109BA0003846C9B2059ADFF8FCC1E04799F84A3057
:109BB000002B3ED0C04799F84A307949069305906A
:109BC00088470790C047069BDDF81CC0059ADB4319
:109BD000D1180CF1FF32431E0120C9B2D2B200905D
:109BE0000197384602970397DBB26E4FB8476E4F26
:109BF000237957F823006D4B98470590C0476C4B6D
:109C000099F84A101B7899F84AE0059AC3EB0E03BD
:109C100003EBD373C1EB630123794118CDF800A0A6
:109C2000CDF804A01046C9B257F823205346614F1F
:109C3000B847594B1F7880E021793046C7EB010CBB
:109C4000DCF1000141EB0C015B4B98475F456ED2A4
:109C50004F4B30461A79594BC7EB020EDEF100022A
:109C600053F8271042EB0E02554B98477B1E032BEF
:109C700052D8DFE803F002353B452978DFF87481DC
:109C8000FF2903D1227930464E4922E0FE2903D133
:109C9000227930464C491CE0A1F14003DBB2BD2BD8
:109CA00014D94A4B4901C91809A8494B9847494B4F
:109CB00028469847484B10B109A8484901E048494F
:109CC00009A898472279304609A902E02279454936
:109CD0003046A2F101035A4242EB0302C04726E09C
:109CE0002279304695F90110022A04E0227995F98B
:109CF00002103046032A14BF002201223A4B15E01D
:109D000022793046A2F1040CDCF1000295F903102F
:109D100042EB0C02354B09E022793549C7EB020EC4
:109D2000DEF10002334B304642EB0E029847324BD5
:109D300001371B78FFB2F618F6B29DF84730BB42E8
:109D40003FF67AAF7EE0BAF1040F7BD8DFE80AF085
:109D5000030E64676D00294B01261E70FF2363719B
:109D600028460421264B984730466CE0134B254E7D
:109D700058682A46FF23B047234B06461B78FF2B23
:109D80005AD0224B984764236B70503BAB7053E022
:109D900068010020915F0008AC040020656B00089A
:109DA000673B0108053401087C0000207950000859
:109DB00020010020BD380108A95E0008E80000204D
:109DC000015A00081E7B0108157B0108C00E002007
:109DD000911600087D3E000849160008087B01081E
:109DE0000E7B0108CA7B0108795C0008A95A0008AB
:109DF000DD7E0108415A00085C33002092000020FB
:109E0000A94F000859950008F1010020DD4601081E
:109E1000143300206B3B01080C486A1C02E00C4B19
:109E2000AA1CD868FF230B4D04E0094BEA1C0A4D1D
:109E30001869FF23A8470646012E03D1074B1E7061
:109E4000FF236371002013B0BDE8F08FF000002005
:109E5000E80000200D670008F15000089200002083
:109E60002DE9F04F874D8FB0874E8046B0472B7855
:109E7000FF2B40F08281A0F10B07F53B97FBF3F736
:109E8000FFB28248824B98474FEA470A814C4021F3
:109E900091FBFAF122462B46013140467E4DDFF818
:109EA0000882A847C0470C3800EBD070401080B241
:109EB0000690B0472478A0F10A05C047640095FBDE
:109EC000F7F57C430746B0470121431E7A1E002068
:109ED00000910190029003900831D2B2DBB26F4E34
:109EE000B04706990698C9B2E4B2400801F10803E8
:109EF0005FFA80F9DBB204F1010B544409F1040864
:109F0000EAB20134994409350D9409905FFA88F852
:109F10000A9107935FFA89F90B92EDB20B2421E1C4
:109F2000059E5F4A7301D31838339B796FF0630144
:109F30005BB28B42B8BF0B46069F642BA8BF64235D
:109F400003FB07F0C921DDF824C090FBF1F1614467
:109F500089B2002B0C914FF0010301F104020DDDD9
:109F60000093FE330193643B0293963B0393404678
:109F70002146D2B22B46494EB0470BE00093FF2357
:109F80000193FA3B02930393D0B2214642462B46FB
:109F9000424FB84704F1020AFF269B275FFA8AFA6C
:109FA0004046214642465346DFF800C100960197DD
:109FB0000297E047AB1EDBB2194608934046424683
:109FC0002B46DFF8E8C0009601970297E0470C990E
:109FD000DFF8D8C0081DC0B202465146089B009663
:109FE00001970297E04705982D4942018A182C32C3
:109FF000104604922B4B9847A8EB50005146049A08
:10A000003346DFF8ACC000960196C0B2E0470A982C
:10A010000023021D009304202146D2B22B46DFF814
:10A020007CC0019602960396E0471D484FEA4B1309
:10A03000C31838339B796FF063025BB29342B8BFA9
:10A040001346069A642BA8BF642303FB02F1DDF8D4
:10A0500024C0C92291FBF2F26244079892B2002B0D
:10A0600005924FF00103024424DD0093043301966E
:10A070000393029748462146D2B22B46074EB0477B
:10A0800023E000BF450000206B3B0108D17B0108A5
:10A0900039610008B2040020915F0008B53501085D
:10A0A000940E002045380108673B01080937010874
:10A0B000753801080093052302930393D0B20196EB
:10A0C00021464A462B46324FB847FF269B2721465A
:10A0D00000960197029748464A465346DFF8B4C0B7
:10A0E000E0472B46DFF8ACC0009601970297484640
:10A0F00008994A46E0470799059A089B8818C0B214
:10A1000002460096019702975146224FB847DFF862
:10A1100094C04FEA4B1767442C3738461E4988478E
:10A12000A9EB50003A4633460096019651461B4F24
:10A13000C0B2B847DDF828C000234FEA4C0208320D
:10A14000009301960296039621462B46079802F04B
:10A15000FE020F4EB0470B9F0BF1020BE419ED19F5
:10A16000E4B2EDB2DDF834C0E3450CD00BF1FF30C2
:10A170003F2805907FF7D4AE05E0094B0120187009
:10A18000FF232B7000E000200FB0BDE8F08F00BF70
:10A19000B535010809370108453801087538010847
:10A1A00092000020940E00202DE9F04F8D4D91B0CB
:10A1B0008D4E8046B0472B78FF2B40F09081A0F168
:10A1C0000B07F53B97FBF3F7FFB28848884B98479E
:10A1D0004FEA470A874C402191FBFAF122462B4671
:10A1E00001314046844DDFF81C82A847C0470C3837
:10A1F00000EBD070401080B20890B0472478A0F1F6
:10A200000A05C047640095FBF7F57C430746B04755
:10A210000121431E7A1E00200091019002900390BC
:10A220000831D2B2DBB2754EB04708990898C9B26E
:10A23000E4B2400801F108035FFA80F9DBB204F1EF
:10A24000010B544409F10408EAB201349944093578
:10A250000F940B905FFA88F80C9109935FFA89F9D3
:10A260000D92EDB20B242FE1654A079E182303FBE4
:10A27000062303F5026318339B8814211BB293FB5A
:10A28000F1F378398B42B8BF0B46089F642BA8BF07
:10A29000642303FB07F0C921DDF82CC090FBF1F12A
:10A2A000614489B2002B0E914FF0010301F10402C9
:10A2B0000DDD0093FE330193643B0293963B0393C1
:10A2C00040462146D2B22B464C4EB0470BE000939D
:10A2D000FF230193FA3B02930393D0B221464246F7
:10A2E0002B46464FB84704F1020AFF269B275FFA28
:10A2F0008AFA4046214642465346DFF80CC1009692
:10A3000001970297E047AB1EDBB219460A9340461D
:10A3100042462B46DFF8F0C0009601970297E047CF
:10A320000E990A9B081DC0B202465146DFF8D8C0FC
:10A33000009601970297E0470798314B182101FBDF
:10A34000003202F502620C3210460692DFF8BCC001
:10A35000E047A8EB50005146069A3346DFF8B0C0FC
:10A3600000960196C0B2E0470C980023021D0093AE
:10A3700004202146D2B22B46DFF880C00196029617
:10A380000396E0471E49182000FB0B1C0CF50263E6
:10A390001B189B8814221BB293FBF2F3783A93426A
:10A3A000B8BF1346089A642BA8BF642303FB02F1CD
:10A3B000DDF82CC0C92291FBF2F26244099892B2F6
:10A3C000002B07924FF00103024423DD0093043376
:10A3D00001960393029748462146D2B22B46074E78
:10A3E000B04722E0600000206B3B0108E07B0108E1
:10A3F000396100087D040020915F0008B53501082F
:10A40000940E0020673B0108093701084538010810
:10A41000753801080093052302930393D0B2019687
:10A4200021464A462B46334FB847FF269B272146F5
:10A4300000960197029748464A465346DFF8B8C04F
:10A44000E0472B46DFF8B0C00096019702974846D8
:10A450000A994A46E0470999079A0A9B8818C0B2A8
:10A4600002460096019702975146234FB847DFF8FE
:10A4700098C0182707FB0BC707F502670C3738464B
:10A480001E498847A9EB50003A463346009601968C
:10A4900051461B4FC0B2B847DDF830C000234FEA29
:10A4A0004C020832009301960296039621462B46F1
:10A4B000099802F0FE020F4EB0470D9F0BF1020B00
:10A4C000E419ED19E4B2EDB2DDF83CC0E3450CD07F
:10A4D0000BF1FF303F2807907FF7C6AE05E0094B30
:10A4E00001201870FF232B7000E0002011B0BDE8A0
:10A4F000F08F00BFB535010809370108453801085C
:10A500007538010892000020940E00202DE9F043D8
:10A5100093B00024724E734B804604A89847724F44
:10A52000724B73488DF83040984796F84950B847B9
:10A530008146B84796F84A106FF001035B1A02355E
:10A54000A9F10402C3180121EDB200910194029413
:10A55000039402202946D2B2DBB2664FB847B14617
:10A5600001E00134E4B212A90B1913F8383C202B96
:10A57000F7D004AA11190DA810225F4FB847002385
:10A580008DF844300F3306E012A9CA180021013BB0
:10A5900002F8141CDBB212A9CA1812F8142C202AD3
:10A5A00000D00AB9002BEFD10DA8544EB047FF23BD
:10A5B00005F10E01C9B2009301930DAA504CA047BA
:10A5C000102101E00131C9B212AA531813F8383C26
:10A5D000202BF7D004AB59180DA81022B847002340
:10A5E0008DF844300F3306E012A9CA180021013B50
:10A5F00002F8141CDBB212A9CA1812F8142C202A73
:10A6000000D00AB9002BEFD10DA8B047FF2305F108
:10A61000170100930193C9B20DAAA047B8F1010F29
:10A62000384D06D12B78042B01D8013307E00023E5
:10A6300005E0B8F1020F06D12B7813B1013B2B7066
:10A6400017E00523FBE7B8F1030F12D12B78052B98
:10A650000FD8DFE803F040030507090B702006E080
:10A66000E02004E0B02002E0D02000E0F020264B03
:10A6700098470DA82549264FB8472A78052A16D8A5
:10A68000DFE802F00306090C0F120DA821490DE0C6
:10A690000DA821490AE00DA8204907E00DA820498E
:10A6A00004E00DA81F4901E01F490DA8B8470DA8F7
:10A6B000B0471E4B0546984799F84A306FF00B019A
:10A6C000C91A4118FF23009301932846C9B20DAA65
:10A6D000A047002000E0012013B0BDE8F08300BFD8
:10A6E00014330020F93B0108673B01083961000879
:10A6F000F07B01080534010859180008795000085A
:10A70000BD3801088C040020193C0108FD7B0108BC
:10A7100091160008017C0108087C01080F7C0108E3
:10A72000177C01081E7C0108237C01086B3B010893
:10A730002DE9F04FB14C93B094F808A0637AA4F5DA
:10A7400012500693AE4BA67A9847AE4B984701231A
:10A750008DF84130DB188DF8423001338DF84330ED
:10A7600001338DF84430013306988DF845300133BC
:10A7700000278DF84630013384F808A08DF840702A
:10A7800060728DF84730A6729F4D780128182C30E2
:10A790009E499F4C0137A047402FF5D1403F1820DC
:10A7A00000FB075000F502600C3098490137A047C4
:10A7B000402FF4D10022342303FB0253FF2003F582
:10A7C000A45383F83400FD2183F840004FF064085F
:10A7D0000138013283F8418083F8380083F83C1057
:10A7E000FD39402A83F83D80874F83F83E10E2D13F
:10A7F00007F5B6708749A04707F5C6708649A04798
:10A8000007F5D6708549A04707F5E6708449A0474B
:10A81000CE2232234FF00A0E0B200C2187F84A205B
:10A8200087F8493087F848E087F86A2087F8693068
:10A8300087F8680087F88A2087F8893087F88810B9
:10A8400087F8AA2087F8A930253B87F8A830323A44
:10A8500007F5105787F8558087F8578087F8598093
:10A8600087F85B2087F854E01A4687F8560087F887
:10A87000581087F85A306B4B102E00F25387DFE8E0
:10A8800016F0110011001100110011001100020357
:10A890000203020351075107D505D5055107950657
:10A8A0005C0695060022711E85F8282010460132AC
:10A8B000042908D8DFE801F007030303060085F840
:10A8C000280002E0022285F82820574853F8261075
:10A8D000A047BAF1020F15D0BAF1030F1BD0BAF19D
:10A8E000000F4FF003000CBF0221012108900CBFA4
:10A8F0004FF001094FF0020907910CBFD3464FF00A
:10A90000000B0FE0002208924FF00109CDF81CA0C7
:10A910004FF0030B06E00023012708934FF00209D4
:10A920000797D3464FEA4B10281840492C30A047D0
:10A93000DDF81CA03E494FEA4A1028182C30A047E9
:10A940004FEA491028183B492C30A047DDF820C0B9
:10A9500039494FEA4C1028182C30A047374938485D
:10A96000A0479DF8420037494001281800F5B6700D
:10A97000A04735493548A04735493648A0473649AC
:10A980003648A04736493748A04737483749A04797
:10A9900006980022012303287AD8DFE800F0020E8F
:10A9A00020698DF8413002238DF8423001338DF853
:10A9B00043308DF8402001331CE08DF840300223F5
:10A9C0008DF84130023B8DF8423003338DF843302F
:10A9D00001338DF8443003338DF8453058E08DF85D
:10A9E000413003238DF84230013B8DF843308DF820
:10A9F000402002338DF844300133EDE7143300205A
:10AA00001D3C000805400008940E0020CA7B010888
:10AA100091160008E2760108E9760108F07601084F
:10AA2000F776010824010020AC0E0020307C0108DC
:10AA3000357C0108517601083A7C0108407C010808
:10AA4000400F0020487C01082C7B0108C01000202A
:10AA5000317B010820110020517C010800110020E9
:10AA6000547C010880100020A01000205B7C0108AD
:10AA70008DF8443002238DF8413001338DF8453094
:10AA800001338DF8433001338DF840208DF842308A
:10AA90009DF840204FF0180A0AFB02F3E81800F571
:10AAA0000260039306920C307949A0479DF841C09B
:10AAB0007849CDF828C00AFB0CFC05EB0C0000F52A
:10AAC0000260CDF810C00C30A0479DF8428072495A
:10AAD0000AFB085000F502600C30A0479DF84300C7
:10AAE0006E490C900AFB005000F502600C30A04744
:10AAF0009DF844106A4F0AFB01F2A81800F50260A5
:10AB0000059209910C306749A0479DF845000AFB62
:10AB100000F10B90681800F502600F910C3062494B
:10AB2000A0479DF8460061490D900AFB005000F5D2
:10AB300002600C30A0479DF847100AFB015000F559
:10AB400002600E910C305A49A04707F50E600C3098
:10AB50005849A047039BCE20EB1803F5026332212E
:10AB600053440A24987259721C72059AAA1802F565
:10AB700002625244917250721472DDF810C00B22BE
:10AB8000AC440CF502635344987259721A720F9BCD
:10AB90004FF0FE0CED1805F502655544A87207F557
:10ABA000A45069722A7280F834B0069C07F5A65248
:10ABB000642314705370099DAAF17C0ACB319570FF
:10ABC00082F803A080F838C080F83C1080F83EA0DE
:10ABD00080F83D30079D544682F82850DDF828A0C3
:10ABE000012E82F834A082F835300B9882F83600B6
:10ABF00082F8373082F82CC082F8301082F8324068
:10AC000082F83130089D07F5A8521577DDF830A09D
:10AC100007F5A95082F828A082F8293009F1020A24
:10AC200080F800C082F8241007F5AC5082F8264066
:10AC300082F8253007F5AA5407F5AE523CD84FEA02
:10AC40004A1A574401250426BD7126740D9F6FF0E2
:10AC5000630A2777637784F814C0217684F81AA0F2
:10AC6000637680F8049080F81080437480F808C000
:10AC7000017380F83860069C14715371099D9571B9
:10AC8000D37180F83CC01170FD3991705370BEE0F3
:10AC9000617C0108687C0108517601083A7C010852
:10ACA000940E00206F7C0108767C0108407C01082E
:10ACB000547C01085B7C01084FEA4A1A07EB0A053D
:10ACC0004FF0010A85F806A00C954FF00E0A6FF0C0
:10ACD000630584F8109084F81C80637784F814C0AE
:10ACE0002176A576637680F804A00E9C047408246F
:10ACF000437480F808C001738573437380F83890FB
:10AD000014710734537180F83C4011709570537082
:10AD10000C9CFF20207207F5065484F8348084F8D8
:10AD200038C008F10A0CFF38E14607F5075C84F8E3
:10AD30003C1084F83E0084F83D308CF800904FF0D1
:10AD40004B0C84F842304FF0EC0984F841C007F511
:10AD50000A5484F8348084F838A084F8399084F850
:10AD60003A5084F83C1084F83E0084F83D5007F5D2
:10AD70000B552970142584F8420084F8413084F87A
:10AD8000448084F848A084F84950A635042E84F8FD
:10AD90004A9084F84C1084F84E0084F84D5084F8A2
:10ADA000501084F8520084F8513030D1122482F8C7
:10ADB000304082F82CB00A9E053D82F8386082F857
:10ADC00039C0DDF82C9082F83A9082F83B5082F836
:10ADD000341082F8360082F8353007F5B05282F828
:10ADE0002440DDF81CA007F5B15787F800A0069CA9
:10ADF00082F82C4082F82DC0099D82F82E5082F8EE
:10AE00002FC082F8281082F82A0082F829307D4A63
:10AE1000FD2100242D20102582F834B082F838500E
:10AE200082F83C1082F83E4082F83D00079E1346AF
:10AE300003F8406F1D7119729C725872089F1F733E
:10AE40001D7419759C7558751334053082F8F4B06B
:10AE500082F8F84082F8FC1082F8FE00193082F87F
:10AE6000FD0002F5807382F8006182F8044182F8E7
:10AE7000081114229A7258721F731C7419759A75EE
:10AE8000587500F088BC042285F828205E4853F8E5
:10AE90002610A047BAF1020F16D0BAF1030F1DD049
:10AEA000BAF1000F4FF00309CDF81C900CBF4FF022
:10AEB00001084FF002080CBF4FF002094FF00109E2
:10AEC00018BF4FF0000A0FE04FF0000CD146CDF84C
:10AED0001CC04FF001084FF0030A05E00020079066
:10AEE0004FF002084FF001094FEA4A1028182C30A1
:10AEF0004649A0474FEA491028182C304449A0473A
:10AF00004FEA481028182C304249A04707990027DB
:10AF1000480128182C304049A04740494048A047E4
:10AF200040494148A04741494148A047414942481A
:10AF3000A04742494248A04742494348A0470AF136
:10AF400002035B01EB18187A4049400128182C30A5
:10AF5000A04709F102035B01EB18187A3C49400154
:10AF600028182C30A04708F102035B01EB18187A6F
:10AF70003849400128182C30A047079A3649931CBD
:10AF80005B01EB18187A400128182C30A04785F88F
:10AF9000E070324985F8DE703148A04785F80071CD
:10AFA000304985F8FE703048A04785F820712F4958
:10AFB00085F81E712E48A04785F840712D4885F808
:10AFC0003E712D49A047069A0523032A64D8DFE87D
:10AFD00002F055020C5501228DF8413002238DF804
:10AFE00042308DF840209B1808E08DF84030012356
:10AFF0008DF84130DB188DF8423001338DF8433045
:10B00000033B47E054200020AC0E00207D7C01086B
:10B01000827C0108877C01083A7C01082C7B0108AE
:10B02000C0100020317B0108A0100020517C0108D5
:10B0300000110020547C0108801000208D7C010844
:10B0400020110020927C0108400F00209D7C010807
:10B05000A77C0108B17C0108BC7C0108C87C010800
:10B06000600F0020D77C0108800F0020E67C0108DB
:10B07000A00F0020C00F0020F17C010801238DF8F3
:10B080004130DB188DF8423001338DF843308DF8B4
:10B09000407001338DF844309DF840304FF0180B6C
:10B0A0000BFB035C0CF5026C0CF10C0C604603937B
:10B0B000CDF810C0D149A0479DF84120D04F0BFBDF
:10B0C00002F0291801F502610C31059209900891EE
:10B0D0000846CC49A0479DF842100BFB01F00A90AE
:10B0E000281800F5026006910C30C749A0479DF86A
:10B0F0004300C6490BFB00F00B90281800F50260D6
:10B100000C30A0479DF844100BFB01FB05EB0B0036
:10B1100000F502600C30BE49A04707F50A60043014
:10B12000BC49A047062E07F5A65407F5A45607F517
:10B13000A855059A039BDDF810C05ED108F1020006
:10B140004001012138188171DDF828C007EB0C009F
:10B1500080F83E18DDF824C007EB0C0080F83E189C
:10B16000DDF82CC007EB0C005F4480F83E1887F830
:10B170003E18563186F834A0237061705231A270A7
:10B180004FF0FE0CE170FD274539002086F838C0ED
:10B1900086F83C7086F83E0086F83D10CE2684F88E
:10B1A000289084F8343084F8356084F8362084F8A8
:10B1B0003760069E84F8386084F8391084F82CC013
:10B1C00084F8307084F8320084F8311085F81C80DF
:10B1D00085F8283085F8291085F82A2085F82B1065
:10B1E00085F82C6085F82D1084F860C085F82470EF
:10B1F00085F8260085F8251038E06046059203930F
:10B20000854F8649B84786490898B84786F834A0DC
:10B21000039BFE272370FD2064230021637086F8C2
:10B22000387086F83C0086F83E1086F83D3084F889
:10B230002890DDF818C084F834C084F8353084F8DC
:10B240002C7084F8300084F8321084F8313085F89E
:10B250001C80059A85F82820724A85F829301770D5
:10B2600085F8240085F8261085F825306E4A64217B
:10B2700082F810809DF843C0FE26082382F81CC087
:10B28000517716751376DA339376C43B537682F88A
:10B2900044809DF84470FD20002582F8507082F8AB
:10B2A000511082F8486082F84C0082F84E5082F8C3
:10B2B0004D10DDF81C90042402F5546382F8789058
:10B2C00082F884C082F885104FF0130C82F87C60FD
:10B2D00082F8800082F8825082F8811082F8AC40B7
:10B2E000013482F8B84082F8B91082F8B06082F870
:10B2F000B40082F8B65082F8B51083F8347083F841
:10B3000038C0ACF10C0C83F83CC00CF1210C83F874
:10B310003EC00CF1B00C83F83DC04FF00E084FF06A
:10B32000140C82F8800D83F8425083F8411083F8A2
:10B33000447083F8488083F849C00CF1D80C83F836
:10B340004AC083F84C40013483F84E5083F84D10C6
:10B3500083F85040963483F8525083F8514083F874
:10B36000547083F8588083F859C083F85A4083F8A2
:10B370005C0083F85E5083F85D1083F8600083F80A
:10B38000625083F861409DF8401002F5446383F8F1
:10B390003410322183F8386083F83C0083F83E1083
:10B3A00083F83D1082F8800C83F8421083F8411036
:10B3B0009DF8412083F8442083F8486083F84C00CE
:10B3C00083F84E1083F84D1083F8500083F8521024
:10B3D00083F851109DF8422083F8542083F8586078
:10B3E00083F85C0083F85E1083F85D1083F86000DA
:10B3F00083F8621083F86110CDE100BFFF7C010883
:10B40000940E0020067D0108827C01083A7C010828
:10B4100051760108927C0108911600087D7C010894
:10B42000877C0108B4230020D423002053F8261081
:10B4300085F82820A748A047A749A848A047A849B9
:10B44000A848A047A849A948A047A949A948A04792
:10B45000A949AA48A0479DF84090182606FB095024
:10B4600000F50260A6490C30A0479DF84180A5492F
:10B4700006FB085000F502600C30A0479DF84270B2
:10B48000A14906FB075000F502600C30A0479DF86B
:10B4900043A09E4906FB0A5505F502600C30A04703
:10B4A0009B49012381F834300B4603F8408F642216
:10B4B000FD249C20FE25183E5A709F70DA7083F898
:10B4C00004A05A7181F8385081F83C4081F83E6000
:10B4D00081F83D2083F8286083F8349083F8352084
:10B4E00083F82C5083F8304083F8320083F8312001
:10B4F00081F89C60032381F8A88081F8A92081F855
:10B50000AA70122781F8AB0081F8A07081F8A440DE
:10B5100081F8A60081F8A52081F8D0309DF844304C
:10B5200081F8DC3081F8DD2081F8D45081F8D840F2
:10B5300081F8DA0081F8D9202DE1132285F828203E
:10B54000D96B6448A047002101200A463E2926DC29
:10B55000342606FB0256642406F5A45300F1010CC0
:10B5600006F5A65683F8342083F8401083F841404E
:10B5700083F8420083F8434086F804C000F1020CCF
:10B58000747186F806C0F471FE2683F83860013EB7
:10B5900083F83C60FD3E83F83E6083F83D40013215
:10B5A00004300431402AC0B2D0D1F4E0132285F82F
:10B5B0002820484853F82610A04700274FEA47188C
:10B5C00005EB080A0AF12C0A52495046A04750469A
:10B5D000DFF848A1D04740444FF0010C0022791C0D
:10B5E0002818CDF800C02C301346CDF810C009B291
:10B5F000DFF82CB1D847A844002288F84020102E4C
:10B600005FFA87F9DDF810C004D1043288F84120D0
:10B6100088F842C0B9F10F0F21D80C2303FB075360
:10B62000FF2003F58E5282F83490FD2182F8380015
:10B63000FF3882F83C1082F83E002D3082F83D0041
:10B6400003F594533222D13083F8349083F83800D4
:10B6500083F83C1083F83E20921883F83D20013790
:10B66000402FABD10023342202FB035202F5A45237
:10B6700082F83430642182F84030FE26013382F8AB
:10B680004110FD2082F83860FE3E402B82F83C00DD
:10B6900082F83E6082F83D10E5D14FF0180808FBB3
:10B6A00006F805EB080707F502670C371A49384614
:10B6B000A0473846D04740442818012300220136CD
:10B6C00000F5026000930C3031B21346D847402E8B
:10B6D000E3D160E0AC0E00200D7D0108C00E00201B
:10B6E000157D0108E00E00201E7D0108000F0020DE
:10B6F000227D0108200F00202C7D01080011002070
:10B70000357D01083B7D0108427D0108497D010826
:10B7100014230020507D0108597D01084D170008B1
:10B7200049450008052253F8261085F828201C48B2
:10B73000A0471C491C48A0471C491D48A0471D495B
:10B740001D48A0471D481E49A0470D2E05D11023B6
:10B75000FB73093B7B73073BBB730023342202FB63
:10B760000352FE2002F5A452FD2482F8343082F800
:10B77000380082F83C40613C82F83E40383C82F818
:10B780003D4082F84030013302F13001102B82F845
:10B7900041400872E2D1012013B0BDE8F08F00BF34
:10B7A000AC0E00200D7D0108C00E0020157D0108A3
:10B7B000E00E00201E7D0108000F0020200F002059
:10B7C000607D01082DE9F047344F354E7B7886B017
:10B7D000FF2B814696F849403D4652D13A467B1CA4
:10B7E0000846304F1121B847DFF8EC802B784146EE
:10B7F0000DF11702484600932B4F1123B8472B4FEA
:10B80000B8472B4B96F84A90824698470646B84769
:10B81000C9EB0A090346012200200092019032463A
:10B820000290244E03905FFA89F1B04798F80060C7
:10B8300021E0297820468A1B514241EB02011E4B30
:10B840009847102E11D8154B20461A781B4B53F8E9
:10B850002610931B5A4242EB0302194B9847194B8F
:10B8600020469957FF22184B9847184B01361B78F2
:10B87000F6B2E418E4B29DF81730B342D9D80020EC
:10B8800009E013701046124B01219847114B01201B
:10B890001870FF237B7006B0BDE8F087AE00002073
:10B8A00014330020915F0008656B00086B3B0108B2
:10B8B000673B010805340108A95E00082401002047
:10B8C000015A0008F0790108D95A00085C330020B9
:10B8D000A94F0008920000205F0400202DE9F047E6
:10B8E000334F344E7B7886B0FF2B814696F8495013
:10B8F0003C4650D13A467B1C08462F4F0421B8479E
:10B90000DFF8E080237841460DF1170248460093A6
:10B910002A4F0423B8472A4FB8472A4B96F84A9033
:10B92000824698470646B847C9EB0A0903460122F2
:10B9300000200092019032460290234E03905FFA5D
:10B9400089F1B04798F800601FE021782846C6EBDF
:10B95000010CDCF1000141EB0C011C4B9847032E5C
:10B960000DD8134B28461A78194BC6EB020EDEF1A0
:10B97000000253F8261042EB0E02164B9847164B66
:10B9800001361B78F6B2ED18EDB29DF81730B342D0
:10B99000DBD8002009E013701046104B01219847B6
:10B9A0000F4B01201870FF237B7006B0BDE8F087B5
:10B9B0005E00002014330020915F0008656B0008D2
:10B9C0006B3B0108673B010805340108A95E0008CC
:10B9D000B0000020015A00085C330020A94F000885
:10B9E00092000020920400202DE9F047314F324EA2
:10B9F0007B7886B0FF2B814696F849503C464CD167
:10BA00003A467B1C08462D4F0421B847DFF8D88002
:10BA1000237841460DF1170248460093284F04232E
:10BA2000B847284FB847284B96F84A90824698471F
:10BA30000646B847C9EB0A090346012200200092D6
:10BA4000019032460290214E03905FFA89F1B0478F
:10BA500098F800601BE0217828468A1B514241EB90
:10BA600002011B4B9847032E0BD8124B28461A781D
:10BA7000184B53F82610931B5A4242EB0302164B05
:10BA80009847164B01361B78F6B2ED18EDB29DF8CB
:10BA90001730B342DFD8002009E013701046104B76
:10BAA000012198470F4B01201870FF237B7006B0CF
:10BAB000BDE8F087E400002014330020915F000807
:10BAC000656B00086B3B0108673B01080534010802
:10BAD000A95E000814000020015A00085C33002011
:10BAE000A94F000892000020830400202DE9F047B0
:10BAF000334F344E7B7886B0FF2B814696F8495001
:10BB00003C4650D13A467B1C08462F4F0521B8478A
:10BB1000DFF8E080237841460DF117024846009394
:10BB20002A4F0523B8472A4FB8472A4B96F84A9020
:10BB3000824698470646B847C9EB0A0903460122E0
:10BB400000200092019032460290234E03905FFA4B
:10BB500089F1B04798F800601FE021782846C6EBCD
:10BB6000010CDCF1000141EB0C011C4B9847042E49
:10BB70000DD8134B28461A78194BC6EB020EDEF18E
:10BB8000000253F8261042EB0E02164B9847164B54
:10BB900001361B78F6B2ED18EDB29DF81730B342BE
:10BBA000DBD8002009E013701046104B01219847A4
:10BBB0000F4B01201870FF237B7006B0BDE8F087A3
:10BBC0005C00002014330020915F0008656B0008C2
:10BBD0006B3B0108673B010805340108A95E0008BA
:10BBE00098000020015A00085C330020A94F00088B
:10BBF00092000020800400202DE9F04F7E4C7F4F02
:10BC000094F859A089B0BAF1FF0F8046914697F891
:10BC1000495040F0BF80084604F15802052104F164
:10BC20005903774EB04794F8583076490DF11F020A
:10BC300040460093744E0523DFF81C82B047C0478E
:10BC4000DFF818B297F84A600590D8470490C047CB
:10BC500005990346891B0120002600900196029653
:10BC600003963046C9B2049ADFF8A0C1E04797F8BE
:10BC70004A30002B3BD0C04797F84A3004900593D8
:10BC8000D8478346C047059B049ADB43D1180BF184
:10BC9000FF32431E0120C9B2D2B200900196304655
:10BCA00002960396DBB2594EB047594E94F858307D
:10BCB00056F82300574B98478346C047564B97F892
:10BCC0004A201B7897F84A10CDF800A0CB1A03EB56
:10BCD000D373C2EB630194F858304118CDF804A037
:10BCE00056F823205846C9B253464C4EB047454BF0
:10BCF0004F461E7849E094F8581028468A1B514256
:10BD000041EB0201464B9847042E38D83A4B28465F
:10BD100093F85820434B53F82610931B5A4242EB9A
:10BD20000302414B9847731E032B28D8DFE803F02A
:10BD3000020B141D397894F858203C4B284653F8D0
:10BD40002110012A16E0797894F85820384B2846BB
:10BD500053F82110022A0DE0B97894F85820354B99
:10BD6000284653F82110032A04E094F85820324959
:10BD70002846042A14BF00220122304B9847304B3A
:10BD800001361B78F6B2ED18EDB29DF81F30B342C4
:10BD9000B1D82CE0BAF1040F29D8DFE80AF01A0371
:10BDA000081117001F4B274D5868FF2304E01D4B57
:10BDB000254D98680132FF23A847012810D016E0CE
:10BDC000184B0232D868214DFF23F5E70846204B77
:10BDD0009847204B01201870FF2384F8593007E062
:10BDE0001C4B1870FF2384F85930013800E0002004
:10BDF00009B0BDE8F08F00BF6801002014330020B7
:10BE0000915F000860040020656B0008053401089C
:10BE1000480000207950000820010020BD380108AA
:10BE2000A95E000828000020015A0008B000002088
:10BE30001400002024010020DD7E0108415A000882
:10BE40005C330020DDB80008E9B90008C5B7000878
:10BE500031A70008920000206B3B0108673B0108F6
:10BE60002DE9FF41C1EB030E9DF828C01FFA8EFE9D
:10BE70000CFB0EFCDCB26FF063039CFBF3FCCEB258
:10BE8000E6446533C7B2D5B206EB0E0100937F33AB
:10BE900001930293039338462A462346C9B2DFF83A
:10BEA0002080C04700230093FF3301930293039344
:10BEB000384631462A462346C047BDE8FF8100BFC9
:10BEC000B53501082DE9F04F5C4B8BB0884698479B
:10BED0005B4B044698470121A21F831FFF240320C8
:10BEE0000091013902910391D2B20146DBB2554D66
:10BEF0000194A8470520009401940146524A234624
:10BF0000524DA847B8F1010F05D1514B1A78022ABA
:10BF100009D8013206E0B8F1020F04D14C4B1A786F
:10BF20000AB1013A1A704B4A13789146CBB91A46B6
:10BF300002F592614848013100EBC1010020C88040
:10BF40004FF6100088804FF4FE60088143490020BE
:10BF5000C85243490132C8520233042AE8D10123AE
:10BF600069E0012B40F090803E4E3F4F3F48B8477C
:10BF700096F84810FF2405312346C9B23B4A009485
:10BF80000194A8473A48B84796F848102346490014
:10BF90000531C9B2364A00940194A8473548B847DC
:10BFA00096F84830334A03EB4303591D009401943B
:10BFB0002346C9B2A847DFF8CCB0BA46FF3C3746A3
:10BFC0005E4620462C4B98470134E4B2042C26F8F8
:10BFD000020FF6D11E4B214C1B78002234F91310AE
:10BFE0000123009307A81346244EB04707A8D04763
:10BFF00097F84810FF238900053100930193C9B2D7
:10C0000007AAA847B8F1030F40F0E1801C490023BC
:10C0100003F59262104D2088013205EBC202013314
:10C02000D0800022042B24F8022B21F8022FEFD11C
:10C0300099F80030013389F80030C8E0673B010807
:10C040006B3B0108B53501087B860108BD38010846
:10C0500065040020A6040020940E00206C0400203B
:10C06000740400201433002079500008697D010811
:10C07000707D0108777D0108A14A01084945000843
:10C08000720400206A040020022B40F0A080524E6F
:10C09000524F5348B84796F84810FF2405312346BD
:10C0A000C9B24F4A00940194A8474E48B84796F841
:10C0B0004810234649000531C9B24A4A0094019408
:10C0C000A8474948B84796F84830474A03EB430326
:10C0D000591DC9B2234600940194A8474348B84764
:10C0E00096F8481023468900053100940194C9B29E
:10C0F0003E4A3F4FA8473F4C0023B346BA461E4630
:10C1000030463D4B984737F9023B984234F9023BA1
:10C11000B8BF27F8020C9842C8BF24F8020C0136B9
:10C12000F6B2042EECD1354E0127337800223AF9CD
:10C13000131007A81346DFF8D4A00097D0479BF848
:10C1400048104FF0050CC9190CFB01F1FF24CDF884
:10C1500014C00A20C9B207AA234600940194A84734
:10C1600033782448002230F913101346009707A8AB
:10C17000D0479BF84830DDF814C0DB190CFB03FCFA
:10C180006420009401945FFA8CF107AA2346A84723
:10C19000B8F1030F1BD11A481A49002303F5926224
:10C1A000194C013204EBC202D48830F8025F01332B
:10C1B0002C1B9480D48831F8025F042BC4EB050457
:10C1C0001481EBD1043B89F80030012000E000200D
:10C1D0000BB0BDE8F08F00BF143300207950000889
:10C1E000697D0108758F0108777D01087E7D010852
:10C1F0006C04002074040020A14A0108650400209A
:10C200006A04002072040020940E002049450008B2
:10C210002DE9F04F002389B082464FF00108954A7E
:10C22000590151183831097A934619B908F10108B2
:10C230005FFA88F80133402BF1D1B8F1010F00F01B
:10C2400012818D4B8D4F93F8019097F84960B9F1A9
:10C25000FF0F1D4640F0CB801A4641460133884C03
:10C260005046A0472B7887480093874943460DF1F5
:10C270001F02864CA04797F84A30002B36D0DFF8D3
:10C2800058A2D04797F84A208149059204908847E0
:10C290000446D047059A049BD2439918431E0120B7
:10C2A000621E00900138C9B2D2B201900290039090
:10C2B000DBB2784CA047784B784898470446D04783
:10C2C000774B97F84A201B7897F84A10CDF80090E2
:10C2D000CB1A03EBD373C2EB63014118CDF8049082
:10C2E0002046C9B26D4A4B466E4CA047664B1C783F
:10C2F00078E0297830460A1B514241EB02016A4B33
:10C300009847444568D254B95B4B30461A78674920
:10C31000D2F1010238BF0022654B98471EE000278A
:10C32000B9467B010BEB03023832127A92B9621ED6
:10C330004A450BD14F4A3046D3182A7803F12C01D5
:10C34000131B5A4242EB0302594B984709F101096A
:10C350005FFA89F90137402FE3D14CB92A7830468A
:10C36000D2F10102534938BF0022534B984733E0C2
:10C370004FF00009CA464FEA49135B4438331A7A32
:10C380002ABB611E51451ED1597A01290FD19F79CF
:10C390002B787FB2C4EB030C6331DCF1000397FB15
:10C3A000F1F1304643EB0C03444FB8470BE02A78D9
:10C3B0009979C4EB020EDEF10002304649B242EB3D
:10C3C0000E023F4B98470AF1010A5FFA8AFA09F117
:10C3D0000109B9F1400FCED13A4B01341B78E4B2D8
:10C3E000F618F6B29DF81F30A34282D83DE0B9F1AD
:10C3F000000F05D1344A01201070FF225A7035E039
:10C4000000242646204662010BEB02033833197ADA
:10C41000F1B96F78013FB74218D1587A01280DD190
:10C420009A7912B964329A7100E0997160015844A6
:10C430003E300121254B9847012007E00D4B244851
:10C440009A1851463E32FF23224FB8470136F6B2C2
:10C450000134402CD7D1012807D11B4B1870FF2382
:10C460006B70013802E0404600E0002009B0BDE8F2
:10C47000F08F00BF940E00203C00002014330020F9
:10C48000915F0008857D010882040020656B00082B
:10C49000673B010805340108795000084D8F0108F9
:10C4A00020010020BD380108A95E0008A07A01081B
:10C4B000015A0008DD7E0108415A0008255B00088A
:10C4C000795C00085C33002092000020A94F00082E
:10C4D000B27B01080D6700086B3B01082DE9F04FA6
:10C4E0003A4CDFF81C916378002587B0FF2B824619
:10C4F0008DF8175099F8496057D108462246062111
:10C50000631C334FB847DFF8FC80237841460DF1B8
:10C510001702504600932F4F0623DFF8ECA0B847D0
:10C52000D0472D4B834699F84A9098470746D04705
:10C53000C9EB0B0901220346009201950295039570
:10C5400028465FFA89F1254D3A46A84798F80050E9
:10C5500025E021783046C5EB010CDCF1000141EB10
:10C560000C011F4B9847052D13D8184B30461A78ED
:10C570001C4BC5EB020EDEF1000253F8251042EB16
:10C580000E02194B9847194B30465957FF22184B4A
:10C590009847184B01351B78EDB2F618F6B29DF8A6
:10C5A0001730AB42D5D8002007E04BB1013B1370E8
:10C5B00010460121104B984702E007B0BDE8F08F0C
:10C5C0000E4B01201870FF236370F6E7AC000020CB
:10C5D000915F0008656B0008673B0108053401089E
:10C5E000A95E000864000020015A0008908E01082E
:10C5F000D95A00085C330020A94F0008920000209F
:10C6000014330020860400206B3B01082DE9F04F15
:10C610005D4F5E4B7D7803F51256FF2D89B096F87D
:10C6200049409A46B84640F094803A467B1C4021E7
:10C63000574FB84798F80030564800935649402362
:10C640000DF11F02554FB84796F84A30002B34D0F1
:10C65000DFF88C91C84796F84A30514A05938346D3
:10C6600090470746C847059B7A1EDB439B44012140
:10C67000431E0020D2B2009101905FFA8BF102902C
:10C680000390DBB2474FB847474B484898470746A7
:10C69000C847474B96F84A201B7896F84A100095F1
:10C6A000CB1A03EBD373C2EB6301411801952B4600
:10C6B0003846C9B23D4A3F4DA847374B1D7843E045
:10C6C00098F800102046C5EB010CDCF1000141EBAD
:10C6D0000C01394B98473F2D2B4F2FD8374B384EF5
:10C6E00085B93A782046D2F1010238BF0022354997
:10C6F000984798F800202046D2F10102324938BF0D
:10C7000000221AE03A786901C5EB020E51440C315F
:10C71000DEF1000242EB0E02204698476B1C5B01E3
:10C7200053449B793A78012BC5EB02030CBF274990
:10C7300027495A42204642EB0302B047254B0135B8
:10C740001B78EDB2E418E4B29DF81F30AB42B7D8C5
:10C7500015E0214C25B90120FF2320707B700FE0EC
:10C76000681C4001181883790121C3F1010300F806
:10C77000063F1A4B984701232370FE337B7000203D
:10C7800009B0BDE8F08F00BF40000020940E0020EB
:10C79000915F0008947D0108AB040020656B0008E0
:10C7A000673B010805340108795000084D8F0108E6
:10C7B00020010020BD380108A95E0008015A0008C8
:10C7C000415A0008A07A0108DD7E01082080010896
:10C7D000B47A01085C33002092000020A94F0008C1
:10C7E0006B3B01082DE9F04F644F654B7D7803F5F5
:10C7F0001256FF2D89B096F849409A46B84640F047
:10C800009C803A467B1C40215E4FB84798F8003028
:10C810005D4800935D4940230DF11F025C4FB8470E
:10C8200096F84A30002B34D0DFF8A891C84796F824
:10C830004A30584A0593834690470746C847059BA8
:10C840007A1EDB439B440121431E0020D2B200919B
:10C8500001905FFA8BF102900390DBB24E4FB84724
:10C860004E4B4F4898470746C8474E4B96F84A20CC
:10C870001B7896F84A100095CB1A03EBD373C2EBE2
:10C880006301411801952B463846C9B2444A464DCA
:10C89000A8473E4B1D784BE098F800102046C5EBAA
:10C8A000010CDCF1000141EB0C01404B98473F2D9E
:10C8B000324F37D83E4B3F4E85B93A782046D2F1B9
:10C8C000010238BF00223C49984798F800202046D2
:10C8D000D2F10102394938BF002222E06A1E4FF02E
:10C8E000180909FB02F93A780AEB0901C5EB020EB7
:10C8F00001F502610C31DEF1000242EB0E0220462E
:10C90000D144984709F5026318339B793A78012B93
:10C91000C5EB02030CBF2A492A495A42204642EB82
:10C920000302B047284B01351B78EDB2E418E4B29E
:10C930009DF81F30AB42AFD81BE0244C25B9012035
:10C94000FF2320707B7015E01822013D55435A19D2
:10C9500092F83E185B19C1F1010103F5026082F8FB
:10C960003E181B4B1E300121984701232370FE33D4
:10C970007B70002009B0BDE8F08F00BF24000020CC
:10C98000940E0020915F0008A37D0108940400200C
:10C99000656B0008673B0108053401087950000801
:10C9A0004D8F010820010020BD380108A95E000854
:10C9B000015A0008415A0008A07A0108DD7E0108EA
:10C9C00020800108B47A01085C3300209200002026
:10C9D000A94F00086B3B01082DE9F04F7A4CDFF8B6
:10C9E000588294F80D9089B0B9F1FF0F8246154630
:10C9F00098F8496040F0B380084604F10C02072122
:10CA000004F10D03714FB847237B504600937049E2
:10CA100007230DF11F026F4FB84798F84A30002BDB
:10CA20003BD0DFF818A2D04798F84A306A4A0593FD
:10CA3000834690470746D047059B7A1EDB439B44BD
:10CA40000121431E0020D2B2009101905FFA8BF1C8
:10CA500002900390DBB2614FB847614F237B57F8D8
:10CA60002300604B98478346D0475F4B98F84A2095
:10CA70001B7898F84A10CDF80090CB1A03EBD373CB
:10CA8000C2EB6301237B411857F82320CDF80490B3
:10CA90005846C9B24B46554FB8474D4B1F7859E0E1
:10CAA000217B3046C7EB010CDCF1000141EB0C01AE
:10CAB0004F4B9847062FDFF8108145D898F80C2087
:10CAC0004C4BC7EB020EDEF1000253F8271042EB8D
:10CAD0000E023046484B98474FB998F864203D21E4
:10CAE000D2F10102304638BF0022444B2BE0BB1E7E
:10CAF000042B04D8DFE803F00D13191F2800227B54
:10CB00003046A2F101035A4242EB030229463C4B54
:10CB100019E0227B3046B5F91010022A0FE0227B83
:10CB20003046B5F91210032A09E0227B3046B5F9E8
:10CB30001410042A03E0227BA97D3046052A314BDC
:10CB400014BF0022012298472F4B01371B78FFB2F8
:10CB5000F618F6B29DF81F30BB42A1D82FE0B9F10C
:10CB6000060F2CD8DFE809F0040A0E1114191E0074
:10CB7000264B01201870FF23637321E02448FF2314
:10CB8000244D13E02448103204E02448123201E01E
:10CB900023481432FF23234D08E023481632FF2395
:10CBA000224D03E02248234D1832FF23A8470128D5
:10CBB00005D1164B1870FF236373013800E0002085
:10CBC00009B0BDE8F08F00BF68010020915F000848
:10CBD0008A040020656B0008673B010805340108E2
:10CBE000047A01087950000820010020BD380108AE
:10CBF000A95E00082C8E0108015A0008D95A0008C5
:10CC0000415A0008A95A00085C3300209200002015
:10CC10000989010815560008B27B0108D37C010878
:10CC2000C680010895550008FA7F0108F1500008F8
:10CC3000977F010881650008143300206B3B0108D1
:10CC40002DE9FF473C4B92463C4A93F84940D37B41
:10CC50000746FF2B154655D108460E32212105F116
:10CC60000F03374EB047DFF8FC80AB7B06460093DE
:10CC700038464146334F0DF10F022123B84798F84B
:10CC800000703AE0A97B2046C7EB010CDCF1000103
:10CC900041EB0C012C4BDFF8A48098474FB998F872
:10CCA0000E102046D1F1010138BF0021274B9847D3
:10CCB0001DE0202F1BD87B1E4FF01C0909FB03A988
:10CCC00098F80E202046C7EB020EDEF1000242EB80
:10CCD0000E0249461E4B984798F80E202046D31B5B
:10CCE0005A4242EB0302B9F910101A4B98471A4BFB
:10CCF00001371B78FFB2E418E4B29DF80F30BB4255
:10CD0000C0D80EE02BB9154B01201870FF23D37348
:10CD10000EE0013B1C2202FB03A2114CDBB2A04738
:10CD20000646012E03D10D4B1E70FF23EB7300202E
:10CD300004B0BDE8F08700BF143300206801002074
:10CD4000915F0008656B0008A95E0008555F000848
:10CD5000015A0008A95A00085C3300209200002004
:10CD6000D9C900085C0400202DE9F04F864CDFF89B
:10CD70009C8294F8199089B0B9F1FF0F824615464C
:10CD800098F8496040F0CA80084604F1180207216B
:10CD900004F119037D4FB847237E504600937C4928
:10CDA00007230DF11F027B4FB84798F84A30002B3C
:10CDB0003BD0DFF85CA2D04798F84A30764A05931A
:10CDC000834690470746D047059B7A1EDB439B442A
:10CDD0000121431E0020D2B2009101905FFA8BF135
:10CDE00002900390DBB26D4FB8476D4F237E57F82A
:10CDF00023006C4B98478346D0476B4B98F84A20EA
:10CE00001B7898F84A10CDF80090CB1A03EBD37337
:10CE1000C2EB6301237E411857F82320CDF804901C
:10CE20005846C9B24B46614FB847594B1F7870E01E
:10CE3000217E3046CA1B514241EB02015C4B9847B0
:10CE4000062FDFF844815ED898F81820594B3046F9
:10CE500053F82710D31B5A4242EB0302564B984714
:10CE60004FB998F864203D21D2F10102304638BF15
:10CE70000022524B46E0BB1E042B04D8DFE803F02F
:10CE8000081F28333900227E30462978012A1AE00B
:10CE900095F801E04A4BBEF13F0F03D9227E3046A0
:10CEA000484905E048494FEA4E1E227E304671440B
:10CEB000A2F1020CDCF1000242EB0C0222E0227E25
:10CEC000A9783046032A14BF002201223F4B19E003
:10CED000227E291DA2F1040EDEF10002304642EB53
:10CEE0000E023B4B0EE0227E304605F10801052A7A
:10CEF00004E0227E304605F10C01062A354B14BFB2
:10CF0000002201229847344B01371B78FFB2F618F4
:10CF1000F6B29DF81F30BB428AD831E0B9F1060F56
:10CF20002ED8DFE809F0040A0E13181D20002B4B41
:10CF300001201870FF23637623E02948FF23294D41
:10CF400015E029480132FF23284D10E0284802321D
:10CF5000FF23284D0BE028480432FF23274D06E02D
:10CF60002748083201E027480C32274DFF23A84705
:10CF7000012805D1194B1870FF236376013800E0B2
:10CF8000002009B0BDE8F08F68010020915F000823
:10CF900087040020656B0008673B01080534010821
:10CFA000B88E01087950000820010020BD38010822
:10CFB000A95E0008F4780108015A0008D95A00084F
:10CFC000415A0008CA7B0108C00E0020A95A000877
:10CFD0009D5D0008015D00085C3300209200002088
:10CFE000FA7F0108F1500008347F010859950008C4
:10CFF000CC7D010841660008DC7D0108199B000812
:10D00000E57D0108E77A0108019800081433002043
:10D010006B3B01082DE9F04F89B005929B46674AAA
:10D02000674B044693F84950D37E1646FF2B40F0D9
:10D03000998008461A32112106F11B03614FB84747
:10D04000B37E614F00938146394620460DF11F02A1
:10D050005E4C1123A0473C787EE0B17E2846C4EBAD
:10D060000108D8F1000141EB0801594B9847DFF85E
:10D0700094814CB9514B2846997E564BD1F1010110
:10D0800038BF0021984761E0102C5FD80598631ED7
:10D090004FF0140A0AFB030A9AF801305B4517D1D6
:10D0A0004D4B98474D4A98F8003011786FF00302C5
:10D0B000521A013B00218218EB180091FF310191B7
:10D0C0000291039102202946D2B2DBB2444FB84705
:10D0D0009AF80170434B3F2F15D9B27E2846C4EB16
:10D0E000020CDCF1000242EB0C023F499847B27E91
:10D0F0002846C4EB020EDEF100023C4942EB0E0270
:10D100003B4B984722E0B27E3A497F017918171BC2
:10D110007A4242EB0702284698472F4B98472F4BFD
:10D1200098F800E01B7898F800706FF00302D21AAC
:10D13000033F611E8218FFB26B1C0197C8B2CDF885
:10D1400000E0FF21D2B2DBB22B4FB84798F8003095
:10D150000134ED18EDB2E4B29DF81F30A3423FF662
:10D160007CAF1EE02BB9254B01201870FF23D3762E
:10D1700020E0BBF1FF0F09D005981422013B02FB10
:10D1800003035A78FF2A08BF83F801B0F37E2046D4
:10D19000059C013B142202FB0342DBB2184CA04762
:10D1A0008146B9F1010F04D1144B83F80090FF239D
:10D1B000F376002009B0BDE8F08F00BF68010020C1
:10D1C00014330020915F000888040020656B00087C
:10D1D000A95E0008555F0008673B01084400002075
:10D1E00005340108015A0008CA7B0108E87D0108DE
:10D1F000415A0008C00E0020C97E0008920000209D
:10D2000069CD00085C3300202DE9F04F7C4DDFF83C
:10D21000688295F81D9089B0B9F1FF0F82461646D5
:10D2200098F8494040F0BF80084605F11C020521EE
:10D2300005F11D03734FB8472B7F50460093724989
:10D2400005230DF11F02714FB84798F84A30002BA3
:10D250003BD0DFF828A2D04798F84A306C4A0593B3
:10D26000834690470746D047059B7A1EDB439B4485
:10D270000121431E0020D2B2009101905FFA8BF190
:10D2800002900390DBB2634FB847634F2B7F57F890
:10D290002300624B98478346D047614B98F84A2059
:10D2A0001B7898F84A10CDF80090CB1A03EBD37393
:10D2B000C2EB63012B7F411857F82320CDF804906F
:10D2C0005846C9B24B46574FB8474F4B1F7865E099
:10D2D000297F2046CB1B594241EB0301524B984713
:10D2E000042FDFF81C8153D898F81C204F4BC7EB54
:10D2F000020CDCF1000253F8271042EB0C0220462E
:10D300004B4B98474FB998F864203D21D2F1010268
:10D31000204638BF0022474B39E0032F98F81C20E5
:10D3200022D0042F2AD0022F14D096F800E0424BCE
:10D33000BEF13F0F02D92046404904E040494FEA80
:10D340004E1E20467144A2F1010EDEF1000242EBB6
:10D350000E021CE0A2F1020CDCF100022046717802
:10D3600042EB0C02374B12E0A2F1030E311DDEF14D
:10D370000002204642EB0E02334B08E0A2F1040308
:10D380005A4242EB0302314B204606F1080198470E
:10D390002F4B01371B78FFB2E418E4B29DF81F3021
:10D3A000BB4295D828E0B9F1040F25D8DFE809F091
:10D3B00003090D121700274B01201870FF236B770C
:10D3C0001BE02548FF23254C0DE025480132FF23B3
:10D3D000244C08E024480432FF23244C03E0244872
:10D3E000244C0832FF23A047012805D1194B18709F
:10D3F000FF236B77013800E0002009B0BDE8F08F13
:10D4000068010020915F000898040020656B000807
:10D41000673B010805340108E078010879500008ED
:10D4200020010020BD380108A95E0008647A0108C7
:10D43000015A0008D95A0008415A0008CA7B01085D
:10D44000C00E0020A95A00089D5D0008015D00087B
:10D450005C33002092000020347F010859950008B9
:10D46000FA7F0108F1500008DC7D0108199B0008D3
:10D47000EF7D010801980008143300206B3B010880
:10D480002DE9F04F89B090460593664A664B814678
:10D4900093F84950D37F1646FF2B40F099800846F9
:10D4A0001E32112106F11F03604CA047604FB37F6D
:10D4B000604C00938346394648460DF11F02112304
:10D4C000A0473C787EE0B17F2846C4EB0109D9F142
:10D4D000000141EB0901584B9847DFF890914CB996
:10D4E000504B2846997F554BD1F1010138BF00219F
:10D4F000984761E0102C5FD8631E4FF00C0A0AFBBE
:10D5000003FA059A18F80A30934217D14C4B984702
:10D510004C4A99F8003011786FF00302521A013B1F
:10D5200000218218EB180091FF31019102910391C3
:10D5300002202946D2B2DBB2434FB84718F80A702E
:10D54000424B3F2F15D9B27F2846C4EB020CDCF1C9
:10D55000000242EB0C023E499847B27F2846C4EBDA
:10D56000020EDEF100023B4942EB0E023A4B9847B5
:10D5700022E0B27F39497F017918171B7A4242EBCA
:10D580000702284698472E4B98472E4B99F800E003
:10D590001B7899F800706FF00302D21A033F611EE6
:10D5A0008218FFB26B1C0197C8B2CDF800E0FF21D2
:10D5B000D2B2DBB22A4FB84799F800300134ED18E7
:10D5C000EDB2E4B29DF81F30A3423FF67CAF1DE000
:10D5D0002BB9244B01201870FF23D3771FE0059A45
:10D5E000FF2A09D00C22013B534318F80320FF2ADD
:10D5F00004BF059A08F80320F37F0C22013B02FBCD
:10D6000003824846DBB2184CA0478346BBF1010FAA
:10D6100004D1144B83F800B0FF23F377002009B046
:10D62000BDE8F08F6801002014330020915F0008EE
:10D630008D040020656B0008A95E0008555F000896
:10D64000673B01084400002005340108015A000826
:10D65000CA7B0108F87D0108415A0008C00E00206D
:10D660007D7D00089200002009D200085C33002074
:10D670002DE9F04F754DDFF8408295F8219089B083
:10D68000B9F1FF0F8246164698F8494040F0B58040
:10D69000084605F12002042105F121036C4FB8472B
:10D6A00095F82030504600936A4904230DF11F027B
:10D6B000694FB84798F84A30002B3DD0DFF8FCA1FD
:10D6C000D04798F84A30654A059383469047074605
:10D6D000D047059B7A1EDB439B440121431E00205B
:10D6E000D2B2009101905FFA8BF102900390DBB20D
:10D6F0005B4FB8475B4F95F8203057F823005A4BE3
:10D7000098478346D047594B98F84A201B7898F899
:10D710004A10CDF80090CB1A03EBD373C2EB630130
:10D7200095F82030411857F82320CDF8049058463A
:10D73000C9B24B464E4FB847464B1F7858E095F854
:10D7400020102046CA1B514241EB0201494B984729
:10D75000032FDFF8F88045D898F82020464B204664
:10D7600053F82710D31B5A4242EB0302434B98470E
:10D770004FB998F864203D21D2F10102204638BF0C
:10D7800000223F4B2DE0022F98F8202016D0032FC7
:10D790001ED096F800E03B4BBEF13F0F02D9204669
:10D7A000394904E039494FEA4E1E20467144A2F13E
:10D7B000010CDCF1000242EB0C0212E0A2F1020EBD
:10D7C000311DDEF10002204642EB0E02304B08E034
:10D7D000A2F103035A4242EB03022E4B204606F10C
:10D7E000080198472C4B01371B78FFB2E418E4B2CC
:10D7F0009DF81F30BB42A2D824E0B9F1030F21D815
:10D80000DFE809F002090D12244B01201870FF23F4
:10D8100085F8213017E02248FF23224C08E02248F7
:10D820000432FF23214C03E02148224C0832FF231D
:10D83000A047012806D1194B1870FF2385F8213025
:10D84000013800E0002009B0BDE8F08F6801002039
:10D85000915F000867040020656B0008673B0108C2
:10D86000053401086C790108795000082001002076
:10D87000BD380108A95E000874780108015A000843
:10D88000D95A0008415A0008CA7B0108C00E00207E
:10D890009D5D0008015D00085C33002092000020BF
:10D8A000347F010859950008DC7D0108199B0008A8
:10D8B000FD7D010801980008143300206B3B01082E
:10D8C0002DE9F04F89B0904605936B4A6B4B81462A
:10D8D00093F8495092F823301646FF2B40F09F8072
:10D8E00008462232112106F12303654CA047654FFB
:10D8F00096F82230644C00938346394648460DF131
:10D900001F021123A0473C7883E096F82210284696
:10D91000C4EB0109D9F1000141EB09015B4B9847C8
:10D92000DFF89C9154B9544B284693F82210584B79
:10D93000D1F1010138BF0021984764E0102C62D872
:10D94000631E4FF00C0A0AFB03FA059A18F80A3016
:10D95000934217D14F4B98474F4A99F800301178AE
:10D960006FF00302521A013B00218218EB1800915C
:10D97000FF3101910291039102202946D2B2DBB21C
:10D98000464FB84718F80A70454B3F2F17D996F8FD
:10D9900022202846C4EB020CDCF1000242EB0C0210
:10D9A0004049984796F822202846C4EB020EDEF143
:10D9B00000023D4942EB0E023C4B984723E096F8AB
:10D9C00022203B497F017918171B7A4242EB07025C
:10D9D000284698472F4B98472F4B99F800E01B7823
:10D9E00099F800706FF00302D21A033F611E82188B
:10D9F000FFB26B1C0197C8B2CDF800E0FF21D2B294
:10DA0000DBB22C4FB84799F800300134ED18EDB275
:10DA1000E4B29DF81F30A3423FF677AF1FE033B961
:10DA2000254B01201870FF2382F8233021E0059A4E
:10DA3000FF2A09D00C22013B534318F80320FF2A88
:10DA400004BF059A08F8032096F823300C22013B06
:10DA500002FB03824846DBB2184CA0478346BBF169
:10DA6000010F05D1144B83F800B0FF2386F8233053
:10DA7000002009B0BDE8F08F6801002014330020B9
:10DA8000915F000881040020656B0008A95E000812
:10DA9000555F0008673B0108440000200534010879
:10DAA000015A0008CA7B0108037E0108415A000898
:10DAB000C00E0020157C00089200002071D60008DE
:10DAC0005C3300202DE9F04F9E4CDFF8D08294F8B3
:10DAD000259089B0B9F1FF0F8246154698F8496044
:10DAE00040F06081084604F124020D2104F1250371
:10DAF000954FB84794F824305046009393490D232E
:10DB00000DF11F02924FB84798F84A30002B3DD0D4
:10DB1000DFF88CA2D04798F84A308E4A05938346A6
:10DB200090470746D047059B7A1EDB439B44012163
:10DB3000431E0020D2B2009101905FFA8BF1029057
:10DB40000390DBB2844FB847844F94F8243057F8E1
:10DB50002300834B98478346D047824B98F84A204E
:10DB60001B7898F84A10CDF80090CB1A03EBD373CA
:10DB7000C2EB630194F82430411857F82320CDF804
:10DB800004905846C9B24B46774FB8476F4B1F7841
:10DB9000D2E094F824103046CB1B594241EB0301EC
:10DBA000724B98470C2FDFF89C8100F2BF8098F8E9
:10DBB00024206F4BC7EB020CDCF1000253F8271056
:10DBC00042EB0C0230466B4B98474FB998F86420F3
:10DBD0003D21D2F10102304638BF0022664BA4E05D
:10DBE000BB1E0A2B07D8DFE803F01A2632454C5F2C
:10DBF00066798096A10095F800E0604BBEF13F0F7A
:10DC000004D994F8242030465D4906E05D494FEA86
:10DC10004E1E94F8242030467144012A77E094F88F
:10DC20002420291DA2F1020EDEF10002304642EB53
:10DC30000E02554B79E094F824203046A2F10303FC
:10DC40005A4242EB030205F10801504B6DE02A7B7A
:10DC50004A4B3F2A04D994F824203046484907E02B
:10DC60004B49182000FB021194F82420304604315F
:10DC7000042A4CE094F82420304695F90D10052A2A
:10DC80004FE0AA7B3D4B3F2A04D994F8242030462C
:10DC90003B4907E03E49182000FB021194F824207C
:10DCA00030460431062A32E094F82420304695F9B3
:10DCB0000F10072A35E02A7C304B3F2A04D994F80C
:10DCC000242030462E4907E03149182000FB02117C
:10DCD00094F8242030460431082A18E094F82420CF
:10DCE000304695F91110092A1BE0AA7C234B3F2AE4
:10DCF00004D994F824203046214907E0244918200B
:10DD000000FB021194F82420304604310A2A14BF83
:10DD10000022012209E094F8242095F913103046DE
:10DD20000B2A1C4B14BF0022012298471A4B0137C3
:10DD30001B78FFB2F618F6B29DF81F30BB423FF6D3
:10DD400028AF78E068010020915F0008930400206C
:10DD5000656B0008673B010805340108A08D0108C8
:10DD60007950000820010020BD380108A95E000894
:10DD700020780108015A0008D95A0008415A0008C1
:10DD8000CA7B0108C00E00209D5D0008015D0008EF
:10DD9000BC160020A95A00085C3300201433002070
:10DDA0006B3B0108B9F10C0F45D8DFE809F0070E0D
:10DDB00010151A1D202326292C313600204B012056
:10DDC0001870FF2384F8253036E01E481DE01E48F9
:10DDD0000432FF231D4D24E01D480832FF231D4D52
:10DDE0001FE01D480C3210E01C480D3212E01C48A8
:10DDF0000E320AE01B480F320CE01B48103204E0E0
:10DE00001A48113206E01A481232FF23194D08E071
:10DE100019481332FF23194D03E01948194D1432E4
:10DE2000FF23A847012806D1054B1870FF2384F86B
:10DE30002530013800E0002009B0BDE8F08F00BFB8
:10DE4000920000200C7E0108DC7D0108199B00086F
:10DE5000177E0108019800081F7E01082C7E01082A
:10DE60003B7E0108487E0108577E0108647E010858
:10DE7000737E010841660008807E01080D67000876
:10DE80008F7E01082D9100082DE9F04F99466C4BCB
:10DE9000904693F849506B4A93F848308BB00693FC
:10DEA00092F827308246FF2B164640F09C800846A9
:10DEB0002632412106F12703634CA047634F96F8B1
:10DEC000263005900093624C504639460DF12702EA
:10DED0004123A0473C7880E096F8261028460B1B8B
:10DEE000594241EB03015B4B564F98474CB997F8A9
:10DEF00026102846D1F1010138BF0021564B984722
:10DF000066E0402C64D8631E34225A4318F802108D
:10DF10000792FF2997F82620504B02D128465049F6
:10DF20000DE0FE2902D128464E4908E03F2904D8D9
:10DF30004F014D492846791801E04C492846C4EB69
:10DF4000020CDCF1000242EB0C02DFF838A198472A
:10DF5000D047DFF834B1464A6FF00101137892F8E8
:10DF600000E09BF80020AEF1030E891A41185FFA19
:10DF70008EF0009096F82600671EC4EB000E6A1C17
:10DF8000DEF1000040EB0E000190C9B2F8B2D2B24F
:10DF9000384FB847B9F1FF0F1AD0079918F8013078
:10DFA0004B4515D1D0479BF8003006996FF0010220
:10DFB000D21A4B1E00218218EB180091FF310191FB
:10DFC0000291039102202946D2B2DBB22A4FB84710
:10DFD000069A0134AD18EDB2E4B29DF82730A342A1
:10DFE0003FF67AAF1EE033B9244B01201870FF23AF
:10DFF00082F8273020E0B9F1FF0F08D03422013B2E
:10E00000534318F80320FF2A08BF08F8039096F836
:10E0100027303422013B02FB03825046DBB2184C0E
:10E02000A0470590059B012B05D1144B059919704C
:10E03000FF2386F8273000200BB0BDE8F08F00BF2B
:10E040001433002068010020915F00089C04002028
:10E05000656B0008A95E0008555F0008015A0008BA
:10E060008D7B01089C7B0108C00E0020CA7B010843
:10E070005C330020C97400080534010892000020B8
:10E08000C5DA0008673B0108440000202DE9F04F85
:10E09000954CDFF8AC8294F8119089B0B9F1FF0F7C
:10E0A000824615469B4698F8496040F071810846C3
:10E0B00004F110020E2104F111038C4FB847237CA8
:10E0C000504600938A490E230DF11F02894FB8472D
:10E0D00098F84A30002B3DD0DFF868A2D04798F876
:10E0E0004A2085490492059088470746D047049AFC
:10E0F000059BD2439918431E01207A1E00900138D7
:10E10000C9B2D2B2019002900390DBB27B4FB84704
:10E110007B4F237C57F823007A4B98470490D047D5
:10E12000794B98F84A101B7898F84AE0049AC3EBA8
:10E130000E0303EBD373C1EB6301237C4118CDF8CD
:10E1400000901046CDF8049057F82320C9B24B46F2
:10E150006E4FB847664B93F8009013E1217C304630
:10E16000C9EB010CDCF1000141EB0C01684B984755
:10E17000B9F10D0F5C4FDFF8D08100F2FB803A7CE3
:10E18000644BC9EB020EDEF1000253F8291042EB9A
:10E190000E023046604B9847B9F1000F09D197F84D
:10E1A00064203D21D2F10102304638BF00225B4B92
:10E1B0009847514B98475A4B6FF003021B78D21A7D
:10E1C000821809F1FF33D2B20C2B00F2D380DFE8C2
:10E1D00013F00D00170022002E0035003C00420015
:10E1E0004900550061006F007D00BD00227C304673
:10E1F000A2F101035A4242EB03022946494B08E0CF
:10E20000227C95F912103046022A474B14BF002297
:10E2100001229847AEE0227C3046A2F1030CDCF1EB
:10E22000000295F9131042EB0C023C4BF1E7237C02
:10E230000222304695F91410042B19E0237C0322A6
:10E24000304695F91510052B12E0227C304695F9E1
:10E250001610062AD9E7237C0122304695F91A10B8
:10E26000072B05E0237C95F91B1005223046082B6F
:10E2700014BF002301232D4FB8477BE0227C30469A
:10E28000A2F1090EDEF1000205F11C0142EB0E02C3
:10E29000274BBEE798F8000098F80010731C03396C
:10E2A000C9B200900191FF205946DBB2214F60E0D6
:10E2B00098F8000098F80010731C0339C9B2009058
:10E2C0000191FF205946DBB21B4F52E098F8000045
:10E2D00098F80010731C0339C9B200900191FF2017
:10E2E0005946DBB2154F44E068010020915F0008F9
:10E2F0008F040020656B0008673B010805340108A6
:10E30000F48D01087950000820010020BD38010873
:10E31000A95E0008E8770108015A0008D95A0008E8
:10E3200044000020415A0008A95A0008255B000853
:10E33000015D0008157C00087D7D0008C97E00088D
:10E34000143300206B3B01085C33002098F8003048
:10E3500098F80010771C0339C9B20091217CA1F113
:10E360000D00414241EB000101911146FAB2344FD8
:10E370005846B84798F8003009F10109F618F6B286
:10E380005FFA89F99DF81F304B453FF6E7AE53E041
:10E39000B9F10D0F50D8DFE809F0070D1114191C61
:10E3A0002126292E33383D42264B01201870FF23A9
:10E3B000637442E02448FF23244D34E024481232A1
:10E3C0000EE024481332FF23234D2CE0234814325F
:10E3D0000EE023481532FF23224D24E02248163256
:10E3E000FF23224D1FE022481A3201E021481B3250
:10E3F000FF23214D17E021481C32FF23204D12E05E
:10E400002048214A5B46214D0DE02148214A5B46C8
:10E41000214D08E02148224A5B46224D03E0224874
:10E42000224A234D5B46A847012805D1054B1870A9
:10E43000FF236374013800E0002009B0BDE8F08FCD
:10E44000CD730008920000200989010815560008C4
:10E45000B27B0108318401084D610008E57E0108A6
:10E46000FA7F0108DDC40008F07E01080D6700088E
:10E4700020800108F87E0108F1500008047F01089F
:10E4800001980008317B010848210020C1D800080C
:10E490002C7B01088820002081D400083A7B0108E9
:10E4A0000822002015D00008877B0108482300209F
:10E4B00089DE00082DE9F04F8DB08A4B09928A4A17
:10E4C00093F84980D37C0546FF2B924640F0ED80BF
:10E4D0000846123241210AF11303844CA0479AF8EE
:10E4E0001230834C0790009328462146814D0DF150
:10E4F0002F024123A8472578D1E09AF81210404610
:10E50000C5EB010EDEF1000141EB0E017A4BDFF8A5
:10E51000D8B19847794C4DB99BF812104046D1F1CB
:10E52000010138BF0021764B9847B2E0402D00F240
:10E53000B0809BF81220099805F1FF39561B4FEA6D
:10E5400049137242034442EB0602194608934046BF
:10E550006C4B98476C4A90476C4A6FF0030C1378E9
:10E5600008F10107C3EB0C0C237822788444033AAA
:10E57000D2B200929BF812205FFA89F9501B4242F6
:10E5800042EB0002FFB25FFA8CFC61460192604EE2
:10E590003A46CDF818C04846B0472278DDF818C092
:10E5A0002378C0EB0C0C033B5FFA8CFCDBB20092CF
:10E5B00001936246FF2049463B46564ECDF818C0AF
:10E5C000B0472278DDF818C02378C0EB0C0C033B71
:10E5D0005FFA8CFCDBB2009201936246FF20494651
:10E5E0003B464D4ECDF818C0B0472278DDF818C034
:10E5F0002378C0EB0C0C033B5FFA8CFCDBB200927F
:10E6000001936246FF2049463B46444ECDF818C070
:10E61000B04723782278DDF818C0033AD2B20092CE
:10E620009BF81220C0EB0C0C511B4A4242EB01023A
:10E630005FFA8CFC61460192394E3A46CDF818C01B
:10E640004846B047DDF818C02F4BC0EB0C0C5FFA02
:10E650008CF698472D4B1A786FF003039B1A1B1802
:10E660009E4216D1089894F800C02278237890F939
:10E670001210CCEB0606033BF6B2DBB2009164212C
:10E68000019603920493029726480A460023264ED9
:10E69000B0472378013598445FFA88F8EDB29DF8C9
:10E6A0002F30AB423FF629AF0EE02BB91F4B0120B4
:10E6B0001870FF23D37412E0099C013B5A01A21881
:10E6C000DBB21B4CA04707900798012806D1174BD7
:10E6D0001870FF238AF81330013800E000200DB0D5
:10E6E000BDE8F08F1433002068010020915F00081E
:10E6F000A4040020656B0008A95E00085C330020BC
:10E70000555F0008015A0008673B010844000020DB
:10E71000CD730008157C00087D7D0008C97E0008C7
:10E72000C58200080B7F0108757800089200002060
:10E730008DE000082DE9F04F7B4DDFF85C8295F805
:10E74000299089B0B9F1FF0F8246164698F84940E2
:10E7500040F0BD80084605F12802052105F1290396
:10E76000724FB84795F828305046009370490523FA
:10E770000DF11F026F4FB84798F84A30002B3DD07B
:10E78000DFF818A2D04798F84A306B4A05938346C1
:10E7900090470746D047059B7A1EDB439B440121E7
:10E7A000431E0020D2B2009101905FFA8BF10290DB
:10E7B0000390DBB2614FB847614F95F8283057F8A6
:10E7C0002300604B98478346D0475F4B98F84A2018
:10E7D0001B7898F84A10CDF80090CB1A03EBD3734E
:10E7E000C2EB630195F82830411857F82320CDF883
:10E7F00004905846C9B24B46544FB8474C4B1F780B
:10E8000060E095F828102046CB1B594241EB0301EC
:10E810004F4B9847042FDFF810814DD898F82820E7
:10E820004C4BC7EB020CDCF1000253F8271042EB13
:10E830000C022046484B98474FB998F864203D2178
:10E84000D2F10102204638BF0022444B33E0032FAF
:10E8500098F8282022D0042F25D0022F14D0307809
:10E860003F4B3F2802D920463E4906E03E494FF043
:10E87000180E0EFB001120460431A2F1010EDEF14C
:10E88000000242EB0E0216E0A2F1020C311DDCF197
:10E890000002204642EB0C02344B0CE0204606F10D
:10E8A0000801032A03E0204606F10C01042A304B3C
:10E8B00014BF0022012298472E4B01371B78FFB26C
:10E8C000E418E4B29DF81F30BB429AD828E0B9F1B1
:10E8D000040F25D8DFE809F0030A0E131600264BB3
:10E8E00001201870FF2385F829301AE02348FF2300
:10E8F000234C0BE023480432FF23234C06E023483B
:10E90000083201E022480C32224CFF23A0470128A4
:10E9100006D1194B1870FF2385F82930013800E023
:10E92000002009B0BDE8F08F68010020915F000869
:10E93000B3040020656B0008673B0108053401083B
:10E94000A47801087950000820010020BD38010892
:10E95000A95E00088C8D0108015A0008D95A0008E8
:10E96000415A0008CA7B0108BC1600209D5D0008C2
:10E97000015D00085C33002092000020347F010814
:10E98000ED960008DC7D0108199B0008E57D010873
:10E99000E77A010801980008143300206B3B010856
:10E9A0002DE9F04F89B0904605936B4A6B4B814639
:10E9B00093F8495092F82B301646FF2B40F0A08078
:10E9C00008462A32112106F12B03654CA047654FFA
:10E9D00096F82A30644C00938346394648460DF138
:10E9E0001F021123A0473C7884E096F82A1028469D
:10E9F000C4EB0109D9F1000141EB09015B4B9847D8
:10EA0000DFF89C9154B9544B284693F82A10584B80
:10EA1000D1F1010138BF0021984765E0102C63D87F
:10EA200004F1FF3A4FEA0A1A18F80A30059A93429D
:10EA300017D1504B9847504A99F8003011786FF031
:10EA40000302521A013B00218218EB180091FF319A
:10EA500001910291039102202946D2B2DBB2474FC5
:10EA6000B84718F80A20464B3F2A17D996F82A20AB
:10EA70002846C4EB020CDCF1000242EB0C024149D7
:10EA8000984796F82A202846C4EB020EDEF10002D1
:10EA90003D4942EB0E023D4B984725E03C4918208A
:10EAA00000FB021196F82A200431171B7A4242EB30
:10EAB0000702284698472F4B98472F4B99F800E0BC
:10EAC0001B7899F800706FF00302D21A033F611EA1
:10EAD0008218FFB26B1C0197C8B2CDF800E0FF218D
:10EAE000D2B2DBB22B4FB84799F800300134ED18A1
:10EAF000EDB2E4B29DF81F30A3423FF676AF1DE0C1
:10EB000033B9254B01201870FF2382F82B301FE00A
:10EB1000059AFF2A08D0013B1B0118F80320FF2AA1
:10EB200004BF059A08F8032096F82B304846013BAD
:10EB300008EB0312194CDBB2A0478346BBF1010F6F
:10EB400005D1154B83F800B0FF2386F82B30002049
:10EB500009B0BDE8F08F00BF680100201433002029
:10EB6000915F000895040020656B0008A95E00080D
:10EB7000555F0008673B0108440000200534010888
:10EB8000015A0008CA7B0108117F0108415A000898
:10EB9000BC160020358000089200002035E70008F0
:10EBA0005C3300202DE9F04F7B4DDFF85C8295F857
:10EBB0002D9089B0B9F1FF0F8246164698F849406A
:10EBC00040F0BC80084605F12C02052105F12D031B
:10EBD000724FB84795F82C30504600937049052382
:10EBE0000DF11F026F4FB84798F84A30002B3DD007
:10EBF000DFF818A2D04798F84A306B4A059383464D
:10EC000090470746D047059B7A1EDB439B44012172
:10EC1000431E0020D2B2009101905FFA8BF1029066
:10EC20000390DBB2614FB847614F95F82C3057F82D
:10EC30002300604B98478346D0475F4B98F84A20A3
:10EC40001B7898F84A10CDF80090CB1A03EBD373D9
:10EC5000C2EB630195F82C30411857F82320CDF80A
:10EC600004905846C9B24B46544FB8474C4B1F7896
:10EC70005FE095F82C102046CB1B594241EB030175
:10EC80004F4B9847042FDFF810814CD898F82C2070
:10EC90004C4BC7EB020CDCF1000253F8271042EB9F
:10ECA0000C022046484B98474FB998F864203D2104
:10ECB000D2F10102204638BF0022444B32E0032F3C
:10ECC00098F82C2021D0042F24D0022F14D0307893
:10ECD0003F4B3F2802D920463E4906E03E494FF0CF
:10ECE000180E0EFB001120460431A2F1010EDEF1D8
:10ECF000000242EB0E0215E0A2F10203311D5A425E
:10ED000042EB03022046354B0CE0204606F1080199
:10ED1000032A03E0204606F10C01042A304B14BFFD
:10ED20000022012298472F4B01371B78FFB2E418CD
:10ED3000E4B29DF81F30BB429BD828E0B9F1040F24
:10ED400025D8DFE809F0030A0E131600264B012030
:10ED50001870FF2385F82D301AE02448FF23244C37
:10ED60000BE024480432FF23234C06E023480832FA
:10ED700001E023480C32234CFF23A047012806D191
:10ED8000194B1870FF2385F82D30013800E0002062
:10ED900009B0BDE8F08F00BF68010020915F000856
:10EDA0006A040020656B0008673B01080534010810
:10EDB000507A01087950000820010020BD38010870
:10EDC000A95E00087C8E0108015A0008D95A000883
:10EDD000415A0008CA7B0108BC1600209D5D00084E
:10EDE000015D00085C33002092000020347F0108A0
:10EDF000ED960008DC7D0108199B0008E57D0108FF
:10EE0000E77A010801980008143300206B3B0108E1
:10EE10002DE9F04F89B0904605936B4A6B4B8146C4
:10EE200093F8495092F82F301646FF2B40F0A080FF
:10EE300008462E32112106F12F03654CA047654F7D
:10EE400096F82E30644C00938346394648460DF1BF
:10EE50001F021123A0473C7884E096F82E10284624
:10EE6000C4EB0109D9F1000141EB09015B4B984763
:10EE7000DFF89C9154B9544B284693F82E10584B08
:10EE8000D1F1010138BF0021984765E0102C63D80B
:10EE900004F1FF3A4FEA0A1A18F80A30059A934229
:10EEA00017D1504B9847504A99F8003011786FF0BD
:10EEB0000302521A013B00218218EB180091FF3126
:10EEC00001910291039102202946D2B2DBB2474F51
:10EED000B84718F80A20464B3F2A17D996F82E2033
:10EEE0002846C4EB020CDCF1000242EB0C02414963
:10EEF000984796F82E202846C4EB020EDEF1000259
:10EF00003D4942EB0E023D4B984725E03C49182015
:10EF100000FB021196F82E200431171B7A4242EBB7
:10EF20000702284698472F4B98472F4B99F800E047
:10EF30001B7899F800706FF00302D21A033F611E2C
:10EF40008218FFB26B1C0197C8B2CDF800E0FF2118
:10EF5000D2B2DBB22B4FB84799F800300134ED182C
:10EF6000EDB2E4B29DF81F30A3423FF676AF1DE04C
:10EF700033B9254B01201870FF2382F82F301FE092
:10EF8000059AFF2A08D0013B1B0118F80320FF2A2D
:10EF900004BF059A08F8032096F82F304846013B35
:10EFA00008EB0312194CDBB2A0478346BBF1010FFB
:10EFB00005D1154B83F800B0FF2386F82F300020D1
:10EFC00009B0BDE8F08F00BF6801002014330020B5
:10EFD000915F0008AD040020656B0008A95E000881
:10EFE000555F0008673B0108440000200534010814
:10EFF000015A0008CA7B0108157F0108415A000820
:10F00000BC1600207D81000892000020A5EB0008BE
:10F010005C3300202DE9F04FA24CDFF81C8394F8FC
:10F02000319089B0B9F1FF0F824616469B4698F899
:10F03000495040F0FD80084604F13002082104F1F7
:10F040003103994FB84794F83030504600939749B0
:10F0500008230DF11F02964FB84798F84A30002B4D
:10F060003FD0DFF8D8A2D04798F84A2091490492BF
:10F07000059088470746D047049A059BD2439918C4
:10F08000431E01207A1E00900138C9B2D2B201900D
:10F0900002900390DBB2884FB847884F94F8303025
:10F0A00057F82300864B98470490D047854B98F833
:10F0B0004A101B7898F84AE0049AC3EB0E0303EB5E
:10F0C000D373C1EB630194F830304118CDF8009050
:10F0D0001046CDF8049057F82320C9B24B467A4F1A
:10F0E000B847724B93F800809CE094F830102846A3
:10F0F000C8EB0102514241EB0201744B9847B8F151
:10F10000070F684FDFF8389200F2848097F83020BC
:10F110006F4B284653F82810C8EB02035A4242EBC3
:10F1200003026C4B9847B8F1000F09D197F864209F
:10F130003D21D2F10102284638BF0022664B984794
:10F140005C4B9847654B6FF003021B78D21A82180C
:10F1500008F1FF33D2B2062B5CD8DFE803F00410CD
:10F160001E26333F4D0094F830202846A2F1010CB2
:10F17000DCF10002314642EB0C02594B0BE094F8F3
:10F180003020B6F91010A2F1020EDEF10002554B4C
:10F19000284642EB0E0298473CE094F830300122BA
:10F1A000284696F91210032B06E094F8303096F9B1
:10F1B000131005222846042B14BF002301234A4FB5
:10F1C000B84727E094F830202846A2F105035A42B8
:10F1D00042EB030206F11401444BDCE799F800000E
:10F1E00099F800106B1C0339C9B200900191FF20FF
:10F1F0005946DBB23E4F0CE099F8000099F8001038
:10F200006B1C0339C9B23B4F00900191FF20594656
:10F21000DBB2B84799F8003008F10108ED18EDB2FB
:10F220005FFA88F89DF81F3043453FF65EAF89E0EE
:10F23000B9F1070F00F28680DFE809F0040B0F1424
:10F24000171C21262C4B01201870FF2384F8313025
:10F2500079E02A48FF232A4D1AE02A481032FF237A
:10F26000294D15E02948123201E029481332FF23C5
:10F27000284D0DE028481432FF23284D08E0284887
:10F28000284A5B46284D03E02848294A294D5B4619
:10F29000A847012856D1184B1870FF2384F8313045
:10F2A000013850E068010020915F0008A5040020AB
:10F2B000656B0008673B010805340108787A01088E
:10F2C0007950000820010020BD380108A95E00081F
:10F2D000EC8C0108015A0008D95A000844000020AB
:10F2E000415A0008A95A0008255B0008015D000882
:10F2F000358000087D8100089200002009890108FE
:10F3000015560008B27B01089555000820800108B9
:10F31000F87E0108F1500008047F010801980008F8
:10F32000417B010848300020A1E90008457B010825
:10F330004831002011EE0008143300206B3B010817
:10F340005C330020002009B0BDE8F08F2DE9F04FBC
:10F350008DB0774B0992774A93F8496092F8333031
:10F360000546FF2B904640F0C680084632324121C8
:10F3700008F13303704CA04798F832306F4C079077
:10F380000093284621466E4D0DF12F024123A847D8
:10F3900037462578A9E098F832103846C5EB010EBB
:10F3A000DEF1000141EB0E01664BDFF888B19847B2
:10F3B000654C4DB99BF832103846D1F1010138BF88
:10F3C0000021624B98478BE0402D00F2898009991B
:10F3D00005F1FF3A182303FB0A139BF83220194664
:10F3E000561B724242EB060208933846584B984728
:10F3F000584A904758496FF0030C0B782278C3EBBA
:10F400000C0C23788444033B07F101095FFA8CFC60
:10F410005FFA8AFA5FFA89F9DBB2009201936246D9
:10F42000FF2051464B464D4ECDF818C0B0472278CC
:10F43000DDF818C02378C0EB0C0C033B5FFA8CFCA2
:10F44000DBB2009201936246FF2051464B46444E88
:10F45000CDF818C0B04723782278DDF818C0033AF9
:10F46000D2B200929BF83220C0EB0C0C511B4A42E6
:10F4700042EB01025FFA8CFC61460192394E4A462A
:10F48000CDF818C05046B047DDF818C0314AC0EB7F
:10F490000C0C5FFA8CF690472F4B1A786FF0030331
:10F4A0009B1A1B189E421BD1089994F800C0B1F911
:10F4B000100022781421237890FBF1F149B2CCEBB3
:10F4C0000606033BF6B2DBB200916421019603927B
:10F4D0000493CDF8089024480A460023234EB047F1
:10F4E00023780135FF18FFB2EDB29DF82F30AB4203
:10F4F0003FF651AF10E033B91D4B01201870FF23C8
:10F5000082F8333011E0099C013B182202FB0342D0
:10F51000DBB2184CA04707900799012904D1144B7E
:10F520001970FF2388F8333000200DB0BDE8F08F4C
:10F530001433002068010020915F00087F04002040
:10F54000656B0008A95E00085C330020555F000869
:10F55000015A0008673B010844000020358000087C
:10F560007D8100088D7400081D7F010875780008F2
:10F570009200002015F000082DE9F04F6E4DDFF8E5
:10F58000148295F8399089B0B9F1FF0F824616467A
:10F5900098F8494040F0A480084605F1380205215A
:10F5A00005F13903654FB84795F838305046009358
:10F5B000634905230DF11F02624FB84798F84A309E
:10F5C000002B3DD0DFF8D0A1D04798F84A305E4AF2
:10F5D0000593834690470746D047059B7A1EDB4339
:10F5E0009B440121431E0020D2B2009101905FFA9A
:10F5F0008BF102900390DBB2544FB847544F95F80B
:10F60000383057F82300534B98478346D047524B26
:10F6100098F84A201B7898F84A10CDF80090CB1A39
:10F6200003EBD373C2EB630195F83830411857F8F8
:10F630002320CDF804905846C9B24B46474FB847EF
:10F640003F4B1F7847E095F838102046CB1B5942B6
:10F6500041EB0301424B9847042FDFF8DC8034D89C
:10F6600098F838203F4BC7EB020CDCF1000253F84E
:10F67000271042EB0C0220463B4B98474FB998F8B5
:10F6800064203D21D2F10102204638BF0022374BD1
:10F690001AE0032F98F83820354B0BD0042F0DD0EB
:10F6A000022F03D020463178012A0AE020467178E3
:10F6B000022A06E02046B178032A02E0F1782046CB
:10F6C000042A14BF0022012298472A4B01371B78D5
:10F6D000FFB2E418E4B29DF81F30BB42B3D826E075
:10F6E000B9F1040F23D8DFE809F0030A0C0F140066
:10F6F000214B01201870FF2385F8393018E01F488E
:10F7000009E01F48013206E01E480232FF231E4C6A
:10F7100003E01E4803321E4CFF23A047012806D1F8
:10F72000154B1870FF2385F83930013800E00020B0
:10F7300009B0BDE8F08F00BF68010020915F0008AC
:10F7400084040020656B0008673B0108053401084C
:10F75000688E01087950000820010020BD3801089A
:10F76000A95E0008A4790108015A0008D95A0008C6
:10F77000A95A00085C33002092000020247F010871
:10F78000307F0108FA7F0108F15000083C7F010832
:10F7900041660008143300206B3B01082DE9FF414E
:10F7A00094463B4B3B4A93F8494092F83B3007461E
:10F7B000FF2B154651D108463A32032105F13B0390
:10F7C000354EB047DFF8F88095F83A30064600939A
:10F7D00038464146314F0DF10F020323B84798F8E0
:10F7E000007035E095F83A102046CB1B594241EBAA
:10F7F00003012B4BDFF89C8098474FB998F83A10DB
:10F800002046D1F1010138BF0021264B984719E06D
:10F81000022F17D898F83A202046C7EB020CDCF1EB
:10F82000000242EB0C022049204B984798F83A20FE
:10F83000791EC7EB020EDEF10002204642EB0E02FB
:10F840001B4B98471B4B01371B78FFB2E418E4B2FF
:10F850009DF80F30BB42C5D80FE033B9164B0120DD
:10F860001870FF2382F83B300FE0013B242202FB9B
:10F8700003C2124CDBB2A0470646012E04D10E4B48
:10F880001E70FF2385F83B30002004B0BDE8F081F6
:10F890001433002068010020915F0008656B0008A8
:10F8A000A95E0008555F00087C800108015A000825
:10F8B000A95A00085C3300209200002079F5000866
:10F8C000A20400202DE9F04F984CDFF8E88294F86C
:10F8D000359089B0B9F1FF0F8246154698F8496016
:10F8E00040F0E480084604F134020A2104F13503B3
:10F8F0008F4FB84794F83430504600938D490A230F
:10F900000DF11F028C4FB84798F84A30002B3DD0BC
:10F91000DFF8A4A2D04798F84A30884A0593834676
:10F9200090470746D047059B7A1EDB439B44012145
:10F93000431E0020D2B2009101905FFA8BF1029039
:10F940000390DBB27E4FB8477E4F94F8343057F8BF
:10F9500023007D4B98478346D0477C4B98F84A203C
:10F960001B7898F84A10CDF80090CB1A03EBD373AC
:10F97000C2EB630194F83430411857F82320CDF8D6
:10F9800004905846C9B24B46714FB847694B93F83B
:10F99000008085E094F834103046C8EB01035942EA
:10F9A00041EB03016B4B9847B8F1090F5F4F6FD8DC
:10F9B00097F83420684BC8EB020CDCF1000253F8D6
:10F9C000281042EB0C023046644B9847B8F1000F08
:10F9D00009D197F864203D21D2F10102304638BFA9
:10F9E00000225F4B53E0A8F10203072B05D8DFE8A4
:10F9F00003F00A121A272D33394394F83420304685
:10FA00002978012A33E094F834300422304695F9FD
:10FA10000110022B0EE094F834300022304695F9A4
:10FA20000210032B06E094F8343095F903100022FD
:10FA30003046042B14BF002301234A4FB84727E068
:10FA400094F834203046A988052A10E094F8342030
:10FA50003046E988062A0AE094F83420304629899D
:10FA6000072A04E094F8342069893046082A14BF34
:10FA7000002201223C4B0AE094F834203B49A2F1D9
:10FA8000090EDEF100023A4B304642EB0E02984777
:10FA9000384B08F101081B785FFA88F8F618F6B2BF
:10FAA0009DF81F3043453FF675AF87E0B9F1090F68
:10FAB00000F28480DFE809F0050C1114171C1F22E6
:10FAC000262C2D4B01201870FF2384F8353076E06A
:10FAD0002A462A48FF232A4D1DE02A486A1C04E0D2
:10FAE0002948AA1C01E02948EA1CFF23284D12E0FE
:10FAF00028482A1D09E02848AA1D06E0274805F1E4
:10FB0000080202E0264805F10A02FF23254D02E023
:10FB10002548264A264DA84701284FD1164B187074
:10FB2000FF2384F83530013849E000BF6801002028
:10FB3000915F000869040020656B0008673B0108BD
:10FB4000053401087C790108795000082001002063
:10FB5000BD380108A95E000844790108015A00086F
:10FB6000D95A0008255B0008A95A0008DD7E010863
:10FB7000415A00085C330020920000203C7F0108BD
:10FB800041660008457F01084C7F0108527F01084B
:10FB9000F15000085D7F0108587F0108DE7A0108F6
:10FBA000637F010841550008697F0108A0320020E9
:10FBB0009DF70008143300206B3B0108002009B0BA
:10FBC000BDE8F08F2DE9FF4194463B4B3B4A93F84B
:10FBD000494092F837300746FF2B154651D1084669
:10FBE0003632032105F13703354EB047DFF8F88090
:10FBF00095F836300646009338464146314F0DF1B0
:10FC00000F020323B84798F8007035E095F83610D6
:10FC10002046CB1B594241EB03012B4BDFF89C8064
:10FC200098474FB998F836102046D1F1010138BFF6
:10FC30000021264B984719E0022F17D898F8362054
:10FC40002046C7EB020CDCF1000242EB0C0220491B
:10FC5000204B984798F83620791EC7EB020EDEF14C
:10FC60000002204642EB0E021B4B98471B4B01370C
:10FC70001B78FFB2E418E4B29DF80F30BB42C5D840
:10FC80000FE033B9164B01201870FF2382F837308C
:10FC90000FE0013B2C2202FB03C2124CDBB2A04757
:10FCA0000646012E04D10E4B1E70FF2385F8373017
:10FCB000002004B0BDE8F08114330020680100206A
:10FCC000915F0008656B0008A95E0008555F000899
:10FCD000727F0108015A0008A95A00085C3300200D
:10FCE00092000020C5F800088E0400202DE9F04F96
:10FCF000954DDFF8C88295F8419089B0B9F1FF0FB2
:10FD00008246144698F8496040F0EC80084605F1B8
:10FD100040020D2105F141038C4FB84795F8403062
:10FD2000504600938A490D230DF11F02894FB847B1
:10FD300098F84A30002B3DD0DFF884A2D04798F8DD
:10FD40004A30854A0593834690470746D047059B2E
:10FD50007A1EDB439B440121431E0020D2B2009156
:10FD600001905FFA8BF102900390DBB27B4FB847B2
:10FD70007B4F95F8403057F823007A4B98478346DD
:10FD8000D047794B98F84A201B7898F84A10CDF85C
:10FD90000090CB1A03EBD373C2EB630195F84030AC
:10FDA000411857F82320CDF804905846C9B24B4665
:10FDB0006E4FB847664B1F788EE095F8401030467E
:10FDC000C7EB010CDCF1000141EB0C01684B9847DB
:10FDD0000C2FDFF8748179D898F84020654BC7EB79
:10FDE000020EDEF1000253F8271042EB0E023046FD
:10FDF000614B98474FB998F864203D21D2F1010238
:10FE0000304638BF00225D4B5FE0BB1E0A2B07D88F
:10FE1000DFE803F00C1319252B31373D434A51001D
:10FE200095F840203046217D012A4AE095F840208F
:10FE3000304694F91510022A43E095F840203046E8
:10FE4000A17D032A3DE095F840203046A2F104034D
:10FE50005A4242EB030204F11801494B35E095F890
:10FE600040203046217F052A2BE095F8402030467F
:10FE7000617F062A25E095F840203046A17F072AB9
:10FE80001FE095F840203046218C082A19E095F8AB
:10FE900040203046618C092A13E095F84020304616
:10FEA00094F825100A2A0CE095F84020304694F882
:10FEB00026100B2A05E095F8402094F827103046CC
:10FEC0000C2A304B14BF0022012298472E4B0137D9
:10FED0001B78FFB2F618F6B29DF81F30BB423FF612
:10FEE0006CAF7CE0B9F10C0F79D8DFE809F0070EB0
:10FEF0001116191E21247272272A6B00234B012030
:10FF00001870FF2385F841306AE0214814325BE025
:10FF100020481532FF23204C58E02048163253E089
:10FF20001F481832FF231F4C50E01F481C324BE083
:10FF30001E481D3248E01E481E3245E01D4825324D
:10FF400042E01D4826323FE068010020915F000832
:10FF5000AF040020656B0008673B01080534010809
:10FF6000D48E01087950000820010020BD38010816
:10FF7000A95E000810790108015A0008D95A000842
:10FF8000015D0008A95A00085C330020920000209F
:10FF9000927F01089D7F01080D670008A97F010875
:10FFA000B67F010801980008C07F0108CD7F0108D5
:10FFB000D97F0108E57F0108F27F01081433002092
:10FFC0006B3B010808482732084CFF23A047012853
:10FFD00005D1074B01221A70FF2385F8413000201C
:10FFE00009B0BDE8F08F00BFFF7F0108416600083F
:10FFF000920000202DE9F04F784BDFF8289293F81B
:020000040801F1
:10000000458089B0B8F1FF0F8246164699F84950ED
:100010001C4640F0C98003F14402084645330821DC
:100020006F4FB84794F84430504600936D49082309
:100030000DF11F026C4FB84799F84A30002B3DD0A4
:10004000DFF8E4A1D04799F84A30684A059383461F
:1000500090470746D047059B7A1EDB439B4401210E
:10006000431E0020D2B2009101905FFA8BF1029002
:100070000390DBB25E4FB8475E4F94F8443057F8B8
:1000800023005D4B98478346D0475C4B99F84A2044
:100090001B7899F84A10CB1A03EBD373C2EB6301B8
:1000A00094F84430411857F82320CDF80080CDF85B
:1000B00004805846C9B24346514FB847494B1F7850
:1000C0006DE094F844102846C7EB010CDCF1000108
:1000D00041EB0C014B4B9847072FDFF8008158D8B4
:1000E00098F84420484BC7EB020EDEF1000253F8AB
:1000F000271042EB0E022846444B98474FB998F818
:1001000064203D21D2F10102284638BF0022404B35
:100110003EE0BB1E052B04D8DFE803F00E141B22C3
:10012000293094F844202846A2F101035A4242EBB8
:1001300003023168374B2BE094F84420311D2846E8
:10014000022A21E094F84420284606F11401032AEB
:100150001AE094F84420284606F12401042A13E00A
:1001600094F84420284606F13401052A0CE094F85E
:100170004420284606F14401062A05E094F844206C
:10018000284606F5A271072A234B14BF002201223C
:100190009847224B01371B78FFB2ED18EDB29DF85E
:1001A0001F30BB428DD80DE0B8F1000F03D0B8F17D
:1001B000070F07D80AE01A4A01201070FF2283F8BF
:1001C000452000E0002009B0BDE8F08F144A01216D
:1001D0001170FF2283F84520F4E700BF680100207A
:1001E000915F00087C040020656B0008673B0108F4
:1001F00005340108207A0108795000082001002008
:10020000BD380108A95E0008488E0108015A00089F
:10021000D95A0008A95A0008415A00085C33002046
:1002200092000020143300206B3B01082DE9F04FB1
:100230005C4FDFF8C08197F84D408146FF2C87B0B6
:10024000084698F849503E4640F08F8007F14C022E
:1002500007F14D030221544FB84796F84C304846F9
:100260000093524902230DF11702514FB84798F8F5
:100270004A30002B3AD0DFF88091C8474D4B824678
:1002800098F84AB098470746C8476FEA0B0BDA441C
:100290007A1E431E01210020D2B2009101905FFA24
:1002A0008AF102900390DBB2434FB84796F84C3086
:1002B000424F57F82300424B98478246C847414B6C
:1002C00098F84A201B7898F84A10CB1A03EBD3739E
:1002D000C2EB630196F84C3041180094019457F832
:1002E000232050462346C9B2374CA0472F4B1C78D9
:1002F00036E096F84C1028460B1B594241EB03019F
:10030000324B9847012C274F24D897F84C20304B7C
:10031000C4EB020CDCF1000253F8241042EB0C0297
:1003200028462C4B98474CB997F864203D21D2F1D0
:100330000102284638BF0022274B0AE097F84C20DC
:100340002649A2F1010EDEF10002254B284642EBC0
:100350000E029847234B01341B78E4B2ED18EDB23E
:100360009DF81730A342C4D818E014B1012C15D160
:1003700006E01D4B01201870FF2387F84D300EE07A
:100380001A4808F10C021A4B9847012806D1164B5F
:100390001870FF2387F84D30013800E0002007B0C7
:1003A000BDE8F08F68010020915F00086404002020
:1003B000656B0008673B010805340108B87901083E
:1003C0007950000820010020BD380108A95E00080E
:1003D000548D0108015A0008D95A0008DD7E010831
:1003E000415A00085C330020920000200E80010872
:1003F000C5BE0008143300206B3B01082DE9F04F07
:100400009B4CDFF8D48294F8519089B0B9F1FF0F7A
:100410008246164698F8495040F00881084604F193
:100420005002092104F15103924FB84794F850301B
:1004300050460093904909230DF11F028F4FB84792
:1004400098F84A30002B3DD0DFF890A2D04798F8BA
:100450004A308B4A0593834690470746D047059B11
:100460007A1EDB439B440121431E0020D2B200913F
:1004700001905FFA8BF102900390DBB2814FB84795
:10048000814F94F8503057F82300804B98478346AB
:10049000D0477F4B98F84A201B7898F84A10CDF83F
:1004A0000090CB1A03EBD373C2EB630194F8503086
:1004B000411857F82320CDF804905846C9B24B464E
:1004C000744FB8476C4B1F78AAE094F85010284638
:1004D000C7EB010CDCF1000141EB0C016E4B9847BE
:1004E000082FDFF88C8100F2958098F850206B4B34
:1004F000C7EB020EDEF1000253F8271042EB0E02AA
:100500002846674B98474FB998F864203D21D2F1AF
:100510000102284638BF0022624B7AE0BB1E062B40
:1005200005D8DFE803F0181F333A4E556C0096F8F3
:1005300000E05D4BBEF13F0F04D994F850202846EF
:100540005A4906E05A494FEA4E1E94F85020284670
:100550007144012A4FE094F85020284696F9011082
:10056000022A52E096F802E04F4BBEF13F0F04D949
:1005700094F8502028464D4906E04D494FEA4E1E5A
:1005800094F8502028467144032A34E094F850200F
:10059000284696F90310042A37E096F804E0424B07
:1005A000BEF13F0F04D994F8502028463F4906E099
:1005B0003F494FEA4E1E94F8502028467144052AC0
:1005C00019E094F85020284696F90510062A1CE0F8
:1005D00096F806E0344BBEF13F0F04D994F8502052
:1005E0002846324906E032494FEA4E1E94F8502020
:1005F00028467144072A14BF0022012209E094F81A
:10060000502096F907102846082A2A4B14BF0022CA
:1006100001229847284B01371B78FFB2ED18EDB245
:100620009DF81F30BB423FF650AF6CE0B9F1080FA8
:1006300069D8DFE809F0050C0E1114171A555A0095
:100640001E4B01201870FF2384F851305CE01C48D9
:1006500048E01C4801324AE01B48023242E01B4895
:10066000033244E01A4804323CE01A4805323EE0C6
:1006700068010020915F000890040020656B00086D
:10068000673B0108053401080C8D0108795000080A
:1006900020010020BD380108A95E0008308D010846
:1006A000015A0008D95A0008415A0008CA7B0108BB
:1006B000C00E0020A95A00085C33002092000020E0
:1006C0001280010819800108288001082F80010884
:1006D0003E80010845800108143300206B3B01086F
:1006E0000B480632FF230B4D03E00B4807320B4D3E
:1006F000FF23A847012806D1094B1870FF2384F86F
:100700005130013800E0002009B0BDE8F08F00BF93
:1007100054800108416600085B8001080D670008ED
:10072000920000202DE9F04F844DDFF8AC8295F85F
:10073000559089B0B9F1FF0F8246144698F8496088
:1007400040F09B80084605F154020C2105F1550349
:100750007B4FB84795F854305046009379490C23A5
:100760000DF11F02784FB84798F84A30002B3DD062
:10077000DFF868A2D04798F84A30744A0593834658
:1007800090470746D047059B7A1EDB439B440121D7
:10079000431E0020D2B2009101905FFA8BF10290CB
:1007A0000390DBB26A4FB8476A4F95F8543057F858
:1007B0002300694B98478346D047684B98F84A20F6
:1007C0001B7898F84A10CDF80090CB1A03EBD3733E
:1007D000C2EB630195F85430411857F82320CDF847
:1007E00004905846C9B24B465D4FB847554B1F78E9
:1007F0003EE095F854103046CA1B514241EB0201CD
:10080000584B98470B2FDFF834812BD898F8542099
:10081000554B304653F82710D31B5A4242EB030284
:10082000524B98474FB998F864203D21D2F101020C
:10083000304638BF00224E4B13E0022F08D001D3C0
:100840000B2F0FD995F8542030462168012A04E077
:1008500098F8542021793046022A464B14BF0022D2
:1008600001229847444B01371B78FFB2F618F6B2C5
:100870009DF81F30BB42BCD85CE0B9F10B0F59D8D2
:10088000DFE809F0060D11161B21272D343B4248E5
:100890003A4B01201870FF2385F855304BE038485B
:1008A000FF23384C3CE038480432FF23374C37E014
:1008B00037484832FF23374C32E0374802F584721C
:1008C000FF23364C2CE0364802F5E472FF23354C0A
:1008D00026E0354802F54272FF23344C20E002F551
:1008E000805233480832FF23324C19E002F5885217
:1008F00031480832FF23314C12E002F59052304863
:100900000832FF232F4C0BE02F4802F59352FF23B0
:100910002E4C05E002F594522D482E4C2832FF2330
:10092000A047012806D1154B1870FF2385F85530D4
:10093000013800E0002009B0BDE8F08F6801002018
:10094000915F000861040020656B0008673B0108A7
:1009500005340108C0790108795000082001002001
:10096000BD380108A95E00085C8D0108015A000825
:10097000D95A0008A95A00085C33002092000020D0
:100980006A800108F9540008708001084166000877
:100990002C7B010881D40008317B0108C1D80008F4
:1009A0003A7B010815D00008877B010889DE000822
:1009B000417B0108A1E90008457B010811EE000810
:1009C0007A800108C5FB0008697F01089DF70008CF
:1009D00085800108FD030108143300206B3B0108EA
:1009E0002DE9F04F9E4DDFF8D88295F861908BB0DD
:1009F000B9F1FF0F8246144698F8496040F00D8126
:100A0000084605F16002082105F16103954FB847DA
:100A100095F8603050460093934908230DF1270262
:100A2000924FB84798F84A30002B3DD0DFF894A297
:100A3000D04798F84A308E4A059383469047074638
:100A4000D047059B7A1EDB439B440121431E0020B7
:100A5000D2B2009101905FFA8BF102900390DBB269
:100A6000844FB847844F95F8603057F82300834B84
:100A700098478346D047824B98F84A201B7898F8CD
:100A80004A10CDF80090CB1A03EBD373C2EB63018D
:100A900095F86030411857F82320CDF80490584657
:100AA000C9B24B46774FB8476F4B1F78AFE095F808
:100AB00060103046CB1B594241EB0301724B984703
:100AC000072FDFF89C8100F29C8098F860206F4B24
:100AD000C7EB020CDCF1000253F8271042EB0C02CA
:100AE00030466B4B98474FB998F864203D21D2F1BE
:100AF0000102304638BF0022664B81E0BB1E052B49
:100B000004D8DFE803F04B555B61677121684EF64E
:100B100060234FF00109B1FBF3F102220023DFF85B
:100B2000A8A109B2CDF8009007A8D047DFF89CB182
:100B3000594907A8D847DFF898C107A8CDF814C0CD
:100B4000E04722684FF47A78B2FBF8F23C23B2FB1C
:100B5000F3F103FB112307AA19B210180023022294
:100B6000CDF80090D0474C4907A8D847DDF814C00D
:100B700007A8E0472368CDF80090B3FBF8F208FB24
:100B8000123807AB032218180FFA88F10023D04758
:100B900095F86020304607A94A4504E095F86020A2
:100BA0003E493046022A14BF002201223C4B27E076
:100BB00095F860203046A188032A10E095F860205F
:100BC0003046E188042A0AE095F860203046217A10
:100BD000052A04E095F86020617A3046062A14BFA1
:100BE000002201222F4B0BE095F860202E4BA2F142
:100BF000070EDEF10002304604F10C0142EB0E025A
:100C000098472A4B01371B78FFB2F618F6B29DF8C9
:100C10002730BB423FF64BAF79E0B9F1070F76D8EA
:100C2000DFE809F0040B101B585D6167204B0120C1
:100C30001870FF2385F861306AE022461D48FF23C3
:100C40001D4C5BE0637A33B1012B0CBFA288E288B4
:100C50004FF47A735343236053E01848221D3BE05E
:100C600068010020915F000868040020656B00089F
:100C7000673B010805340108D48D0108795000084C
:100C800020010020BD380108A95E0008988E0108E7
:100C9000015A0008D95A00089E7A0108DD7E010831
:100CA000415A0008A95A00089D5D00085C330020E5
:100CB0009200002004860108F9540008CA80010847
:100CC000143300206B3B0108494500084916000811
:100CD0004D1700081048A21DFF23104C0EE01048CD
:100CE00004F1080202E00F4804F10902FF230E4C50
:100CF00004E004F10C020D480D4CFF23A04701282D
:100D000005D10C4B01221A70FF2385F861300020B9
:100D10000BB0BDE8F08F00BFD1800108415500083D
:100D2000D880010884760108416600081E85010804
:100D3000199B0008920000202DE9FF4194463B4B8F
:100D40003B4A93F8494092F863300746FF2B15461B
:100D500051D108466232032105F16303354EB04795
:100D6000DFF8F88095F86230064600933846414631
:100D7000314F0DF10F020323B84798F8007035E0AA
:100D800095F862102046CB1B594241EB03012B4BD7
:100D9000DFF89C8098474FB998F862102046D1F14F
:100DA000010138BF0021264B984719E0022F17D8C0
:100DB00098F862202046C7EB020CDCF1000242EBFF
:100DC0000C022049204B984798F86220791EC7EB07
:100DD000020EDEF10002204642EB0E021B4B98474A
:100DE0001B4B01371B78FFB2E418E4B29DF80F30BB
:100DF000BB42C5D80EE033B9164B01201870FF2353
:100E000082F863300EE0013B0CEB0312124CDBB2B4
:100E1000A0470646012E04D10E4B1E70FF2385F815
:100E20006330002004B0BDE8F08100BF143300201F
:100E300068010020915F0008656B0008A95E00084A
:100E4000555F000850860108015A0008A95A000899
:100E50005C33002092000020E1090108A304002077
:100E60002DE9F04F7C4CDFF86C8294F8659089B0E6
:100E7000B9F1FF0F8246154698F8496040F0A4800A
:100E8000084604F16402082104F16503734FB84772
:100E900094F8643050460093714908230DF11F0205
:100EA000704FB84798F84A30002B3DD0DFF828A2A1
:100EB000D04798F84A306C4A0593834690470746D6
:100EC000D047059B7A1EDB439B440121431E002033
:100ED000D2B2009101905FFA8BF102900390DBB2E5
:100EE000624FB847624F94F8643057F82300614B63
:100EF00098478346D047604B98F84A201B7898F86B
:100F00004A10CDF80090CB1A03EBD373C2EB630108
:100F100094F86430411857F82320CDF804905846CF
:100F2000C9B24B46554FB8474D4B1F7847E094F830
:100F300064103046CA1B514241EB0201504B9847A6
:100F4000072FDFF8148134D898F864204D4B3046D1
:100F500053F82710D31B5A4242EB03024A4B9847DF
:100F600047B998F864203D21D2F10102304638BFDC
:100F700000221CE0022F0FD001D3072F19D994F8BB
:100F800064203046A2F1010CDCF1000205F11801E9
:100F900042EB0C023D4B0BE098F8642095F92810C9
:100FA000A2F1020EDEF10002304642EB0E02384B97
:100FB0009847384B01371B78FFB2F618F6B29DF808
:100FC0001F30BB42B3D843E0B9F1070F40D8DFE888
:100FD00009F0040B10151A21282F2F4B012018702F
:100FE000FF2384F8653034E02C481832FF232C4D61
:100FF00024E02C482832FF232B4D1FE02B482C32B5
:10100000FF232B4D1AE002F502622A480C32FF231F
:10101000294D13E002F5626228480C32FF23284D67
:101020000CE002F58C5227482C32FF23264D05E0B8
:1010300002F510522548264D5C32FF23A8470128AF
:1010400006D1154B1870FF2384F86530013800E095
:10105000002009B0BDE8F08F68010020915F000812
:10106000AA040020656B0008673B010805340108ED
:10107000547801087950000820010020BD3801088B
:10108000A95E000884780108015A0008415A000846
:10109000D95A00085C330020920000200989010819
:1010A00015560008318401084D6100080B7F0108C6
:1010B000B5E400081D7F01084DF30008E584010830
:1010C00041CC0008DD8001082507010804860108DD
:1010D000390D0108143300206B3B01082DE9F04F56
:1010E0007F4C804E94F86D8087B0B8F1FF0F814639
:1010F00096F8495040F0B580084604F16C020A2188
:1011000004F16D03784FB84794F86C30484600936B
:1011100076490A230DF11702754FB84796F84A3001
:10112000002B3CD0DFF83492C847724B96F84AB097
:10113000824698470746C8476FEA0B0BDA447A1E87
:10114000431E01210020D2B2009101905FFA8AF182
:1011500002900390DBB2684FB84794F86C30674F49
:1011600057F82300664B98478246C847654B96F868
:101170004A201B7896F84A10CDF80080CB1A03EB72
:10118000D373C2EB630194F86C30411857F82320F5
:10119000CDF804805046C9B243465B4EB047534B2E
:1011A0001E7859E094F86C1028468A1B514241EB96
:1011B0000201564B9847092E494F47D897F86C20A3
:1011C000534B284653F82610931B5A4242EB030216
:1011D000504B98474EB997F864203D21D2F1010257
:1011E000284638BF00224C4B2FE0B31E072B05D8F2
:1011F000DFE803F00A10161C2C2C2C2294F86C202B
:1012000028464649012A1CE094F86C2028464349A8
:10121000022A16E094F86C2028464049032A10E080
:1012200094F86C2028463D49042A0AE094F86C2082
:1012300028463A49052A04E094F86C2037492846A4
:10124000092A374B14BF002201229847354B01363B
:101250001B78F6B2ED18EDB29DF81730B342A1D865
:101260003AE0B8F1090F37D8DFE808F0050C0F12A3
:1012700015181B1F242A2C4B01201870FF2384F8FB
:101280006D302AE00846294B1CE00846284B19E03F
:101290000846284B16E00846274B13E00846274B24
:1012A00010E02748FF23274D08E027482032FF237E
:1012B000264D03E02648274D4832FF23A84702E089
:1012C000254B08469847012806D1174B1870FF2375
:1012D00084F86D30013800E0002007B0BDE8F08FE1
:1012E0006801002014330020915F00085E04002094
:1012F000656B0008673B010805340108B8780108F0
:101300007950000820010020BD380108A95E0008BE
:10131000B0770108015A0008D95A0008DD7E01089B
:10132000415A00085C33002092000020619E0008B2
:10133000A9A1000811C200080DC60008E5C70008F1
:101340007B8601082D020108F57B0108EDFC0008F1
:10135000E4800108F5FF00080DA500086B3B0108BB
:101360002DE9F04F604C614E94F8718087B0B8F170
:10137000FF0F814696F8495040F08880084604F1F6
:101380007002042104F17103594FB84794F870308A
:1013900048460093574904230DF11702564FB847AA
:1013A00096F84A30002B3CD0DFF89891C847534B51
:1013B00096F84AB0824698470746C8476FEA0B0B33
:1013C000DA447A1E431E01210020D2B2009101901E
:1013D0005FFA8AF102900390DBB2494FB84794F864
:1013E0007030484F57F82300474B98478246C8470C
:1013F000464B96F84A201B7896F84A10CDF80080A4
:10140000CB1A03EBD373C2EB630194F8703041182D
:1014100057F82320CDF804805046C9B243463C4ECD
:10142000B047344B1E782CE094F870102846C6EB79
:10143000010CDCF1000141EB0C01364B9847032E07
:10144000294F18D897F87020334BC6EB020EDEF107
:10145000000253F8261042EB0E0228462F4B984705
:101460004EB997F864203D21D2F10102284638BFD9
:1014700000222B4B98472B4B01361B78F6B2ED1808
:10148000EDB29DF81730B342CED828E0B8F1030F83
:1014900025D8DFE808F002090D14234B012018704D
:1014A000FF2384F871301BE02048FF23204D0CE01F
:1014B00002F512521F480832FF231F4D05E002F5C6
:1014C00012521E481E4D0C32FF23A847012806D198
:1014D000154B1870FF2384F87130013800E00020AC
:1014E00007B0BDE8F08F00BF680100201433002072
:1014F000915F000863040020656B0008673B0108EA
:1015000005340108407A01087950000820010020C4
:10151000BD380108A95E0008D8770108015A000803
:10152000D95A00085C33002092000020A9820108EB
:10153000610E0108EC800108F9BB0008F380010886
:10154000DD1001086B3B01082DE9F04F0F4C9BB0FB
:1015500023788246FF2B41F0EE81042804D02346F5
:101560000F210B4A0B4CA047094BDFF838801F783E
:10157000094C012F094DDFF8309017D0022F084F8A
:1015800007F5105640F06985BDE300BF93000020C9
:101590009B040020915F0008673B01086B3B01083A
:1015A000940E00203961000805340108A548C047A1
:1015B000A0470646A847DFF8C8A2721E431E0026B1
:1015C000009730460921D2B2DBB20196029603960B
:1015D000C847BAF838103B46009709B23246DFF8E0
:1015E000A4B215A8D8479849984A15A89047984B8F
:1015F00015A89847BAF854100DF1540C3B466044B6
:101600003246009709B2D847FF27924915A8884764
:101610003B460B2115AADFF870C200970197E047FF
:10162000A04740085FFA80F9A8478046A8470938D4
:1016300000EBD070A8F10908401008EBD8780D38FD
:101640004FEA680880B2DFF834C208F109085FFA8F
:1016500080FE5FFA88F80790009701973B46CDF827
:1016600020E0484641467246CDF810C0E047374674
:101670003846794B9847FF260F370346009001966E
:101680000296039648464146089ADFF8ECC1BFB27D
:10169000E047B7F5B47FEBD1DDF820E04FF0000B69
:1016A000AEF10502484641466C4FD2B25B46CDF8DA
:1016B00000B0CDF804B0B847DDF820E0DFF8CCA1E9
:1016C000AEF1040C5FFA8CFC484641466246CDF808
:1016D00028C05B46CDF800B0CDF804B0B8470AF595
:1016E0008651088F0B8F5E4F0993089B00B29A1E9C
:1016F0005FFA82FCCDF810C0B8475A4A5A49904761
:101700005A4F5B49B847DDF824E0034605930FFACA
:101710008EF053498847534A534990475449B84734
:10172000DDF810C0414662460090DFF84CC14846E3
:10173000019602960396059BE0470AF58851888A30
:101740008B8A00B21A460692454B9847DFF814C1BF
:101750004549E0474649B8474FF07E51454B9847C9
:10176000069A0346059310B23D4988473D4A3E49D3
:1017700090473F49B8474FF07E51B84741460090E7
:1017800001964846029603960A9A059B3A4FB84737
:10179000DDF820C04846ACF10707FFB241463A46A3
:1017A000DFF8B8C05B46CDF800B0CDF804B0E04734
:1017B000484641463A463346009601962F4FB84771
:1017C000DDF81CE0BAF8381F4FEA5E0CBAF8383F73
:1017D0005FFA8CFCCCEB0900079ACDF820C009B267
:1017E000DDF81CC01BB2A1F50071A3F500735143D5
:1017F00003FB0CF30327BEFBF7FE5FFA8EF791FBAA
:10180000F6F193FBF6F3C7EB09024144434400961B
:1018100001960296C0B2C9B2D2B2DBB2DFF870C094
:10182000E047BAF8382FBAF8383FDDF81CC011B2DB
:101830001BB2079AA1F50071A3F50073514303FB96
:101840000CF327E0E5840108FA8001084916000836
:101850004D170008A5500008BD2A000839390108B5
:10186000C52A0008D52C0008000020415D29000889
:101870000000B44259290008653B0108513A0108AB
:10188000541F00204945000875380108940E0020B7
:1018900009370108DDF820E091FBF6F193FBF6F340
:1018A0000EEB090007EB090241444344D2B2009613
:1018B00001960296C0B2C9B2DBB2DFF864C2E0475B
:1018C000BAF8383FDDF81CE01BB2A3F5007303FB48
:1018D0000EF3BAF81C0F93FBF6F3BAF81CCF053FD2
:1018E0004344DBB2FFB200B2CDF810C009930897B1
:1018F0007D49A0F5007088477C4A90477C4F0022C4
:101900004FF07E53B84774A3D3E90023B847794B0F
:101910009847DDF810C00A900FFA8CF0A0F500701F
:10192000DFF8C4C1E047714A904700224FF07E5370
:10193000B84769A3D3E90023B8476E4B9847DFF84F
:10194000B8C1009001964846029603960999089AF4
:101950000A9BE047BAF8382FDDF81CE012B2A2F576
:10196000007202FB0EF2BAF81C0F92FBF6F2BAF804
:101970001C3F90445FFA88F800B20993CDF81C80B0
:101980005949A0F500708847584A904700224FF007
:101990007E53B84750A3D3E90023B84750A3D3E9F7
:1019A0000023DFF88081C047524B9847DDF824E0E0
:1019B00084460FFA8EF0CDF810C04B49A0F50070A8
:1019C00088474A4A904700224FF07E53B84742A3C7
:1019D000D3E90023B84742A3D3E90023C047454BCE
:1019E0009847DDF810C0009063464846019602967D
:1019F00003960799089A404EB047A847BAF8007F67
:101A00000D3880B2BFB207905646DFF814913B4BB9
:101A100097B915A83A4998473A4B3A4619880A2384
:101A200089B2B1FBF3F1093B00930DF1570009B204
:101A30000133354FB84714E0344915A89847B6F834
:101A4000001F4FF47A7309B2890291FBF3F101236D
:101A500000930DF1570009B25A46DB18DFF8A8C011
:101A6000E0472B492B4A15A890472B4B15A89847C0
:101A70000746A847FF23A0F10901284D38460093E7
:101A80000193C9B215AAA847079F00254FEA570836
:101A9000A8F102080B271AE06B01F31893F83E2017
:101AA000394652B2002AB8BF0F321211FF230A3250
:101AB0000093019302930A203B46D2B201350237CC
:101AC000C847402DFFB202D10B2700254FE0454506
:101AD000E2DBF9E7AFF30080000000000080464041
:101AE0000000000000806640C52A0008452200086A
:101AF000ED220008B1280008653B01089116000896
:101B0000FC800108CE06002049450008008101083C
:101B1000AA86010849160008A55000087538010872
:101B200009370108891F0008A0478246A0471823EB
:101B300003FB056303F5026318339B88AAF10A0AC5
:101B40001BB2002BB8BFFF331B120A3BC2185FFA4F
:101B50008AFAFF2300930193029339463B4650468D
:101B6000D2B201350237C847402DFFB201D04545FA
:101B7000DADBB6F8742EDDF81CC00327BCFBF7F7E0
:101B8000642112B2FB1D4A4348BF1F32DFF80884AC
:101B9000521119254FF0320BD2B2DFF8009408939E
:101BA0000092CDF804B00295CDF80C8014200B21E2
:101BB0002A461BB2C84707F10B037F00BFB2099347
:101BC000FB1D0A93B6F8583E4FF0640A1BB20AFB9D
:101BD00003F3FF22DDF824E0029593FBF2F32A469B
:101BE0000A9DDBB20FFA8EF10093CDF804B0CDF868
:101BF0000C8014202BB2C847B6F8902E504612B273
